:100000000C94E00F0C9408100C9408100C94081039
:100010000C9408100C9408100C9408100C94081000
:100020000C9408100C9408100C9412150C943F6654
:100030000C94BD680C946E660C9408100C947115A9
:100040000C9400150C9408100C94C96C0C940810B6
:100050000C9408100C9408100C9408100C940810C0
:100060000C942F690C94B9150C94D8660C946F6994
:100070000C9408100C9408100C9408100C940810A0
:100080000C9408100C9408100C9408105217561772
:1000900019171F172517251725174A174E17521717
:1000A00056175A175E176217723D323D3D3D4C3D63
:1000B000523D563D5B3D48425E426C4281428F421A
:1000C0009E42B042D642FF420D43334351435F4309
:1000D0006D437B432C61166110611A611F612561BC
:1000E000136129612E61D16AD76AE46AED6A036BF4
:1000F0001C6B2F6B3E6B526B676B706B8D6B936BD6
:100100009B6BA06BA56B0D6C176CAD6BB46BBE6B72
:10011000C86BCE6BD26BD96BF46BF96BFE6B066C54
:10012000DD6ADD6BE46BEC6BF96CFB6D146D196DC6
:10013000FB6D2E6D336DFB6D486D4D6DFB6D626D0E
:10014000676DFB6D7C6D816DFB6D966D9A6DB06D0D
:10015000B26DB46DB66DBA6D204F6C642056657289
:1001600073696F6E20454550524F4D202020434803
:1001700045434B2053455454494E47532F43414C1C
:10018000494200416C61726D732044697361626C15
:10019000656400506C6561736520526573657420F9
:1001A0005377697463686573005468726F74746C14
:1001B00065206E6F742069646C65005265736574A8
:1001C000207468726F74746C6500454550524F4DD1
:1001D000206C6F77206D656D004C4F4144494E4750
:1001E000006D537461636B206F666C6F77006D53A5
:1001F0007461636B2075666C6F77004D4553534196
:10020000474500414C45525400707265737320613C
:100210006E79204B657900507265737320616E7939
:10022000206B657920746F20736B697000414C45B9
:10023000525400034F46464142535255735255257E
:10024000454C73454C25544873544825414C7341E3
:100250004C2550312050312550322050322550331A
:100260002050332500544852525544454C4549448A
:100270003049443149443241494C47454154524E3A
:1002800053573153573253573353573453573553CA
:100290005736535737535738535739535741535796
:1002A00042535743002D2D2D004348002D2D2D2066
:1002B000000450312020503220205033202048416B
:1002C0004C4646554C4C43594331435943324359AC
:1002D000433350504D3150504D3250504D335050AB
:1002E0004D3450504D3550504D3650504D37505084
:1002F0004D38434831204348322043483320434857
:10030000342043483520434836204348372043486B
:10031000382043483920434831304348313143483D
:10032000313243483133434831344348313543480F
:10033000313633504F5347563120475632204756B7
:1003400033204756342047563520475636204756E7
:100350003720002D2D2D2D000000642810070301EB
:1003600052554420454C45205448522041494C2088
:100370000001020304010302040402030104030256
:10038000014F4E20004F4646001B1E272D36394B8D
:100390004E636C7278878D939CB1B4C6C9D2D8E194
:1003A000E453706C6173680080400000000000003E
:1003B000000000000000000000000000000000003D
:1003C000000000000000000000000000000000002D
:1003D000000000000000000000000000000000001D
:1003E000000000000000000000000000000000000D
:1003F000000000000080C0E0E0F0F8F8FCFCFCF831
:10040000F8F8F0400000000000808080000000004C
:10041000000000000000000000000000000000805C
:10042000C0C0E0E0E0F0F0F0E0C00000000000C07C
:10043000F8FFFF9F878383838383838383838383FF
:1004400083838383838383838383830383808383FF
:10045000838383838383838383838383838383836C
:100460008383838383C3E3733F1F0000000080E026
:10047000F0F8FCFEFFFFFFFF7F3F1F1F0F0783C346
:10048000E1E1E0E0C0000E1F3F7F7FFFF3E0E0808E
:100490000000000000000000000080F0FCFEFFFFF4
:1004A000FFFF7F3F0F0301010100000080F0FEFF0E
:1004B000FFC7C1C1C1C1C1C1C1C1C1C1C1C1C1C1E8
:1004C000C1C1C1C1C1C1C1C101C1F0FEFF3F0F0720
:1004D0000F0D0D0D1D19191919313131317161616E
:1004E00061E1C1C1C18100000080E0F8FCFFFFFFB5
:1004F000FF2F170F038180C0E0F0F8FCFEFFFFFF25
:10050000FFFFFF7F01000000000000000101030762
:10051000070E1E1C3870E0F0F8FEFFFF7F1F0F0370
:1005200000010000000000000000000000000000CA
:1005300000000000000000000000000000000000BB
:1005400000000000000000000000000000000000AB
:10055000000000000000000000000000000000009B
:1005600000000000000000007EFFFFFFFFFFFFFB18
:10057000F8FCFCFEFF7F3F1F0F07C3FFFFFFFFFFDD
:10058000FF7F0700000000000000000000000000E6
:1005900000C0E0F8FEFFFF7F1F0F1F3D7CF8F8F062
:1005A000E0800000000000000000000000000000EB
:1005B000000000000000000000000000000000003B
:1005C000000000000000000000000000000000002B
:1005D000000000000000000000000000000000001B
:1005E0000000000000000000000001010101010303
:1005F0000707070301000000E0FCFFFFFFFFFF1FEC
:10060000030000000000000000000000C0F078DEE1
:100610002713090E0703000000000000000001037B
:100620000F7FFFFC7878F800000000000000000059
:1006300000008080808080808080800080800080BA
:10064000800000000000000080808080808080802A
:10065000808080808080808080800000000000009A
:10066000000000000000000000000000000000008A
:10067000000000000080F0FEFFFFFFFF3F0F0100C1
:1006800000000000000000C0E0381E0F0300010061
:10069000000000000000000000000000000000005A
:1006A0000000000000030301000000000000000043
:1006B00000000E0E02020202020303000F0F000FE1
:1006C0000F080808080808080F0F08080808080F8E
:1006D0000F000000000F0F000000000000000000ED
:1006E000000000000000000000000000000000000A
:1006F000000000C0F8BFFFFFFF1F7F0100000000E7
:1007000000000000F0FCFF7F7830000000000000D7
:1007100000000000000000000000000000000000D9
:1007200000000000000000000000000000000000C9
:1007300000000000000000000000000000000000B9
:1007400000000000000000000000000000000000A9
:100750000000000000000000000000000000000099
:100760000000000000000000000000000000000089
:1007700000301C070E0F0701000000000000000001
:100780000000000000000000000000000000000069
:100790000000000000000000000000000000000059
:1007A0000000000000000000000000204D4F443A0F
:1007B00020415244552020202020002053564E3AFC
:1007C00020657239782D723739310054494D453AD8
:1007D0002032313A31333A333100444154453A20E2
:1007E00031312E30352E3230313300564552533AA6
:1007F0002056312E3635382D4D696B650022047C2C
:100800005E54546D0003457870457846466E654DDC
:1008100065644372730011544F54000153544B11DB
:100820005354250001544D4511545357005354411E
:100830005400035B4D454E555D20746F2072656614
:100840007265736800746D61696E0F6D7300746D0D
:100850007231204A69747465720F757300746D7219
:10086000314C6174206D696E0F757300746D723157
:100870004C6174206D61780F75730053544154328C
:10088000004D6F64650043726F73735472696D003D
:10089000456E61626C652050504D53494D00426178
:1008A0006E6447617000537469636B5363726F6C5D
:1008B0006C00506F745363726F6C6C00416C6172AA
:1008C0006D205761726E696E67004D656D6F72794C
:1008D000205761726E696E670044656661756C745D
:1008E000205377005468726F74746C65205761727E
:1008F0006E696E670053706C617368204E616D6540
:100900000053706C6173682073637265656E004C90
:1009100069676874206F6E2053746B204D76004CAD
:1009200069676874206F666620616674657200424C
:1009300061636B6C6967687420696E7665727400B8
:100940004C696768742073776974636800466C61EA
:100950007368206F6E206265657000426565702067
:10096000636F756E74646F776E004D696E75746534
:100970002062656570005468726F74746C652072D3
:1009800065766572736500496E6163746976697432
:100990007920616C61726D136D00426174746572CF
:1009A00079207761726E696E6700436F6E74726151
:1009B0007374002048617074696320537472656EAB
:1009C0006774680020537065616B657220506974AC
:1009D000636800566F6C756D65000A4265657065E9
:1009E0007220202020506953706B722020202042FA
:1009F00065657072566F696365506953706B566FA9
:100A000069636500536F756E64204D6F6465000601
:100A10005175696574204E6F4B6579207853686F06
:100A2000727453686F7274204E6F726D20204C6F19
:100A30006E672020784C6F6E672000426565706598
:100A400072004F776E6572204E616D6500524144B1
:100A5000494F20534554555000036D6F64650A2576
:100A600020737263202073770043616C004D756CB6
:100A70007469706C6965720003636831636832631E
:100A8000683363683400036F6666202B3D203A3D6F
:100A90000007536C617665000003030303005452A2
:100AA00041494E45520056455253494F4E005472EB
:100AB000696D2D202B0005204D656E7520457869E8
:100AC0007420446F776E20202055705269676874D7
:100AD000204C656674004449414700424700414E3E
:100AE0004100034D4F564520535449434B532F501B
:100AF0004F54530005534554204D4944504F494EDF
:100B00005400035B4D454E555D20544F20535441D6
:100B100052540043414C4942524154494F4E0009FE
:100B200066726565004D4F44454C53454C00434F3C
:100B30004C20446972656374696F6E0041494C20B2
:100B4000446972656374696F6E00454C4520446961
:100B500072656374696F6E005377617368205269C0
:100B60006E6700436F6C6C65637469766500062D73
:100B70002D2D2020203132302020203132305820BD
:100B8000203134302020203930202020200053779D
:100B90006173682054797065000048454C492053C2
:100BA0004554555000464D00464D300F5245544176
:100BB000004D4F444553005472696D73005377697B
:100BC000746368000003464C204D4F4445000152B9
:100BD0004554410044454C455445204D4F44454CF7
:100BE0000F5B4D454E555D00543254685472696731
:100BF00000547261696E657200452E204C696D6902
:100C000074730003504F534E454700536869667430
:100C10002053656C0050504D20317374204368613F
:100C20006E004C50342F4C5035202044534D326FC1
:100C30006E6C792044534D322F44534D5800445329
:100C40004D20547970650053656E64205278204EB3
:100C5000756D626572205B4D454E555D0050504D7F
:100C60002046724C656E0D6D536563000B52784ED5
:100C7000756D0004344348203643482038434820EB
:100C800031304348313243483134434831364348A8
:100C9000001375530011755365630050504D2020AB
:100CA0002050585820202044534D32202050504D81
:100CB00031362050504D53494D0050726F746F00C3
:100CC00052455441313233004265657020436E74A1
:100CD000005472696D2053770006457870202020FB
:100CE000457846696E6546696E6520204D65646984
:100CF000756D436F61727365005472696D20496E42
:100D00006300542D4578706F00542D5472696D0046
:100D10000A436F756E7420446F776E436F756E74FF
:100D20002055702020005472696767657242005434
:100D300072696767657200566F69636520496E6402
:100D40006578114D454E55004E616D6500000900F6
:100D500001000000000000000602005345545550F9
:100D6000004475706C69636174696E67206D6F64AF
:100D7000656C0044454C455445204D4F44454C005E
:100D80004455504C4943415445204D4F44454C0037
:100D9000657870202025202073773120737732000A
:100DA00000034558504F2F44520044522048696771
:100DB00068004452204C6F77004452204D69640013
:100DC0004472537732004472537731005765696734
:100DD0006874004578706F00004558504F2F44529A
:100DE00000012B2A52004D4958455200032044452A
:100DF0004C455445200003204D4F564520202000EF
:100E00000320434F5059202020000320494E5345D2
:100E100052542000032045444954202020004445DA
:100E20004C455445204D49583F00035B4D454E55B8
:100E30005D0B5B455849545D00035945530B4E4FBC
:100E4000005072657373205B455849545D20746F80
:100E50002061626F7274004D6178206D69786572EF
:100E6000732072656163683A2033320002536C6FFD
:100E700077202055700002536C6F772020446F77E5
:100E80006E000244656C6179205570000244656C07
:100E9000617920446F776E0008416464202020202F
:100EA000204D756C7469706C795265706C61636506
:100EB0002000024D756C74707800025761726E6983
:100EC0006E670002537769746368004375727665D4
:100ED000000D4469666600025472696D0002466C3A
:100EE0004D6F64657472696D0002466978204F66C3
:100EF00066736574004F666673657400466D547260
:100F0000696D56616C000257656967687400025329
:100F10006F757263650045444954204D495820005F
:100F2000494E53455254204D49582000032D2D2D34
:100F3000783E30783C307C787C663E30663C307C55
:100F4000667C633120633220633320633420633551
:100F500020633620633720633820633920633130C3
:100F6000633131633132633133633134633135633B
:100F70003136000E4F6E00072D2D2D2D20202076AE
:100F80003E6F66732020763C6F667320207C767CF3
:100F90003E6F66737C767C3C6F6673414E442020C6
:100FA00020204F522020202020584F522020202047
:100FB00076313D3D7632207631213D7632207631D4
:100FC0003E7632202076313C7632202076313E3D0E
:100FD00076322076313C3D76322054696D654F661D
:100FE00066005357000003435553544F4D20535749
:100FF00049544348455300064F4E202020204F4679
:1010000046202020424F54482020313553656373D9
:101010003330536563733630536563735661726959
:10102000626C0056530007203820536563733132D9
:10103000205365637331362053656373004E756DBD
:1010400062657220566F6963652053770000000265
:10105000534146455459205357495443484553003A
:10106000434C454152204D49584553205B4D454E18
:10107000555D00205245544100014368616E6E6524
:101080006C204F726465720054454D504C4154457C
:101090005300032D2D2D52746D45746D54746D41A4
:1010A000746D52454E525544454C45544852414941
:1010B0004C50312050322050332063312063322095
:1010C0006333206334206335206336206337206325
:1010D0003820633920633130633131633132633119
:1010E00033633134633135633136004756000001D4
:1010F000474C4F42414C205641525300434F5059A8
:10110000205452494D205B4D454E555D0000034C27
:10111000494D4954530043560043555256455300D8
:1011200050524553455400454449542D3E00090052
:10113000435552564500032D2D2D494E5600475616
:10114000005B4D454E555D205748454E20444F4E5F
:101150004500EF46B024DF236423E422612661309A
:10116000AF4D1752142F182D2945D05297432B4CB1
:101170002E545D440D2412081200081C0808081C97
:101180000800000822004900220800000000002298
:101190007F220000000822004900220800000822E7
:1011A0000049002208000000227F22000000000009
:1011B000082200490022080000081C0808081C0832
:1011C00000065761726E31205761726E322043689B
:1011D0006561702052696E672020536369466920FB
:1011E000526F626F74204368697270205461646149
:1011F0002020437269636B74536972656E20416C81
:101200006D436C6B5261746174615469636B20202F
:1012100048617074633148617074633248617074FE
:1012200063330054696D6572005452453031324168
:101230004700204142434445464748494A4B4C4DAC
:101240004E4F505152535455565758595A61626334
:101250006465666768696A6B6C6D6E6F70717273D6
:101260007475767778797A30313233343536373869
:10127000395F2D2E00FEFFFDF6F7F8F9FAFBFC04AE
:101280002D2D2D2D54494D3154494D324241545448
:1012900047767231477672324776723347767234C8
:1012A00047767235477672364776723700537769DC
:1012B000746368205761726E696E670067656E7748
:1012C00072697465206572726F7200454550524FA5
:1012D0004D20466F726D617474696E67004261647F
:1012E00020454570726F6D2044617461004D4F441C
:1012F000454C2020202020004D452020202020206B
:10130000202000454550524F4D206F766572666C27
:101310006F7700A060800000000000000000000067
:1013200000000000FFFF0000000000001F3F000061
:101330003F1F00003030FFFF3030FFFF303030788B
:10134000CCCCFFFFCCCC8C0C060F0F86C0E07038E5
:101350001C0C3CFEC7E3F33B1E0C00000000333BBB
:101360001F0F000000000000F0F81C0E0703000033
:10137000000003070E1CF8F000003030E0C0FCFC59
:10138000C0E03030C0C0C0C0FCFCC0C0C0C0000065
:101390000000000000000000C0C0C0C0C0C0C0C04D
:1013A000C0C000000000000000000000000000803D
:1013B000C0E070381C0C00000000000000000000BD
:1013C00000000000383800000000000000000000AD
:1013D0000000000003033F3F03033F3F03030C0CE7
:1013E0000C0C3F3F0C0C07030C0E07030100183CCC
:1013F0003C180F1F383133331E1E333300000000FA
:10140000000000000000000003070E1C3830000040
:10141000000030381C0E07030000030301000F0F0B
:1014200000010303000000000F0F00000000000097
:10143000333B1F0F00000000000000000000000010
:1014400000000000183C3C18000000000C0E0703D0
:101450000100000000000000FCFE87C3E377FEFCF3
:1014600000000C0EFFFF0000000000000C0E0783C0
:10147000C3E77E3C00000303C3C3C3E7FE3C000098
:10148000C0E070381C0EFFFF00003F3F3333337362
:10149000E3C30000FCFEC7C3C3C78E0C00000303F8
:1014A000C3E3733B1F0F00003CFEE7C3C3E7FE3CF2
:1014B00000003C7EE7C3C3E7FEFC0000183C3C187C
:1014C000000000000000183C3C1800000000000074
:1014D000C0E0F0381C0E0703303030303030303090
:1014E000303003070E1C38F0E0C000000C0E07037C
:1014F0000383C3E77E3C00000F1F3B3130381F0FD2
:10150000000030303F3F3030000000003C3E3733B9
:101510003130303000003030303030391F0F0000B3
:101520000303030303033F3F00000C1C3830303833
:101530001F0F00000F1F383030391F0F0000000050
:101540003F3F0000000000000F1F393030391F0FEF
:101550000000000030381C0E07030000060F0F06C5
:10156000000000000000333B1F0F000000000000DF
:10157000000103070E1C38300303030303030303B6
:10158000030330381C0E07030100000000000000B8
:1015900033330100000000003C7EE7C3C3E77E3C1C
:1015A000F0F8DCCEC7C7CEDCF8F0FFFFC3C3C3C37F
:1015B000C3E7FE3CFCFE0703030303070E0CFFFF1B
:1015C000030303070E1CF8F0FFFFC3C3C3C3C3C369
:1015D0000303FFFFC3C3C3C3C3C30303FCFE07036B
:1015E000C3C3C3C7CECCFFFFC0C0C0C0C0C0FFFFD5
:1015F00000000303FFFF03030000000000000303DB
:10160000FFFF0303FFFFC0E0F0381C0E0703FFFFDE
:101610000000000000000000FFFF0E1CF8F81C0E88
:10162000FFFFFFFF3870E0C08000FFFFFCFE0703F4
:1016300003030307FEFC00000000000000000000A0
:101640003F3F0000000000003F3F3F3F3030303060
:1016500030391F0F0F1F3830303030381C0C3F3FEF
:10166000303030381C0E07033F3F303030303030E0
:1016700030303F3F00000000000000000F1F3830F6
:10168000303030303F3F3F3F0000000000003F3F20
:10169000000030303F3F303000000C1C3830303814
:1016A0001F0F00003F3F000103070E1C38303F3F73
:1016B00030303030303030303F3F0000000000002C
:1016C0003F3F3F3F0000000103033F3F0F1F383003
:1016D000303030381F0FFFFFC3C3C3C3C3E77E3CA6
:1016E000FCFE070303030307FEFCFFFFC3C3C3C3E2
:1016F000C3E77E3C3C7EE7C3C3C3C3C78E0C030372
:101700000303FFFF03030303FFFF000000000000CB
:10171000FFFFFFFF000000000000FFFFFFFF0000D1
:1017200000000000FFFF0F1F38F0E0E0F0381F0F4F
:101730003F7FE0C08080C0E07F3F03030383C3E3BB
:10174000733B1F0F0000FFFF0303030300000C1C8B
:101750003870E0C080000000000003030303FFFFB7
:10176000000030381C0E07070E1C38300000000047
:101770000000000000003F3F0000000000000000EB
:101780000F1F383033371E1C3F333F3F0000030725
:101790000E1C38300C1C3830303030391F0F000030
:1017A00000003F3F000000000F1F3830303030385D
:1017B0001F0F03070E1C38381C0E07030F1F383885
:1017C0001F1F38381F0F3C3E0703010103073E3C33
:1017D000000000013F3F010000003C3E3733313044
:1017E0003030303000003F3F3030303000000000FB
:1017F0000000000103070E0C0000303030303F3F86
:101800000000000000000000000000003030303018
:10181000303030303030000003070E1C383000000C
:101820000000303030303070E0C0FFFFC0E070307A
:101830003070E0C0C0E07030303030300000C0E0C8
:1018400070303070E0C0FFFFC0E07030303030707A
:10185000E0C0C0C0FCFEC7C303070E0CF0F89C0C30
:101860000C0C0C0CFCFCFFFFC0E070303070E0C0D2
:1018700000003030F3F300000000000000003030C2
:10188000F3F30000FFFF0080C0E0703000000000B4
:101890000303FFFF00000000F0F03070E0E0707024
:1018A000E0C0F0F0C0E070303070E0C0C0E07030F8
:1018B00030303070E0C00000000000000000000088
:1018C0000C1E3F33333333333F3F3F3F30303030F4
:1018D00030381F0F0F1F3830303030381C0C0F1FBE
:1018E0003830303030303F3F0F1F3B3333333333EA
:1018F000030300003F3F00000000000000013333FD
:101900003333333B1F0F3F3F0000000000003F3FD9
:10191000000030303F3F303000000C1C3830303891
:101920001F0F00003F3F03070F1C3830000000006E
:1019300030303F3F303000003F3F000003030000E5
:101940003F3F3F3F0000000000003F3F0F1F383087
:10195000303030381F0FF0F03030303030F0E0C031
:10196000C0E0F0303030E0C0F0F0F0F0C0E07030B7
:101970003070E0C0C0E0F030303030300000303047
:10198000FFFF303000000000F0F000000000000019
:10199000F0F0F0F0000000000000F0F0F0F00000C7
:1019A00000000000F0F03070E0C08080C0E07030D7
:1019B000F0F0800000000000F0F03030303030B047
:1019C000F0F070300000C0E03C3E07030000000073
:1019D0000000FFFF00000000000003073E3CE0C0E5
:1019E0000000C0C0C0C00C1CF8F0E0C0C0E0F0F8BF
:1019F0001C0CC0C0C0C03F3F03030303030301002E
:101A000000010303030303033F3F3F3F00000000C7
:101A100000000000303133333333333F1E0C0000FD
:101A20000F1F383030381C0C0F1F383030381C0C6A
:101A30003F3F03070E1C38381C0E07030F1F3838B2
:101A40001C1C38381F0F30381C0F07070F1C38308C
:101A5000000133333333333B1F0F30383C3E3733D1
:101A600031303030000000010F1F3830000000001E
:101A700000003F3F00000000000030381F0F010051
:101A80000000000000000C0E070301000001030726
:101A90000E0C000000005008500000000000000084
:101AA000006F000007000700147F147F14242A7FB2
:101AB0002A12231308646236495522500005030098
:101AC00000001C2241000041221C0014083E0814A2
:101AD00008083E0808005030000008080808080000
:101AE000606000002010080402003E49453E0000EE
:101AF000427F40006251494600414949360018146E
:101B0000127F0027454539003E49493200017905D9
:101B1000030036494936000649291E0000363600C2
:101B20000000563600000814224114141414144105
:101B300022140800020151090600060909067E095F
:101B400009097E7F494949363E414141227F414151
:101B5000221C7F494949417F090909013E41494900
:101B60007A7F0808087F00417F41002040413F0103
:101B70007F081422417F404040407F020C027F7F5B
:101B80000408107F3E4141413E7F090909063E415C
:101B900051215E7F09192946264949493201017FB1
:101BA00001013F4040403F1F2040201F3F40304048
:101BB0003F631408146307087008076151494543DF
:101BC000007F41410002040810200041417F0004D1
:101BD0000201020440404040400001020400205441
:101BE0005454787F4844443838444444203844446A
:101BF000487F3854545418087E0901020C5252523E
:101C00003E7F0804047800447D40002040443D00AD
:101C10007F1028440000417F40007C041804787C39
:101C20000804047838444444387C14141408081414
:101C300014187C7C080404084854545420043F447D
:101C400040203C4040207C1C2040201C3C40204048
:101C50003C44281028440C5050503C4464544C449C
:101C6000000836410000007F0000004136080008EF
:101C700008221C08081C22080840800804201002C2
:101C800001536572766F2054657374004779726FE3
:101C90002053657475700048656C692053657475D0
:101CA0007000456C65766F6E5C44656C74610056BF
:101CB0002D5461696C00537469636B7920542D4312
:101CC000757400542D4375740053696D706C6520F4
:101CD000342D434800C91CC31CB61CAF1CA21C9762
:101CE0001C8C1C811C0000891112239B322446ADE0
:101CF000573665BF74488CC19D5AAFD3BE6CCAE5D8
:101D0000DB7EE9F7F88110080193331A22A5562CDF
:101D100047B7753E64C99C408DDBBF52AEEDDA64B7
:101D2000CBFFF976E802218B30100299132667AFBA
:101D3000763444BD554AADC3BC588ED19F6EEBE797
:101D4000FA7CC8F5D983310A2091121803A7772E9F
:101D500066B5543C45CBBD42ACD99E508FEFFB6677
:101D6000EAFDD874C904428D5316619F702004A9FE
:101D7000153227BB364CCEC5DF5EEDD7FC6888E157
:101D8000997AABF3BA85520C4397711E60A114285F
:101D900005B3373A26CDDE44CFDFFD56ECE9986037
:101DA00089FBBB72AA06638F7214409D512225AB3A
:101DB000343006B9174EEFC7FE5CCCD5DD6AA9E317
:101DC000B8788AF19B87730E6295501C41A3352A1F
:101DD00024B1163807CFFF46EEDDDC54CDEBB962F7
:101DE000A8F99A708B088481951AA793B62CC2A57E
:101DF000D33EE1B7F04008C919522BDB3A644EEDEF
:101E00005F766DFF7C899400859BB712A6ADD224C6
:101E1000C3BFF136E0C1184809D33B5A2AE55E6CCE
:101E20004FF77D7E6C0AA583B4188691972EE3A7A1
:101E3000F23CC0B5D14229CB38500AD91B666FEFAE
:101E40007E744CFD5D8BB502A499961087AFF32686
:101E5000E2BDD034C1C3394A28D11A580BE77F6E8E
:101E60006EF55C7C4D0CC685D71EE597F42880A1E5
:101E7000913AA3B3B2444ACD5B5669DF78600CE96E
:101E80001D722FFB3E8DD604C79FF516E4A9902046
:101E900081BBB332A2C55A4C4BD7795E68E11C684E
:101EA0000DF33F7A2E0EE787F61CC495D52AA1A321
:101EB000B03882B193466BCF7A5448DD59622DEB2E
:101EC0003C700EF91F8FF706E69DD414C5ABB12206
:101ED000A0B9923083C77B4E6AD5585C49E33D6A0E
:101EE0002CF11E780F20415244552050494C4F543C
:101EF000204D656761203F2F3820002052544C2030
:101F000044697374616E6365002041726475506941
:101F10006C6F74204D6F6465002050697463682095
:101F2000416E676C650020526F6C6C20416E676C6F
:101F3000650020436C696D62205261746520002049
:101F40004169722053706565642000204469737490
:101F5000616E636520002057617920506F696E744F
:101F6000202320002042656172696E670020436F64
:101F7000757273650020416C7469747564652048DE
:101F80006F6C640020416C74697475646500204353
:101F90006C696D622072617465002047726F756EA6
:101FA0006420737065656400204C6F6E676974759A
:101FB000646500204C6174697475646500009372F7
:101FC00011241FBECFEFD0E1DEBFCDBF11E0A0E0F6
:101FD000B1E0E4E1F7EE02C005900D92A434B10740
:101FE000D9F71DE0A4E4B1E001C01D92A537B10707
:101FF000E1F71FE1C0ECDFE104C02297FE010E947F
:102000004373CE3BD107C9F70E94C5700C94887307
:102010000C940000EDE3F5E040E0842F806487B984
:10202000369A3699FECF24B135B1369A3699FECF1D
:1020300084B195B1820F931F819391934F5F483084
:1020400061F70895853050F0883020F08E3020F40C
:1020500082E0089581E0089583E0089580E0089586
:102060002AE0829FC001112481509E4F089525E0EF
:10207000829FC0011124815C9C4F08958F929F9292
:10208000AF92BF92DF92EF92FF920F931F93CF9385
:10209000DF93C82FD62F5A01122FF02E822F847073
:1020A000D82E57FF10C0882311F08CE101C08FE0BB
:1020B000212F4DE26D2F9C2F981B892F0E94505C81
:1020C000B194A194B108212F2F214AE36D2F8C2FB9
:1020D0000E94505C6CE370E0C5010E94EC724B0101
:1020E0005C01012F00619B0140E050E062E0E62EC0
:1020F0006D2F8C2F0E94425EDD2011F08AE101C01D
:102100008FE00F2D0061950140E050E092E0E92E54
:102110006D2F8C0F0E94425EDF91CF911F910F9126
:10212000FF90EF90DF90BF90AF909F908F900895B9
:10213000CF93DF93D62FC22F206250E00E94525FD0
:10214000C7FD09C02C2F46E76D2F8091580CDF91F9
:10215000CF910C94505CDF91CF910895242F409142
:1021600002010C9498100F93022F24FF03C00F7EDE
:102170009CE201C094E2411104C024E043E553E035
:1021800015C04530B0F4E091160594E0E99FF001E8
:1021900011243197E40FF11DEF58FC4FE49194E0C6
:1021A000E99FA0011124445A5C4F24E00E94055D80
:1021B00008C0941730F02BEF240F41EB52E00E943F
:1021C000275D0F9108950F93CF93DF93C82FD62FDC
:1021D000022F411104C024E04CEA52E00EC04A3004
:1021E00010F086E101C081E18C0F50E0202F6D2FAF
:1021F0000E94525F22E049EA52E06D2F8C2F0E942C
:10220000055DDF91CF910F9108950F931F93CF93A9
:10221000DF93D62FC42F022F16E0180F442341F06E
:10222000463151F04A3E61F423E045E853E016C0E0
:1022300023E045EA52E012C023E041E853E00EC03B
:1022400047FF04C041E20E94505CC195C1504C2F31
:10225000440F4C0F50E04B595D4F23E06D2F812F01
:102260000E94055DDF91CF911F910F91089585E642
:1022700092E00895DF92EF92FF920F931F93CF9316
:10228000DF93F82ED62F142FE22EC091F00181E0BB
:102290008217E0F14FE04C0F4F31D0F42C2F332751
:1022A00027FD309537FF03C0319521953109012F66
:1022B00043E352E06D2F8F2D0E94275DCF3FC4F581
:1022C000212F41E26D2F8AEF8F0D0E94505C30C0AC
:1022D00074E2D72EDC0E0AEF0F0D88E48D1520F086
:1022E0001C1674F441EF09C0212F4DE682E18F0DD9
:1022F0000E94505C1C161CF44CED4C0F01C04D2D7F
:10230000212F6D2F802F0E94051112C082E028130B
:1023100013C0212F409160046D2F8AEF8F0DDF9144
:10232000CF911F910F91FF90EF90DF900C940511CA
:10233000E11002C0C13069F3DF91CF911F910F917D
:10234000FF90EF90DF9008958C3038F4E82FF0E0A4
:10235000EE0FFF1FEE55F84F22C08431C0F4482F16
:1023600050E0DA01AA0FBB1FA25DBE4F2D913C9138
:10237000803148F4FA01EE0FFF1FE451FB4F8081DA
:102380009181281B390BC901880F991F0895843248
:1023900048F4E82FF0E0EE0FFF1FE65AF84F808177
:1023A000918108958E3218F484520C94D51D80E0EA
:1023B00090E008950E94C1708111FCCF1092890CA9
:1023C00008950F931F93CF93DF938C01EB010E942D
:1023D000005C24E04DE252E060E082E20E943B5D5E
:1023E000B80180E20E945B5DBE0188E20E945B5DF5
:1023F00067E172E080E30E945B5D0E9416600E94CC
:102400001260DF91CF911F910F910C94DA110F930D
:10241000462F50E04B595D4F00E023E060E10E9401
:10242000055D0F9108950F931F93CF93DF93082FAE
:10243000C5EED1E01AE0499124E0602F812F0E947F
:10244000505C155F1837B9F7DF91CF911F910F914D
:1024500008951F93CF93DF93EC01162F0E94005C29
:10246000BE0188E10E945B5D111109C049E052E0A4
:1024700068E38CE10E94615D43E052E002C04BEFF3
:1024800051E024E060E082E20E943B5DDF91CF9169
:102490001F910C94166061E00E9429120C94126046
:1024A00070E0882399F090E0019725E0289FF001E3
:1024B000299FF00D1124E60FF71FEE0FFF1FE655C1
:1024C000FB4F808191818B509E4F0895FB01EE0F51
:1024D000FF1FED5FFE4F0190F081E02D8081992775
:1024E00087FD909508951F93CF93DF93D82F162FD4
:1024F000C4E0DD2399F0612F8D2F0E9450129C01C2
:10250000253F81E0380764F08BE0820F8D1710F0D3
:102510008CE0820FC15029F0D82FEBCFC0E001C072
:10252000CD2F8C2FDF91CF911F910895CF93C62F80
:102530000E9473126C2FCF910C9450120F931F9323
:10254000CF93DF93EA01062F10E08823B9F00E94B1
:102550007312882399F090E0019725E0289FF001FD
:10256000299FF00D1124E00FF11FEE0FFF1FE6551C
:10257000FB4FC55FD140D183C08317C0CE018358C4
:102580009F4F8B3F910540F01C161D061CF4CDE7B4
:10259000D0E002C0C3E8DFEFF801EE0FFF1FED5FF0
:1025A000FE4F0190F081E02DC08386E0DF91CF9156
:1025B0001F910F910C9498579F92AF92BF92CF9218
:1025C000DF92EF92FF920F931F93CF93DF938C01D3
:1025D0007B016A01922EB090C7019B2D9F7D9434A0
:1025E00039F080918007882309F487C0933439F447
:1025F000E801219683E10E94326C85E00BC095349E
:1026000019F0923409F07CC0E801219784E10E941E
:10261000326C84E00E94F460811164C0E114F10422
:10262000E1F481E0C816D104C1F480E6B81619F0CF
:102630008EE2B81212C010928007C1E00115110598
:1026400009F0C0E0D0E08B2D0E9445618EE2B81207
:1026500006C081E08093B00702C0A12C02C0AA246A
:10266000A39440915C0150915D01C41BD50B8091F6
:10267000B007833031F48091D001C80FD11D87FDA0
:10268000DA95CC16DD0644F48B2D0E94456183E17A
:102690000E94326CE6010AC0CE15DF053CF48B2D9A
:1026A0000E94456184E10E94326CE701C017D107A6
:1026B000B1F0209761F4A11003C08B2D0E94356109
:1026C00017FF02C083E101C084E10E94326C892DB2
:1026D00083700E94985781E08093640113C0109228
:1026E000640110C0CC27DD27C01BD10B85E00E9400
:1026F000456184E00E94456191CF953409F484CF0F
:10270000E8018CCFCE01DF91CF911F910F91FF9007
:10271000EF90DF90CF90BF90AF909F900895552796
:1027200047FD5095772767FD7095992787FD909510
:102730000E94DC12089522E00C948F13462F22E0B1
:1027400060E00C948F1321E00C948F13462F21E04E
:1027500060E00C948F13E0916501F0E0EE0FFF1F35
:10276000E859FE4F808191810895FC01A091650197
:10277000B0E0AA0FBB1FAA59BE4FED93FC938FEB9D
:10278000099587E10C94326CE1EBF7E0108E168A24
:10279000158A178A0895E8E2FDE037A1303180F408
:1027A00020A541E0420F40A7DF01A20FB11DA20FFB
:1027B000B11D8D939C93403108F010A63F5F37A365
:1027C000089590E08C5F9E4F0C94CB1390E00C9496
:1027D000CB1380912E05992787FD909509970C942E
:1027E000CB13FC019091210580A191FF74C091A1B0
:1027F000882311F0946001C09B7F91A386A1813052
:1028000059F5C79A37A121A1332321F181A541E0D0
:10281000480F41A7DF01A80FB11DA80FB11D8D9171
:102820009C9195A384A3403108F011A6315037A3A1
:1028300097FD02C031E101C038E233A32C7F97FD40
:10284000226021A381A18BBBC7988FE182A382E084
:1028500086A308952BBB48C081110CC0C79A81A1E3
:10286000836081A38BBB8091590C8D3308F43CC0ED
:1028700086E02FC0823009F438C081A18BBBC79A93
:10288000BF9800C0000000C086B38078BF9A96A1B0
:10289000933049F4882329F083A1815083A38111C7
:1028A00023C084E016C0943021F48823E9F083E04B
:1028B0000EC0953039F483A1815083A3811114C0D7
:1028C00081E007C0963081F4882371F084E183A30E
:1028D00085E086A309C090911E0596FB992790F983
:1028E000891711F0C79A0895C79808951BBA8FE108
:1028F0008ABB00C099B38FEF8ABBE8ECF1E0878117
:10290000882311F080E202C0892F807E8483292FE2
:10291000207C8081281759F08074880F907831814D
:10292000891711F0315001C03F5F318320838281CC
:102930009381891711F083838183089590911605FF
:1029400090FD02C093E08927E82FF0E0EE0FFF1F13
:10295000EE55F84F8081918197FF02C081589F4FBB
:10296000880F892F881F990BE82F181624F08823C9
:1029700021F0E19502C080E801C080E0E8300CF071
:10298000E7E0F0E0E85AFC4FE491EE2319F099E01B
:10299000909370018E2B0895833021F0811103C034
:1029A00083E001C080E0E82FF0E0EE0FFF1FE35C62
:1029B000FA4F808191810895FF920F931F93CF93D7
:1029C000DF93F12CC0E0D0E08F2D0E94CC14092FB2
:1029D00010E0C00FD11FF39484E0F812F5CFCE01C0
:1029E000DF91CF911F910F91FF9008950E94CC1419
:1029F0002091180520FF03C09195819591090895B4
:102A000078941F920F920FB60F9211248F9380919A
:102A100044018F5F809344018F910F900FBE0F9000
:102A20001F90189578941F920F920FB60F92112451
:102A30002F938F939F93EF93FF93F89487B78F7B98
:102A400087BF789420919101809193019091210505
:102A5000882359F090FF07C08091720D820F8093F8
:102A6000720D87FF02C01B9A01C01B9891FF2AC0FC
:102A700080915708811126C0E8E2FDE086A18230EE
:102A800009F583A1882311F081501BC021A1C79AA9
:102A900082A180FD09C02D7F84A195A196FD2260B1
:102AA000880F991F95A384A381E082278BBB81A304
:102AB000C79882A1815082A3811104C083E086A3BC
:102AC00085E083A3F89487B7806487BF7894FF91EB
:102AD000EF919F918F912F910F900FBE0F901F90AC
:102AE000189578941F920F920FB60F9211242F937E
:102AF0003F934F935F936F937F938F939F93AF9386
:102B0000BF93EF93FF9381B7845681BF8FE891E025
:102B10000E94E3690E9454618091950C82608093C9
:102B2000950CEBE0F1E08081815011F0808307C0CB
:102B300084E6808381818F5F818381E082838381CA
:102B4000815011F0838304C08AE0838381E0848311
:102B5000FF91EF91BF91AF919F918F917F916F9175
:102B60005F914F913F912F910F900FBE0F901F904B
:102B7000189578941F920F920FB60F9211242F93ED
:102B80003F934F935F936F937F938F939F93AF93F5
:102B9000BF93EF93FF932091800030918100F894D0
:102BA00080917D008F7D80937D00789480913605A3
:102BB00090913705A901481B590BCA019695879535
:102BC00030933705209336059C01215A3F402F3D15
:102BD0003E4220F481E0809345012FC0E091450101
:102BE0002FEF2E0F283048F59C0121523340273714
:102BF000354008F521E02E0F20934501F0E0EE0F5F
:102C0000FF1FEC5BFE4FAC014C5D554020911C0555
:102C1000332727FD3095265F3F4F429FC001439FDA
:102C2000900D529F900D11246AE070E00E94EC72AA
:102C30007183608302C010924501F89480917D00F9
:102C4000806280937D007894FF91EF91BF91AF9166
:102C50009F918F917F916F915F914F913F912F91B4
:102C60000F900FBE0F901F9018959C0155E0359561
:102C700027955A95E1F7280F391FAC01440F452FCE
:102C8000441F550B241B350B892F990F990B8595E4
:102C9000820F931F08959DE7980F9B3FA0F08E57DA
:102CA000282F30E0220F331FF901E456FB4F8081BB
:102CB000861714F46083862F48172CF4F901E45624
:102CC000FB4F4083842F089544E66CE90C944B1627
:102CD00020911605217092E0921B21E0981320E0CC
:102CE000822F08959091F60194FF08C00E94681603
:102CF00091E0811101C090E0892F089580E008954E
:102D000049E2840290011124359527953595279540
:102D100087FD815C86FB880F880B80F9A901481B21
:102D2000510987FD5395CA0108954F925F926F92A2
:102D30007F928F929F92AF92BF92CF92DF92EF924B
:102D4000FF920F931F93CF93DF93782E642E25E08D
:102D5000241708F4D4C0882309F4CFC036E18317C0
:102D600021F08AEE781203C0CAC081E0CCC096E19F
:102D700097150CF4C4C0872D992787FD909597FF70
:102D800003C09195819591098A3040F4825F0E9439
:102D9000F46017140CF4B7C091E01CC026EF280FA4
:102DA000E22EF12CE701CC0FDD1FCE0DDF1DC55C3F
:102DB000DB4F8A818F7009F4A2C0F701EA58FE4FF9
:102DC0006F01F5E06F1208C0F601908117140CF442
:102DD00092C081E0892797C0588049800E942210C4
:102DE000811109C08FEF850D0E94A4118C0189818A
:102DF0000E94801610C0823051F48FEF850D0E9422
:102E0000A4118C01898181500E94A41104C080E02A
:102E100090E000E010E02A812F70822E912CF401C6
:102E20003197EE30F10508F06CC0EA5BFF4F0C946F
:102E3000417317FF37C011950195110933C017FF72
:102E400035C011950195110931C001E0060D402FE3
:102E500060E0852D0E949516182F402F60E0842D8C
:102E60000E9495162A812F70253061F4112309F4F0
:102E700048C0882309F445C08A81982F907F69F55E
:102E800091E036C0263019F41111F6CFF2CF982F09
:102E9000912720C008171907A1F5EECF08171907C9
:102EA00059F72FC0801791073CF32BC0081719075B
:102EB0001CF327C008171907FCF623C080179107D9
:102EC000DCF61FC0F701EE57FE4F90819095991FD9
:102ED0009927991F9111D0CF0BC082958F7089309F
:102EE0000CF08F5F41E0460D60E00E949516982F30
:102EF000F60190836BCF892F06C0862F04C080E037
:102F000002C090E0F5CFDF91CF911F910F91FF901C
:102F1000EF90DF90CF90BF90AF909F908F907F9079
:102F20006F905F904F90089540E060E080910305BE
:102F30000E949516811114C08091570190915801FB
:102F4000892B71F41092480D8091590C90913C0599
:102F5000981751F080933C0588E29DE00C94F113A2
:102F600081E08093480DF0CF089520915701309172
:102F700058012115310511F021503109882319F02C
:102F800080911A0501C080E090915601992329F0A3
:102F900090912205891708F4892F4AEF849FC00178
:102FA0001124880F991F8217930708F4C901909381
:102FB0005801809357010C949417CF92DF92EF92AF
:102FC000FF920F931F93CF93DF93F89480915A0C45
:102FD00090915B0C789441E020913A0530913B054B
:102FE0008217930709F440E04093590190933B0501
:102FF00080933A0560E08BE597E00E9491368091DE
:103000005901882309F4BFC2809172019091730124
:10301000A0917401B0917501AC01BD014F5F5F4F8C
:103020006F4F7F4F4093720150937301609374010F
:1030300070937501443651056105710598F083560A
:103040009109A109B1098093720190937301A09332
:103050007401B093750180917001882319F081503B
:1030600080937001E1EBF7E0878980FF0DC0808DD0
:1030700091E0980F908F943638F08356808F858931
:1030800096890196968B858B80E00E94AA570E94B4
:10309000005C0E948860182F082F0F700650C091A6
:1030A000F701C43021F0C33019F4C4E001C0C8E016
:1030B000083008F09FC0F02EF6948091320580FF12
:1030C00003C083E08F19F82E6F2D80914D050E946B
:1030D0007312E82E6F2D0E9496129C01C1110DC033
:1030E000AC0197FF04C044275527481B590B559541
:1030F000479555954795C1E0C40F8091160580FB13
:10310000CC24C0F8D12C42E050E04C195D098F2D41
:1031100090E04817590761F48091F60180FF31C2B1
:1031200081E0C4E09091180590FF03C0C19501C0F3
:1031300080E0DD27C7FDD09500FF03C0C20FD31F7D
:1031400004C0A9014C1B5D0BEA01209721F09D2FC3
:10315000932797FF11C081110FC0232B69F040E026
:1031600050E06F2D8E2D0E949E12812F0E9445618E
:1031700086E10E94326C3DC0CE0184589F4F893F4A
:10318000910580F4AE016F2D8E2D0E949E12D7FF07
:1031900003C0D195C195D109D595C795D595C7954A
:1031A0004C2F21C01C161D061CF44DE750E002C038
:1031B00043E85FEF6F2D8E2D0E949E12CE01835843
:1031C0009F4F8B3F9105A8F4D7FF03C0D195C195C0
:1031D000D109D7FD2396AE0155954795559547954D
:1031E000519541955109445C65E18FE891E00E9459
:1031F000B46A10E0EAE5F1E08091AE079091AF0784
:1032000020813181281B390B37FF02C0215E3F4FDF
:10321000C5E035952795CA95E1F72115310561F08F
:1032200024813581281B390B37FF02C02F5F3F4FA8
:1032300035952795918380839583848380911805A4
:1032400085FF02C020E030E033832283C8ECD1E068
:103250002D818981821B8F3F09F480E087FD8F5F7C
:1032600085958887982F990F920F9D83812B0E94B7
:10327000B517E0916501F0E0EE0FFF1FEA59FE4F30
:103280008081918180569F43B9F488858823A1F07D
:103290002E81992787FD9095820F911D27FD9A9584
:1032A0008E37910514F08DE705C08338EFEF9E0748
:1032B0000CF483E88E83188680911E0587FF3BC03F
:1032C000809171018823B9F1809170018823A9F15F
:1032D0008091390587FD03C08F5F8093390582E0B7
:1032E0000E949E14982F9F7789F02091390592179C
:1032F00020F510923905111120C0182F1095111FBB
:103300001127111F83E6811B182F17C083E00E942D
:103310009E14982F9F7789F020913905921768F4B1
:1033200010923905111109C0182F1095111F11277E
:10333000111F1C5902C01092700181E0809371012D
:103340007DE9E72E74E0F72ECCE9D4E0EAE0CE2E5A
:10335000D12CF7018081882309F462C0853068F49C
:103360000E945C62E82FF0E0EE0FFF1FEF5FFE4F60
:103370000190F081E02D808104C0853021F480919E
:10338000CE0188834DC08A30B8F485500E945C62BB
:10339000E82FF0E0EE0FFF1FE056F84F808191819B
:1033A00097FD079643E0959587954A95E1F7833811
:1033B000FFEF9F07DCF015C08D30D0F4E82FF0E070
:1033C000EE0FFF1FEA56F84F8081918197FD079617
:1033D00023E0959587952A95E1F783382FEF92079B
:1033E0002CF08D3791056CF28DE7CBCF83E8C9CFF8
:1033F0008D31B0F4E82FF0E0EE0FFF1FE859F84FE1
:1034000080819181B6010E94EC7263384FEF74079E
:103410002CF06D3771051CF06DE701C063E868831F
:1034200052E0E50EF11C22968BEAE81684E0F806DD
:1034300009F08FCF8091E3019091E401009761F052
:1034400060E00E9429120E94C170882399F01092B6
:10345000E4011092E3010EC01093C701E0916501F1
:10346000F0E0EE0FFF1FEA59FE4F0190F081E02DD2
:10347000812F09950E941660C09165008FE891E048
:103480000E94CF69882311F084E105C08091740DFA
:10349000882321F081508093740D06C080916300D1
:1034A000869581708093730D8091730D8093E101F7
:1034B000882309F464C080911E0585FD60C0CF7E1D
:1034C000C09365008091590C8F71823009F054C00F
:1034D00080914B0590914C05AC0114E0440F551FB1
:1034E0001A95E1F797FD0796BC01D3E075956795AE
:1034F000DA95E1F720910205332727FD30952A5F01
:103500003F4F629FC001639F900D729F900D1124E9
:10351000840F951F2091180526FD05C060910001BC
:103520007091010102C060EF70E00E94D87280913A
:103530000201680F711D6F5F7F4F759567956093EE
:10354000020180913805805F80933805811114C095
:1035500080910105681780F4623370F06EE281E1BA
:103560000E94386C8091180583FF06C082E390E0CA
:1035700090935801809357011092560104C0C06186
:103580009FCF80E0CFCDDF91CF911F910F91FF9022
:10359000EF90DF90CF900895CF93DF93C62F2091C7
:1035A000E201222329F09093E4018093E30133C0E8
:1035B00060E00E942912C11103C08091000501C082
:1035C00089E10E94036067E182E10E94386C0E94F9
:1035D000DA11D1E00E94C17081111DC08091950C5B
:1035E000833019F4A8951092950C40E060E080912A
:1035F00003050E949516811106C080911A0581115C
:1036000002C0CC2329F0D093480D0E949417E2CF3A
:103610001092480DFACFDF91CF91089590916501F6
:10362000911103C0811106C017C0811103C08FEF33
:10363000890F01C080E08093650187E10E94326CB0
:10364000E0916501F0E0EE0FFF1FEA59FE4F019097
:10365000F081E02D8EEB099460E08EEE91E00C9409
:10366000CC1ACF93DF93EC0180916501843038F060
:1036700060E081EE91E0DF91CF910C94CC1A87E16C
:103680000E94326CA0916501AF5FA0936501B0E02C
:10369000AA0FBB1FAA59BE4FCD93DC938FEBFE013F
:1036A000DF91CF9109941F93CF93DF93C2EBD4E0C6
:1036B00090E0888111E0190F882341F040E060E03C
:1036C0000E949516882311F0812F05C0912F2A960C
:1036D000143079F780E0DF91CF911F910895DF9248
:1036E000EF92FF920F931F93CF93DF93809144014A
:1036F000C2B7909144018913F9CFD0E0D82B60E193
:10370000F62E80916104F81A0E940A101EE517B97E
:103710000E9476140E94DD1717B9369A3699FECFAB
:1037200084B195B10496409100015091010167E088
:10373000649F9001659F300D1124820F931F53E009
:10374000969587955A95E1F7909301018093000132
:103750008091950C833019F4A8951092950C2091C6
:10376000440182B7909144012913F9CF90E0922B44
:103770008C1B9D0B2091AC063091AD0628173907A4
:1037800020F49093AD068093AC0680910C018230BA
:1037900078F480910F01882309F4F1C080913305FA
:1037A000909134050196909334058093330589C038
:1037B00010920C01809135058F5E982F977F90367F
:1037C00018F49093350503C0877080933505C5EED6
:1037D000D1E0E12CEF14E9F28E0103581D4FF801FE
:1037E0008081982F907C9034C9F4880F880F40E036
:1037F00060E0859585950E949516882379F08091E3
:10380000210580FF05C0FE01E258FD4F608101C027
:1038100061E046E48FE891E00E94B46AF80180819B
:10382000982F907C9038D1F5880F880F85958595D5
:10383000873114F1992787FD90954797813091053D
:1038400049F08230910561F0892B41F58091350571
:10385000837003C080913505807F81111FC005C032
:103860008091350587708230C9F4FE01E258FD4F22
:1038700080810E94FB1D12C09091350590FD0EC005
:1038800040E060E00E949516882341F0FE01E25876
:10389000FD4F8081805890E00E94CB13E3942296E4
:1038A00099CF0F2D10E0E801CC0FDD1FCE59DB4F73
:1038B0008881E82EE294E69447E0E4228F7129F4AF
:1038C000F394FFE0FF1568F758C040E060E00E9405
:1038D0009516D82E80910F010F521E4F823009F499
:1038E00049C08E2D857051F4F8018081811106C088
:1038F000DD2021F0898190E00E94CB138FEF8E0DA7
:10390000823060F4F80180818130A1F5D11032C09D
:103910008981F2E0EF122BC08F5F29C085E08E1500
:1039200050F4F8018081811125C0DD2019F18981D1
:103930000E94FB1D1FC0F2E0FE15E0F4DD20D1F077
:1039400084E0E81631F095E0E91631F066E970E0C0
:1039500005C06CE271E002C068E572E08091330559
:10396000909134050E94D872892B21F4898190E0CE
:103970000E94CB13F801D082A3CF10920F01809147
:103980000D018823D1F110920D010BE314E0C2E880
:10399000D1E0EE24EA94F801F2808F2D8F700E941E
:1039A0002210833019F59881911104C0F8018081AB
:1039B000809508C097FF08C09F5F9883911106C04B
:1039C000F8018181888302C0915098838F2D807F78
:1039D00069F08F2D82958F7089300CF08F5F40E0F9
:1039E00060E00E949516811101C0E8820D5F1F4FB3
:1039F0002196F1E0CE38DF0771F6DF91CF911F916C
:103A00000F91FF90EF90DF9008951F93CF93DF9376
:103A1000182FD62FC42F8091B007811101C0C2E0AA
:103A20004D2F50E02C2F60E08FE70E94525FDA307C
:103A300010F0DFE601C0D5E72C2F4FE260E08D2FBC
:103A40000E94505C412F50E04F5F5F4F2C2F60E091
:103A50008FEF8D0FDF91CF911F910C94525F1F93C9
:103A6000CF93DF93D82F162FC42FB9010E945B5D2F
:103A7000112329F06FE08C2F0E949E13C82F4C2F2A
:103A800050E0212F6D2F80E60E94525F8C2FDF9136
:103A9000CF911F910895813649F40E94456181E0DC
:103AA0000E940E1B89E295E40E94311B67E57EE0CF
:103AB00080E10E945B5D61E47EE080E20C945B5DEE
:103AC000FF920F931F93CF93DF93182FF62E0AE0E8
:103AD0008AE0189FE0011124C150DE4F2FE130E051
:103AE000211B3109029FA001039F500D1124BE012B
:103AF000CE010A960E945673FF2049F0BE016A501B
:103B000071094AE050E0CE010E9456730AC0FE01DE
:103B100011920A95E9F78091F3078883898384E6F7
:103B20008A831093F507DF91CF911F910F91FF903A
:103B300008959C01220F331F280F391F95958795F3
:103B400095958795280F391F959587959595879514
:103B500095958795820F931F0895429643E7489F56
:103B60009001499F300D1124C901E6E09595879594
:103B7000EA95E1F7089581E00895E82FFF27E7FD32
:103B8000F095EB58FD4EE491862F992787FD90958F
:103B900083589F4FEE5FE23038F42AE0AC01249F57
:103BA000C001259F900D11240895E82FFF27E7FD00
:103BB000F095EB58FD4EE491ED3F4CF4EE0FFF0B0A
:103BC000E055FB4F8081992787FD90950895ED3F43
:103BD00059F074F0EF3F09F05CF4EE0FFF0BEB547B
:103BE000F84F8389948908958091020190E00895A7
:103BF00080E090E00895CF92DF92EF92FF92F82E4E
:103C00000E94D51DEF2DFF27E7FDF095EB58FD4EE7
:103C1000E491ED3F09F15CF4E63FDCF0EE0FFF0BC1
:103C2000E055FB4F8081992787FD909512C0EF3FAB
:103C300009F07CF46CE370E00E94EC726B017C0193
:103C400046E260E0C6010E94416CC70160E045E3C6
:103C500005C060E040E002C061E044E2FF90EF9008
:103C6000DF90CF900C94416CBF92CF92DF92EF9295
:103C7000FF920F931F93CF93DF93F82ED62EC42E6F
:103C8000E901102F8E2D8170B82EE0FE12C000E0E9
:103C900021E0240F4FE752E18F2D0E94275D12FD96
:103CA00003C088E18F0D06C08CE18F0D98EFD90E0F
:103CB00001C08F2D9E2D9870E3FC1F7BEC2DFF27FC
:103CC000E7FDF095EB58FD4EC49022E02C0D22301C
:103CD00088F412FF8450B110865F1770012F212FD6
:103CE000AE016D2D86500E943E10C3E3CC0D8AEFCD
:103CF000F80E0AC0992311F08DE38F0D212FAE012C
:103D00006D2D0E94525FC0E28E2D867069F0E2FE3A
:103D100004C08AE08F0D1B7F02C08091580C212FB8
:103D20004C2F6D2D0E94505C8C2FDF91CF911F91F5
:103D30000F91FF90EF90DF90CF90BF900895DF92AA
:103D4000EF92FF920F931F93CF93DF93D82F162FED
:103D5000C42FD22E8E2D8370F82EA1F08091C70132
:103D6000803881F48DE7840F8B3F40F0E42FF0E042
:103D7000EE0FFF1FE056FC4FC08101C0CEE782E08E
:103D80000E9498578DE78C0F2E2D8B3FE0F04EE36D
:103D900051E1612F8EEE8D0F0E943B5D2E2D43EB86
:103DA0004C0F612F8AEF8D0F0E94505CFF2009F1AC
:103DB00022E042E850E06EE770E08C2F90E00E9435
:103DC000DC12C82F16C04C2F552747FD5095612F88
:103DD0008D2F0E94525FFF2061F0402F6D2D8C2FA0
:103DE000DF91CF911F910F91FF90EF90DF900C9496
:103DF0009B138C2FDF91CF911F910F91FF90EF902C
:103E0000DF900895CF93DF939EE0899FE001112416
:103E1000CB51DE4FFE01EA54FE4F40E060E080816E
:103E20000E949516882359F0C954DE4F40E060E0A7
:103E300088810E949516811104C081E003C080E052
:103E400001C082E0DF91CF910895EF92FF920F932E
:103E50001F93CF93DF93F82EE62EC42FD42FD69541
:103E6000062F0D1B182F1D1B602F812F0E94F65D42
:103E70006D2F6E0D4C2F812F0E94F35D4C2F602F04
:103E80008D2F8F0D0E94F65D4C2F602F812FDF91BB
:103E9000CF911F910F91FF90EF900C94F35D21E073
:103EA000AC0160E080E00C943B5D1F93CF93DF9307
:103EB000182FC0E1D1E08BE798E00E944F1F113628
:103EC000B1F068F41036D1F48FEF88831982109224
:103ED000AD061092AC0687E10E94326C0FC012361C
:103EE00019F0133621F00AC08AEC9FE102C080E687
:103EF0009FE3DF91CF911F910C94B5136CE678E0AE
:103F000088E00E945B5D4981469550E068E084E569
:103F10000E94615F6DE578E080E10E945B5D488111
:103F2000469550E060E184E50E94615F6EE478E0D0
:103F300088E10E945B5D498150E08881481B5109FE
:103F400057FF02C04F5F5F4F5595479568E184E585
:103F50000E94615F65E478E080E20E945B5D809191
:103F6000AC069091AD0629E1289FA001299F500D34
:103F70001124569547955695479520E360E284E5D0
:103F80000E94525F62E378E088E3DF91CF911F9156
:103F90000C945B5D0F931F93CF93DF93182FC1EBAE
:103FA000D7E08DE298E00E944F1F113678F013366B
:103FB00028F0133659F485E59FE102C080E69FE3BF
:103FC000DF91CF911F910F910C94B51364E278E0CB
:103FD00088E00E945B5D4A815B8100E020E068E050
:103FE0008AE20E943E104C815D8120E068E08EE410
:103FF0000E943E106BE178E080E10E945B5D4E81A3
:104000005F8120E060E18AE20E943E104885598588
:1040100014E0569547951A95E1F720E060E18EE4AB
:104020000E943E1066E178E080E00E945B5D48817E
:10403000598120E060E08EE40E943E104EE76CE380
:1040400082E00E94F35D43E26CE185E00E94F65D50
:10405000CBE043E06BE38C2F0E94F65DCA5FC33870
:10406000C1F71091AF068091AE06893710F4C0E019
:1040700001C0C12FD6E00CE3EC2FF0E0E055F94F82
:104080004081602F641B8D2F0E94F65DCF5FC83783
:1040900008F0C0E0C11719F0DF5FDE3769F7DF9184
:1040A000CF911F910F91089591E0211101C090E0EF
:1040B000442319F041E853E002C045E853E0292FBA
:1040C0000C943B5D0F9301E0211101C000E0242F0F
:1040D00046E351E10E94275D0F9108956F927F9210
:1040E0008F929F92AF92CF92DF92EF92FF920F93B7
:1040F0001F93CF93DF93EC01162F842F4901602F7C
:10410000D0905A076090AA077090AB07A091AC07B7
:10411000B091AD07EAE5F1E026813781261937092C
:1041200037FF02C0215C3F4F76E0359527957A95A1
:10413000E1F7422F20937D07208531852A1B3B0B19
:1041400037FF02C0215C3F4F56E0359527955A95C1
:10415000E1F7922F20937B07442311F07782668248
:10416000992311F0B187A08790917C07911104C029
:104170009091180595FF06C010927D0710927B075D
:1041800010927C0790917D07911108C020917B07C8
:10419000211104C022813381232B61F020911A0563
:1041A0004AEF249F90011124220F331F30935801AE
:1041B0002093570181149104B1F02881211177C116
:1041C0002091B007222309F47BC1213009F48AC170
:1041D00091118FC1153609F4AFC1143609F4B6C177
:1041E00041E00E94051DE114F10451F098818C2DED
:1041F0009C1508F4892FF701E80FF11DE49101C027
:10420000E0E08091B007813081F58091D0011816EF
:104210006CF4DE1610F4D39411F588818A1518F425
:104220008F5F888301C01882D12C19C08823B9F010
:10423000D11014C08881882319F08150888301C06F
:10424000A882E114F10459F098818C2D9C1508F492
:10425000892FF701E80FF11DD49001C0DA94109274
:10426000D0011E3249F483E005C0833029F41E32A8
:1042700019F481E08093B007E114F10451F09881C2
:104280008C2D9C1508F4892FF701E80FF11D54912E
:1042900001C050E080918007811145C080917B076B
:1042A000882301F14881481B47FD40E08A2D90E0BA
:1042B000242F332727FD3095281739070CF04A2D76
:1042C0004883E114F10459F0C41608F44C2DF701A9
:1042D000E40FF11DE491ED1518F4DE2E01C0D12C90
:1042E00010927B0728812223F1F080917D0788239B
:1042F000D1F0D81AD7FCD12C8D2D992787FD909518
:10430000E114F10479F03C2D2C1508F4322FF7015B
:10431000E30FF11DE4912E2F30E0821793071CF07C
:10432000DE2E01C0D12C103669F190F4123409F45C
:1043300073C028F41132A9F11E3221F197C0143450
:1043400009F446C008F476C0153409F451C08EC093
:10435000153609F451C040F4133609F46EC0D8F58F
:10436000123609F45CC082C01E38C1F01F3B31F028
:10437000113809F07BC01092800721C0188210927A
:10438000800738C08881882309F470C081E090914B
:104390008007911180E08093800768C08EE80E94BA
:1043A000456180918007882319F0109280075EC0D4
:1043B0008881882311F0892831F41092B00780E0B9
:1043C0000E940E1B53C087E10E94326C18824EC0BF
:1043D000D51609F44BC0EF2809F448C08091800736
:1043E000811144C0D51610F4D39411C0D12C0FC044
:1043F000D11002C0D12C3AC0EF28C1F180918007C2
:10440000811134C0DD2011F0DA9401C0D52E55237E
:1044100069F11092C7012AC088818A1539F180910B
:104420008007811123C088818A1510F48F5F0DC029
:1044300018820EC088818823C9F08091800781117D
:1044400015C08881882319F08150888301C0A88213
:10445000E114F10479F288818C1508F4C82EF70173
:10446000EC0DF11DE490ED1408F4DE2C8091800732
:1044700081110AC021E080915C0190915D01892B3E
:1044800009F420E0822F01C081E080937F07D09261
:104490005A07DF91CF911F910F91FF90EF90DF901E
:1044A000CF90AF909F908F907F906F900895909154
:1044B0008007911103C091E09093B00740E091CE46
:1044C0002091D001121624F0222319F015E601C024
:1044D00014E61092D0011E3209F07ACE21E020932A
:1044E000B00705C01E3209F073CE1092B00710E07D
:1044F0006FCE2091800721116DCEE82FE91BE7FDDB
:10450000E0E0462F50E02E2F332727FD309524176B
:10451000350714F0EFEFE60FFF27E7FDF095282FA2
:1045200030E0E217F30729F0EE0FFF1FE80DF91D49
:104530001DC010927D074ECE811101C0862FF4015F
:10454000E80FF11DE80FF11D329710C0282F30E061
:1045500070E0615071092617370714F48F5F01C0AE
:1045600080E0880E911C880E911CF4018591949135
:10457000DF91CF911F910F91FF90EF90DF90CF903F
:10458000AF909F908F907F906F900C94B513AF92E7
:10459000CF92EF92FF920F93AE2CC12CE12CF12C15
:1045A0000E946E200F91FF90EF90CF90AF900895F2
:1045B000EF920F93E42E00E020E030E040E00E9414
:1045C000C7220F91EF900895BF92CF92DF92EF92A2
:1045D000FF920F931F93CF93DF93C82F8EED9AE036
:1045E0000E944F1FEE24E39406E022E531E144E00F
:1045F0006C2F87ED97E00E94C722B090D7071092EA
:104600007101C2EAD7E010E000E0C12CE4E0DE2E48
:10461000E12CF12C41E4612F88E10E94025D41E32D
:10462000400F612F8EE10E94025D802F0E94CC140A
:10463000AC01612F8AE20E94645D073081F0A8819D
:10464000B98124E630E00E94AE72A70196010E9473
:104650002273A901612F8AE50E94615F0AC081E08F
:10466000B81611F040E201C041E2612F8AE50E94D4
:10467000AE100F5F185F2296083061F622E04BED16
:104680005AE068E28CE60E94355D4091000150914D
:10469000010160E388E70E94615F81E0B8120AC00F
:1046A000B0927C074FE761E8809102050E94A31356
:1046B00080930205DF91CF911F910F91FF90EF90B2
:1046C000DF90CF90BF900895EF920F931F93CF93F9
:1046D000DF93C82F86ED9AE00E944F1FE12C06E081
:1046E00022E531E143E06C2F86ED97E00E94C7227E
:1046F000D0E0C0E0C43018F018EF1D0F01C01D2F2E
:104700008FE08C0F0E94F460082FCF5F20E04C2FC9
:10471000612F8AE20E94051140E3400F202F612F94
:1047200084E40E94505CD85FC93021F7D8E3C0E030
:104730008C2F0E94F460182F00E02C2F46EB5AE0DB
:104740006D2F80E00E94275D40E3410F212F6D2FE8
:1047500080E20E94505CCF5FD850C63049F74EEAE5
:104760005AE068E184E50E94615D16E0C0E2D0E0B5
:104770002D2F46E751E16C2F84E50E940B5C812FC1
:104780000E94F46040E3480F282F6C2F8CE60E94B3
:10479000505C81E0810F0E94F46040E3480F282FB5
:1047A0006C2F88E70E94505CDF5FC85F1E5FD430CB
:1047B000F9F6DF91CF911F910F91EF900895EF924D
:1047C0000F93CF93C82F86EA9AE00E944F1FE12CE7
:1047D00006E022E531E142E06C2F85ED97E00E9492
:1047E000C7226BEB77E080E10E945B5D6BEE77E0C8
:1047F00088E10E945B5D6AED77E080E20E945B5D8C
:104800006BEC77E088E20E945B5D6BEA77E080E327
:10481000CF910F91EF900C945B5D4F925F926F92EE
:104820007F928F929F92AF92BF92CF92DF92EF9240
:10483000FF920F931F93CF93DF93C82F80EF90E1E8
:104840000E944F1FA7E0AA2ECC24C394BEEEEB2EED
:10485000B0E1FB2E0CE02EE531E14BE06C2F8BEE4E
:1048600097E00E946E206090EB0780905A07CDE998
:10487000EC2EC4E0FC2ECCE9D4E0AA24A394B12C05
:1048800018E0712C992487FC9094C12CD12CF0E372
:104890004F2E4A0C0C2D6BEE70E1812F0E945B5D58
:1048A000442D612F8CE00E94025D6A147B0449F460
:1048B0008C149D0431F480918007811105C021E0A2
:1048C00001C020E0512C03C022E055245394013054
:1048D00099F0022FF701208142E950E1612F88E42D
:1048E0000E94275D5520C1F06CE1F70180810E9494
:1048F0009E13F701808310C04881552747FD5095CE
:10490000612F8CE60E94525F552031F04DE763E83D
:1049100088810E949B138883FFEFCF1ADF0A82E011
:10492000C816D10409F0B6CFE2E0EE0EF11C2296D3
:10493000185FFFEFAF1ABF0A103409F0A6CFDF915E
:10494000CF911F910F91FF90EF90DF90CF90BF908C
:10495000AF909F908F907F906F905F904F90089551
:104960007F928F929F92AF92BF92CF92DF92EF92FF
:10497000FF920F931F93CF93DF93D82E8EE99AE087
:104980000E944F1F56E0A52E65E0C62E78E9E72E5F
:104990007AE0F72E06E022E531E141E06D2D84ED6D
:1049A00097E00E946E20C090D40780905A078091B3
:1049B000630081FF04C061E97AE088E1FCC0CA9429
:1049C00080918007882319F043E0942E02C0992437
:1049D0009394CCE0D5E0B12C10E1AA24A394AB0CC5
:1049E00020E04A2D612F80E00E94B310F12CCB1003
:1049F00002C08F1411F000E001C0092D802F8270D9
:104A0000782E92E0F91609F444C0E3E0FE1609F4AA
:104A100055C0F1E0E980FF16D1F0E294E694E69407
:104A200033E0E3222E2D46E85AE0612F88E10E9410
:104A3000275D772009F45AC062E08E2D0E94A613EC
:104A40008295880F880F807C99819F731FC0EE0C20
:104A5000EE0CE594E5948E2D9DE08902F001112481
:104A6000F7FD3396AF015595479555954795202FFE
:104A7000612F82E40E94525F7720C1F14FE161EE25
:104A80008E2D0E94A3138F739981907C982B99830C
:104A90002DC0E880EE2DE770EE2E2E2F48E75AE06D
:104AA000612F88E40E94275D772001F163E08E2D5D
:104AB0000E94A61387709881987F16C0E880E594BD
:104AC000E594E594202F4E2D612F8AE50E94051173
:104AD000772061F046E16AEE8E2D0E94A313880FC5
:104AE000880F880F98819770982B9883F394F4E03F
:104AF000FF127DCF185F2296AF1611F0BA2C6DCF42
:104B00006DE67AE080E30E945B5D84E0C8120AC033
:104B100048E266EF80911C050E94A31380931C0558
:104B200021E201C020E240911C05552747FD509528
:104B3000465F5F4F60E38EE40E94525FEE24E39491
:104B400095E0C912E12C2E2D49E65AE068E380E099
:104B50000E943B5D06E411E0C4E0D5E090E3F92E4D
:104B6000F801419151918F0169917991461B570B41
:104B7000440F551F20E268E38F2D0E94525FF8E139
:104B8000FF0E80E9F812ECCFEE2091F090E6D912FA
:104B90000FC088E0E6E4F1E0A4E0B5E001900D92FA
:104BA0008A95E1F781E00E94985787E10E94326C74
:104BB00069E57AE088E0DF91CF911F910F91FF9036
:104BC000EF90DF90CF90BF90AF909F908F907F90AD
:104BD0000C945B5DFF920F931F93CF93DF93F82E9E
:104BE000EB018A0147E16CE20E94251F43E06BE282
:104BF0008F2D0E94F65D43E06CE28FEF8F0D0E94D7
:104C0000F35DC8016FE87FEF0E94EC722CE2260F83
:104C1000CE0161E770E00E94EC72862F45E0622FC2
:104C20008F0DDF91CF911F910F91FF900C94251F55
:104C3000CF92DF92EF92FF920F931F93CF93DF9368
:104C4000C2EAD7E04A815B81688179818AE20E9469
:104C5000EA254C815D816E817F8186E50E94EA258F
:104C60002896EAE3FE2E0DE510E0F7E3CF2E8991BA
:104C700099919C5FB8010E94EC72DD24D394D60E0A
:104C8000EC2CE61A4D2D6E2D8F2D0E94F65D4D2DCC
:104C90006E2D81E08F0D0E94F65D4D2D6E2D82E010
:104CA0008F0D0E94F65D85E0F80E89E4F812DFCFE3
:104CB000DF91CF911F910F91FF90EF90DF90CF90F8
:104CC0000895DF92EF92FF920F931F93CF93DF939C
:104CD000F82E83E19BE00E944F1FEE24E39406E050
:104CE00022E531E145E06F2D88ED97E00E94C72273
:104CF0001092D807CBE3D7E010E0812F0E94CC14AC
:104D000048815981841795070CF4AC014993599354
:104D10002C853D85281739070CF49C013D872C878D
:104D2000143060F0FE017097240F351F37FF02C06A
:104D30002F5F3F4F35952795318320831F5F1730B5
:104D4000E1F68091570780937C0790E2F91621F0F5
:104D50008FEBF8120EC00BC08F5F80935707833024
:104D600041F487E10E94326C81E00E9498571092D2
:104D70005707809157078130E1F0A8F0823009F0A1
:104D80007BC01092710162EE7AE080E10E945B5D6F
:104D900041E451E168E182E10E94615DC3EDD4E04C
:104DA000EBE3F7E028C062E07BE088E10E945B5D16
:104DB00063C064EF7AE080E10E945B5D41E451E111
:104DC00068E182E10E94615DCDE2D7E0D12C18E973
:104DD000E12E1AE3F12E08E615ECFF86EE861D8F14
:104DE0000C8F8D2D0E94CC1489939993D39497E0C6
:104DF000D912F3CF41C061917191848595859B0152
:104E0000281B390B37FF03C0319521953109233316
:104E100031053CF1DF0150974D915C9159834883F6
:104E20009A01261B370BB90137FF02C0615C7F4F27
:104E3000B6E075956795BA95E1F7261B370B3F8766
:104E40002E87841B950B9C0197FF02C0215C3F4F6E
:104E5000A6E035952795AA95E1F7821B930B9D8FC8
:104E60008C8F229687E0E934F80729F60E940156D4
:104E70009093FE048093FD04DF91CF911F910F91D9
:104E8000FF90EF90DF900C941826FF920F931F93E2
:104E9000CF93DF93182F062FEA01F22E222321F061
:104EA00061E00E94A613182FBE01802F0E945B5D57
:104EB0002F2D412F602F86E60E945420812FDF91F5
:104EC000CF911F910F91FF900895FF920F931F9321
:104ED000CF93DF93182F062FEA01F22E222321F021
:104EE00061E00E949E13182FBE01802F0E945B5D1F
:104EF0002F2D412F602F86E60E945420812FDF91B5
:104F0000CF911F910F91FF9008951F93CF93DF933F
:104F1000D62F122F0E946527C82F212F482F6D2FC3
:104F200086E60E9462208C2FDF91CF911F91089519
:104F3000CF93482FCAE02AE0829FC00111248150FC
:104F40009E4F2FE130E0241B3109C29FA001C39F77
:104F5000500D1124BC01665F7F4F0E945673E5E33C
:104F6000F3E0DF011D92CA95E9F782E00E949857AD
:104F7000CF910C9437580F93CF93C42F0E940511F3
:104F8000002339F046E16AEE8C2FCF910F910C94FB
:104F90009B138C2FCF910F9108950F931F93CF9355
:104FA000DF93D82F162FC42F022F47FF08C041E2EE
:104FB0008AEF8D0F0E94505C86E08C1BC82F2C2F2F
:104FC0004CE25FE0612F8D2F0E94275DDF91CF9132
:104FD0001F910F9108950F931F93CF93DF93162F77
:104FE0008132C0F5811103C0611108C033C0803225
:104FF00019F4662329F02EC0662311F001E001C0E8
:105000000FEF080F0E943010EC01802F0E9430102B
:10501000FC0198818FEF890F8031E0F420812131EC
:10502000C8F4291302C08BE009C0112329F0903184
:1050300088F49F5F98830EC088830CC0815029F04C
:105040009081288121939993F9CF82E00E9498570B
:105050000093F407DF91CF911F910F9108958091F4
:105060003503882329F08BE49DE10E94311B81E008
:10507000089569E37EE088E20E945B5D6AE27EE07B
:1050800080E30C945B5DCF93C82F813669F08F3B32
:1050900039F0803699F480912C070E94982704C03B
:1050A00080E00E94326C0AC08C2F0E94456181E032
:1050B0000E940E1B89E295E40E94311B6EE17EE0A6
:1050C00088E00E945B5DCF910C9439280F93CF93B9
:1050D000C82F80912907882319F060E87DE002C07D
:1050E00063E77DE088E00E945B5D4FE06DE277E082
:1050F000809128070E94635600E12AE04DE257E0C4
:1051000060E181E00E94055D4FE360E182E40E947E
:10511000025D0E943928C13609F44EC0CF3B21F010
:10512000C03609F055C005C080E0CF910F910C94B6
:10513000326C809129078823A9F081E69DE00E94C6
:105140004B12809128070E94D156882339F087E1BD
:105150000E94326C82E0809329072CC080E00E947C
:10516000326C28C08091FF048F5F0E948859C091E3
:10517000FF0481E08C0F0E945859811109C0C15071
:10518000C13108F0CFE08091FF04C813F2CFC0E036
:10519000C093FF0481E00E9498570E943758809185
:1051A000FF040E949A568091EF010E94E11382E071
:1051B00080930F0180E601C081E60E94456181E095
:1051C0000E940E1B81E690E3CF910F910C94311B4E
:1051D000CF910F9108959091D00181E0191624F09C
:1051E000911101C080E081951092D0010895CF9374
:1051F000C82F0E94EB2890912B072091C7012236DF
:1052000071F028F4203639F02136A9F006C0233693
:1052100061F02E3611F481E00FC0181624F49C17AB
:1052200030F49F5F04C0882311F091119150909346
:105230002B0780E001C082E0CF91089564E17EE019
:1052400088E00E945B5D6AE07EE080E10E945B5D39
:1052500060E07EE088E10E945B5D66EF7DE080E2D9
:105260000E945B5D6CEE7DE088E20E945B5D2AE25D
:1052700040E367E082E10C94645FCF93DF9380E0CA
:105280000E941E2984E00E94F728D82FC0912B0786
:105290006C2F660F660F660F685F20E044E288E1BE
:1052A0000E94895DD130B9F5C13089F40E942F2860
:1052B00081110FC0C093F2078091F5078F5F809333
:1052C000F50760E00E94601D10922A0702C0C230FC
:1052D00018F485E092E40EC08091F507C43069F4BB
:1052E00080932C078091C7010E9445611092C701ED
:1052F00083E498E20E94311B0BC0C23031F48F5F0F
:105300008093F50761E00E94601D81E080932A0789
:10531000109259070AC0D23041F410925907809177
:10532000C7010E9445611092C7018091F5078093E3
:10533000F407DF91CF910895CF92DF92EF92FF9221
:10534000CF93DF93FC01EB019C01DC010E949F7273
:105350009B01AC01DE010E94B572272F382F492F27
:105360005527DF010E94B5726B017C013CE0F69489
:10537000E794D794C7943A95D1F724E630E02C1BF4
:105380003D0B0E949F726E5C7F4F8F4F9F4F6C0D45
:105390007D1D8E1D9F1D24E630E040E050E00E9400
:1053A0000073C901DF91CF91FF90EF90DF90CF9014
:1053B00008951F93CF93DF936115710529F1192F7C
:1053C000111F1127111F19F091958195910977FFF0
:1053D00010C0719561957109C0E0D4E09E01281B51
:1053E000390BC9010E949C299E01281B390BC90158
:1053F00002C00E949C29112329F022273327281B51
:10540000390B01C09C01C901DF91CF911F91089513
:105410006F927F928F92AF92CF92EF920F93CF9332
:10542000DF93CDB7DEB7382F562F822F602F9C2DFC
:10543000442321F0552329F022E00AC020E000E0B7
:1054400008C0E0915C01F0915D0121E0EF2BB9F320
:1054500001E0442311F0311121E03EE0E39E3001F0
:105460001124A30141575C4F3A01933639F4FA01F4
:1054700044850E94BB27F30184872AC0923639F401
:10548000FA0145850E94BB27F301858721C04A2D7B
:1054900050E0490F511D490F511D440F551F480D34
:1054A000511D460D571DFA013F01A11007C0408153
:1054B000E22E04E62CE90E949F1E08C040814C5950
:1054C000E22E04E620E00E949F1E8456F3018083B2
:1054D000DF91CF910F91EF90CF90AF908F907F9011
:1054E0006F9008952F923F924F925F926F927F92AA
:1054F0008F929F92AF92BF92CF92DF92EF92FF92E4
:105500000F931F93CF93DF9300D000D000D0CDB77F
:10551000DEB7182F89ED9DE00E944F1F93E0A92E62
:10552000C12C28EDE22E2DE0F22E00E020E030E04C
:1055300040E0612F85EE97E00E946E20109271018D
:105540004091F1074F5F20E060E080E30E94B310DC
:10555000F090E5078091F1070E94021F182F8091BB
:10556000F107E82FF0E0EE0FFF1FEE55F84F208116
:1055700031812A3131051CF01092E40706C0273E24
:105580003F4F1CF491E09093E4070E947216811142
:105590001092E40763ED7DE080E10E945B5D41E0F5
:1055A000F11040E08090E407A12CC12EE090F107BB
:1055B00000E126E361E081E00E94082A6CEC7DE0D6
:1055C00088E10E945B5D41E0F41240E08090E407D6
:1055D000AA24A394C12EE090F10708E126E361E03C
:1055E00081E00E94082A66EC7DE080E20E945B5D1B
:1055F00041E0E2E0FE1240E0812CA12C83E6C82EBF
:10560000E090F10700E22EE161E081E00E94082ACB
:1056100060EC7DE088E20E945B5D41E0F3E0FF1218
:1056200040E0812CA12C02E6C02EE090F10708E2B8
:105630002EE161E081E00E94082A113029F0123049
:1056400031F462EB7DE005C069EB7DE002C06AEAFF
:105650007DE080E30E945B5D2091F1078EE0289F52
:105660009001112494E0199F200D311D11242B511C
:105670003E4FF901E655FE4FD901A555BE4F1C918D
:10568000D901A455BE4FFC9084E6F80ED901A3556C
:10569000BE4F0C910C5980810E946416682E812F98
:1056A0000E946416382E44E660E08F2D0E944B164F
:1056B000782E44E660E0802F0E944B16582E809191
:1056C000F1070E947216E62DFF27E7FDF095FE8395
:1056D000ED83E72CFF24E7FCF094882309F464C0F1
:1056E000812C912C540110E0A4E6CA2ED12CB0E4F8
:1056F0004B2E6D817E81D501C401B595A7959795F7
:1057000087950E94D929880F991F61E270E00E9455
:10571000EC726E9DC0016F9D900D7E9D900D1124C9
:105720000FE3010FB6010E94D872F42DF61B6F2F04
:10573000802F0E94A65D812F837051F46FE3802F2C
:105740000E94A65D612F6695605E8FE30E94A65D54
:105750001F5F21E2820E911CA11CB11C1E3349F671
:10576000E091F107F0E0EE0FFF1FEE55F84F0081DA
:1057700011814801AA2497FCA094BA2CC501B40158
:1057800021E230E040E050E00E9422734EE361E00D
:105790008EE5820F0E94F65D8091F1070E947216DD
:1057A000882309F4ABC06CC000E010E0912C31E21A
:1057B000C32ED12C44E6A42EB12C50E2252E832DED
:1057C000992787FD90959A838983E52DFF27E7FD2B
:1057D000F095FC83EB836D817E81C8010E94D929FD
:1057E000B6010E94EC726E9DC0016F9D900D7E9D72
:1057F000900D11242EE5822E890CB5010E94D872DD
:10580000F22DF61B6F2F882D0E94A65D292D237087
:10581000422E49F460E2882D0E94A65D60E2690D87
:105820008EE50E94A65D69817A81C8010E94D9290E
:10583000B6010E94EC72EB81FC816E9FC0016F9FEC
:10584000900D7E9F900D1124BEE58B2E8918B50119
:105850000E94D872605E882D0E94A65D411009C02A
:1058600060E2882D0E94A65D622D69198EE50E9476
:10587000A65D93940F5D1F4FFFE19F12ACCF70CFD9
:10588000C501B4017C5F8F4F9F4F22E030E040E0C4
:1058900050E00E9422736D817E81C9010E94D92946
:1058A0009C01220F331FA72D77FCAD5FA595A59511
:1058B000BB27A7FDB0950E94977229E130E040E038
:1058C00050E00E94227369017A01CA01B9012FEDEB
:1058D0003FEF4FEF5FEF0E94227360E4620F4EE3F1
:1058E0008FE30E94F35DC701B60122E030E040E0A3
:1058F00050E00E94227369017A0135C0181419041E
:105900001A041B040CF0632C662D772767FD709535
:10591000C8010E94D929181419041A041B0414F48C
:10592000A72D01C0A52DA7FDAD5FA595A5959C014F
:10593000BB27A7FDB0950E94977229E130E040E0B7
:1059400050E00E94227369017A01CA01B9012FED6A
:105950003FEF4FEF5FEF0E94227360E2620F4EE372
:105960008FE30E94F35D29E130E0D8010E94AE721E
:10597000412C512C32015394A30192010E942273B5
:10598000A90160E382E70E94615FA9E1B0E0A7019D
:1059900096010E94B572A30192010E942273A9018F
:1059A00068E084E50E94615F181419041A041B045E
:1059B0005CF46D817E81C80144970E94D9299601CB
:1059C000281B390BC9010AC0632D772767FD709525
:1059D000C80144960E94D9298C199D0945E0489F29
:1059E0009001499F300D1124442737FD4095542FD5
:1059F000E3E0EE2E00E360E184E50E94425E26963D
:105A00000FB6F894DEBF0FBECDBFDF91CF911F91CF
:105A10000F91FF90EF90DF90CF90BF90AF909F904D
:105A20008F907F906F905F904F903F902F90089550
:105A30002F923F924F925F926F927F928F929F929E
:105A4000AF92BF92CF92DF92EF92FF920F931F938C
:105A5000CF93DF93CDB7DEB72B970FB6F894DEBFA9
:105A60000FBECDBF182F82EA9DE00E944F1FF4E0C9
:105A7000AF2ECC24C394A0EAEA2EADE0FA2E0CE0BF
:105A80002EE531E144E0612F83EE97E00E946E2025
:105A90008091E307FF24FA94F80E20915A07298396
:105AA000811110927101103871F480E80E944561F3
:105AB0001092C701F7FC52C182E79AE20E94311BA3
:105AC000F092F1074BC140E95DE068E085E10E949A
:105AD000615D7FED672E77E0772E82EA97E09F8306
:105AE0008E8310E11B861A86EEE05E2EEF2DFF27D7
:105AF000E7FDF095FB83EA83BA848B2D0E94021F99
:105B0000982E84E0989E900111243D832C83EA8591
:105B1000FB855E9EC0015F9E900D1124820F931F36
:105B20008B519E4FDC01A355BE4FFC01E455FE4F47
:105B30003C91208132130DC0FC01E555FE4FDC0184
:105B4000A655BE4F31E020818C91281330E0432EC2
:105B500001C0412CEE81FF8181919191FF83EE8301
:105B60009C01275E3F4F2333310508F0412C798695
:105B70006886F301F0808A31910534F4873E9F4FA7
:105B800024F4FF24F39401C0F12C8B2D0E94721693
:105B9000882319F0F12C44244394F301F08220E08F
:105BA00041E04B0D612F80E00E94B3103324339409
:105BB000F110312C8091800781110AC021E0809181
:105BC0005C0190915D01892B09F420E0D22E02C086
:105BD000DD24D3942A813B818A859B852817390748
:105BE00031F481E09981911180E0282E01C0212CAF
:105BF000F3018080A12CC92CEB2C012F27E2422D30
:105C00006D2D80E00E94082A2220C9F0DD20B9F025
:105C10004420A9F02A853B85529EC001539E900DD9
:105C20001124EC81FD818E0F9F1F81579C4FFC0139
:105C3000EF0DF11D2081FC01E30DF11D20832A8170
:105C40003B818A859B852817390739F481E0998142
:105C5000913009F080E0282E01C0212CEFEF6E1A60
:105C60007E0AE885F9858080AA24A394C92CEB2CB0
:105C7000012F29E3422D6D2D80E00E94082A222069
:105C8000C9F0DD20B9F04420A9F02A853B85529E59
:105C9000C001539E900D1124EC81FD818E0F9F1F3A
:105CA0008F569C4FFC01EF0DF11D2081FC01E30D8F
:105CB000F11D20832A813B818A859B85281739071E
:105CC00021F441E09981923009F040E0812CA12C2F
:105CD00063E6C62EEB2C012F2FE36D2D80E00E9492
:105CE000082AEA81FB812A853B85E217F30721F424
:105CF00041E03981333009F040E0812CA12C52E69B
:105D0000C52EEB2C012F27E56D2D80E00E94082A7F
:105D1000411004C0FF2029F04FE701C04DE28AE3A3
:105D200002C04EE78BE3612F0E94025D81E098166E
:105D300029F092E0991204C04CE403C04DE401C084
:105D400048E4612F85E70E94025DEA85FB85319674
:105D5000FB87EA87185F103309F0CECE2B960FB67B
:105D6000F894DEBF0FBECDBFDF91CF911F910F9191
:105D7000FF90EF90DF90CF90BF90AF909F908F906B
:105D80007F906F905F904F903F902F90089590E09C
:105D9000E92FFF27E7FDF095EE5CFD4EE491E81357
:105DA00002C0892F0895EE2311F09F5FF1CF80E0AC
:105DB0000895823430F4E82FF0E0EE5CFD4E8491DB
:105DC000089580E20895FF920F931F93CF93DF937E
:105DD000C82FD62FF42E122F622F842F0E9450121C
:105DE000FC01E53F81E0F80794F09BE09E0F9F15D2
:105DF00010F09CE09E0F40E3490F202F6D2F8C2F59
:105E0000DF91CF911F910F91FF900C94505C212F47
:105E10004EEC5BE06D2F8C2F0E94275DDF91CF91C0
:105E20001F910F91FF900895BF92CF92DF92EF9252
:105E3000FF920F931F93CF93DF93C82F81EB9BE0CB
:105E40000E944F1F06E0E02E0CE02EE531E143E01A
:105E50006C2F8CED97E00E94C722B090DC07C03613
:105E600011F0CE3669F48FEF8B0D843048F48093B7
:105E7000F7078C2F0E94456182E89FE20E94311B48
:105E800068EA7BE088E00E945B5DC5EED1E010E14E
:105E9000F12E11E0CC24C3941B11C12C65EA7BE0E8
:105EA0008F2D0E945B5D40E3410F6F2D8CE00E94BF
:105EB000025D2C2DFE01E353FD4F40816F2D8AE2E0
:105EC0000E940511BAE5DB2EE12C0C2D2E2D412F61
:105ED0006F2D8D2D0E94E32EE39486E0D80E84E092
:105EE000E812F3CF1F5F88E0F80E2A96153091F67E
:105EF000DF91CF911F910F91FF90EF90DF90CF90A6
:105F0000BF9008956F927F928F929F92AF92BF92AF
:105F1000CF92DF92EF92FF920F931F93CF93DF9375
:105F2000C82F8090F7072AE0829E40011124C40107
:105F300086559B4F4C0186EC9BE00E944F1FAA2484
:105F4000A394CC24C39424ECE22E2BE0F22E00E0A8
:105F500020E030E040E06C2F8DED97E00E946E2055
:105F60004091F7074F5C60E080E30E94025DC090C3
:105F7000DD076090800718E0E12CF12CDD24C7FCE0
:105F8000D0948E2DCE14DF0429F416142CF492E054
:105F9000A92E04C0A12C02C0AA24A394813081F0B0
:105FA0006DEB7BE0812F0E945B5D0A2D2A2DF401B1
:105FB0004085612F80E30E94BB27F401808751C098
:105FC00067EB7BE0812F0E945B5D80E3782EB12C34
:105FD00080915A078B1511F000E001C00A2D409105
:105FE000F7074F5F2B2D612F872D0E94E32EAA20EC
:105FF00091F120915A072B112EC0161434F0809184
:106000005C0190915D01892B31F1E401C20FD11D3A
:10601000C20FD11DE881F981CF018B509E4F843F83
:10602000F1E09F0714F484EF91E022E048EF51E0A3
:1060300064EF71E00E94DC12AC018091640188235E
:1060400051F0443F21E0520711F440E050E0455F39
:10605000514059834883B39486E0780E94E0B91296
:10606000B7CFEFEFEE1AFE0A185F183109F089CFAB
:10607000DF91CF911F910F91FF90EF90DF90CF9024
:10608000BF90AF909F908F907F906F900895CF9327
:10609000C62F0E9445610E943758C093FF048C2F81
:1060A0000E949A568091EF010E94E11382E0809352
:1060B0000F0181E00E9498570E94375881E0CF91EC
:1060C0000895BF92CF92DF92EF92FF920F931F93AA
:1060D000CF93DF93D82F85E29BE00E944F1F8091E2
:1060E0008007811110C0E0917D07E7FF0CC0E195AA
:1060F000EC3008F0EBE0F0E0EE0FFF1FE25AFE4E4E
:10610000859194915BC01091DA074FE06D2F8AED75
:1061100097E00E94D8226FE17BE080E00E945B5D07
:106120000E94AB58AC0160E086E60E94615F41E0EE
:106130006CE080E00E94051DC091DA07809129077C
:10614000823021F41092D90710922907D63638F4FC
:10615000D436F0F4D036E9F1D13659F05EC0D138FA
:1061600009F440C0DF3B09F44FC0D03809F055C0F6
:106170003DC08091D907882359F01092D90787E153
:106180000E94326C6091DA0781E60E94473045C078
:106190008091FF048C1739F06C2F8D2F0E944730AF
:1061A00081E00E94326CD53629F48DE094E20E94A1
:1061B000B51333C0D43689F58FEA9DE4DF91CF91D2
:1061C0001F910F91FF90EF90DF90CF90BF900C94B4
:1061D000B51381E08093D9071092800787E10E9470
:1061E000326C1BC081E00E940E1B17C08091D90742
:1061F000882399F081E080932907C093280786E6D9
:1062000098E20E94311B09C01092D9078091FF04C7
:106210008093DA0781E00E94AA578091D9078823EA
:1062200041F01C1731F061E06C0F81E0810F0E949A
:106230006659DD27C7FDD095809181079E01281BF7
:106240003109C901181619065CF0CE01019797FFB4
:1062500002C080E090E08093810710E1B12C0BC078
:1062600025303105D4F3CE0104978B3091059CF392
:106270008AE090E0F0CFF0908107FB0CCF2CD12C7E
:10628000CC15DD0511F401E101C000E196012F5F9D
:106290003F4F442737FD4095542F62E0E62E612F93
:1062A00082E10E94425E8091FF04F81205C04AE23A
:1062B000612F81E00E94025D4FE06DE277E08F2D5B
:1062C0000E946356CC15DD0531F48091D9078823EF
:1062D00011F001E101C000E12FE04DE257E0612F34
:1062E00088E10E94055DB394185F36E0B312C3CF16
:1062F000DF91CF911F910F91FF90EF90DF90CF90A2
:10630000BF900895DF92EF92FF920F931F93CF9368
:10631000DF93E82E0091F001C1EBD7E0109160040B
:10632000202F332727FD309537FF03C03195219566
:1063300031092532310554F12D853E854F85588927
:10634000242B352B4B855C85242B352B8989282BD9
:106350008A89282B232B29F4802F881F8827881FC0
:106360008A8B101614F48CED01C084E2800F40E09B
:1063700060E00E949516882341F09A89911105C02A
:1063800091E02989211190E0998B8A8B112339F0B2
:1063900040E060E0812F0E949516882319F0FF24C9
:1063A000F39402C0F12CE12C2D853E852F5F3F4FE9
:1063B0003E872D872F8538892E0D311D388B2F87ED
:1063C000F89420915A0C30915B0C78948B859C85C5
:1063D000281B390B2436310508F423C18C599F4FF3
:1063E0009C878B872F853889ED85FE85C901BF0184
:1063F0000E94D872E62ED62E6E9FC0016F9F900D20
:106400001124281B390B388B2F871E861D868FE0A1
:10641000800F8F3110F4198A0DC094E2900F9934D7
:1064200048F4101614F481EF800F40E060E00E9401
:106430009516898B2091F001332727FD309537FF82
:1064400003C0319521953109622F88819981019688
:1064500099838883EA81FB813196FB83EA83DD207F
:1064600029F08E819F8101969F838E83613009F48C
:10647000698B8989882341F0FF2031F04C815D814F
:106480004F5F5F4F5D834C83E694488559854E0D81
:10649000511D59874887E090F201F090F301FC8A82
:1064A000EB8A611102C01A8620C0613031F41111EB
:1064B00014C0C7018E1B9F0B16C0603170F420FF03
:1064C00006C0E4E056954795EA95E1F702C04E8193
:1064D0005F81C701841B950B06C08C819D8197014C
:1064E000281B390BC9019C8B8B8B8A850B891C89D6
:1064F000813049F018F0823069F017C08091F001C6
:10650000882399F010C017FF10C0E114F10469F05E
:1065100082E00AC0053C3FEF130714F483E08A874A
:10652000E114F10411F481E08A87898D9A8D801736
:10653000910709F46AC08A85813009F057C08091BB
:10654000180582FF31C0E114F10471F10E3111051B
:1065500019F469E289E10BC00431110519F46AE20A
:106560008AE105C00A30110531F46BE28BE10E942B
:10657000386C81E00DC0063011054CF417FD03C0E6
:10658000602F8CE1F4CF8CE10E94326CF2CF80E07E
:106590009091180593FF08C0882331F082E390E0C2
:1065A00090935801809357018091F10180FF04C0BE
:1065B000C701801B910B01C0C8016CE370E00E9411
:1065C000EC72DC01CB014091180541FF1EC0AB2BE2
:1065D000E1F44091210541FF07C0009761F046E2D8
:1065E00060E00E94416C07C080E003C0823069F423
:1065F0008CE10E94326C8091180583FF06C082E313
:1066000090E090935801809357018B899C899A8FD1
:10661000898F2091F10120FF04C0E81AF90AFC8A51
:10662000EB8ADF91CF911F910F91FF90EF90DF9058
:1066300008959091F00197FD91958EEF890F8E301E
:1066400020F5892F85959A3024F40E945C6290E0B1
:1066500003C0992787FD90950197FC01EE0FFF1F5E
:10666000EE55F84F208131818091F00187FF05C000
:1066700080E094E0821B930B02C0C9019C5F26E07E
:10668000969587952A95E1F702C080E090E00E94F8
:10669000823183E00E945C62E82FF0E0EE0FFF1F82
:1066A000E056F84F808191819C5FB6E09695879582
:1066B000BA95E1F72091F10122FF0AC085309105DA
:1066C00038F02091C807211103C023E02093C807A8
:1066D0002091D1073091D2072F5F3F4F3093D207DF
:1066E0002093D1072091CF073091D007280F391F71
:1066F0003093D0072093CF07F89480915A0C909153
:106700005B0C78942091CD073091CE07AC01421BF1
:10671000530B9A01283E3340D8F19093CE078093D3
:10672000CD078091F401823039F440E060E085E1EA
:106730000E949516811128C08091CF079091D007B3
:106740006091D1077091D2070E94D8721092D00741
:106750001092CF071092D2071092D1078091AE0607
:10676000893718F48F5F8093AE06E091AF0681E021
:106770008E0F8093AF06F0E0E055F94F60838837C5
:1067800038F01092AF06089587E00E94326CD4CFA3
:106790000895E1EBF7E012861382128217821682C7
:1067A00015821482118610868091F2019091F30176
:1067B000928F818F0895CF92DF92EF92FF92CF93C5
:1067C000DF936B017C01C0E1D0E040E050E8E0E005
:1067D000F0E89A01DA010E949F72C616D706E80611
:1067E000F90610F44E275F27F695E7952197209735
:1067F00019F04E2B5F2BEDCFCA01DF91CF91FF90A7
:10680000EF90DF90CF9008951F9341E0262F30E066
:10681000683050F440E055E0529FF001539FF00D76
:106820001124E553FC4F0AC02850310959E0529F0A
:10683000F001539FF00D1124ED50FC4F9C5F97FD2C
:106840000DC0811528E0920784F0442319F088E0F8
:1068500090E002C084E090E0E80FF91F2081332728
:1068600027FD3095322F222725C0442329F0492FB8
:106870009927880F991F03C0492F46959170242F9F
:1068800030E0E20FF31F608140E052E0481B590BFB
:106890005595479564039001659F300D1124118132
:1068A000BC01759567951603A001179F500D112423
:1068B000240F351FC90169E170E00E94EC72CB0121
:1068C0001F9108953F924F925F926F927F928F92A5
:1068D0009F92AF92BF92CF92DF92EF92FF920F936F
:1068E0001F93CF93DF93982EBB24B3948091F60728
:1068F000883008F4B12C80E391E10E944F1FBB2047
:1069000011F08AE001C086E0A82ECC24C394FEE2F8
:10691000EF2EF1E1FF2E00E020E030E040E0692DB5
:106920008FEE97E00E946E204091F60750E04F5F97
:106930005F4F21E060E084E20E94525FC091F60761
:10694000BB2061F08C2F90E0089729E0289FE001A0
:10695000299FD00D1124CD50DC4F06C025E0C29FE9
:10696000E0011124C553DC4F6090EF076A94A090BA
:106970005A0741E6941681F0491538F054E495160B
:10698000E1F085E4981689F02EC0E4E69E16A9F0A1
:10699000F5E69F1651F027C0AA2029F110925A0758
:1069A00081E60E944561A12C1EC08091800788234A
:1069B000D1F01A14C4F48FEF13C08091800788239C
:1069C00091F02A2D332727FD3095BB2019F089E05F
:1069D00090E002C085E090E02817390724F481E0B8
:1069E0008A0D80935A0780915A07809380078C2ED6
:1069F0007D2ECC2EDD2E05E010E0E0E15E2EE62CB3
:106A0000FF24E7FCF094F60141916F0121E0C801F9
:106A10000597E816F90609F020E0552747FD50953F
:106A2000652D88E10E94525FBB2091F0093081F012
:106A300021E0E016F10609F020E0FE01E00FF11F71
:106A40004081552747FD5095652D80E30E94525F98
:106A5000F8E05F0E0F5F1F4F28E35212D4CF4FEFC5
:106A6000641202C021E0A11020E047E251E168E099
:106A70008CE00E943B5DBB2019F089E090E002C0F1
:106A800085E090E021E0E816F90609F020E040E218
:106A900051E168E38CE00E943B5DBB2019F089E086
:106AA00090E002C085E090E0E816F9066CF467FC1F
:106AB00050C0EC0EFD1E44E66CE9F70180810E9497
:106AC0009B13F701808345C016140CF042C020E0F0
:106AD00044E06CEF8091EE070E948F138093EE07E5
:106AE000909164019923A9F1BB2021F090E164E029
:106AF00049E003C098E062E045E0F4E68F028001DF
:106B0000112470E0719561957109582F5603900119
:106B1000579F300D112484E6829F6001839FD00C23
:106B20001124E82DF72D20E030E0E92EF12CC901E9
:106B30008C0D9D1DB7010E94EC726193200F311FD7
:106B40008E2F8819841798F382E00E9498570E942C
:106B5000375880918007882309F459C0712C7CE94B
:106B6000E72EFF24FA94CA2CDD24C7FCD094892D8B
:106B70008F7DA82EEEEBAE0E40C0C90155E0880F08
:106B8000991F5A95E1F7BB2009F44AC064E070E010
:106B90000E94EC72462E4E01820E931EF4018081FB
:106BA000F0E28F02C0011124B7010E94EC72662E40
:106BB00040E2542E560E2F5F3F4F052D10E0C216B7
:106BC000D30609F05EC0023411056CF12FE32515E0
:106BD00030F045E0652D8AE3840D0E94F35D0F33AC
:106BE0001105A4F180915C0190915D01892B09F060
:106BF0003FC051E05A15E0F57394272D30E0BB20DB
:106C000061F089E090E0281739070CF4B6CFC0E0B6
:106C1000DCEF10E060E2F62E52C085E090E0F3CFAA
:106C200062E070E0B5CF3AE3332E340C45E06EE11C
:106C3000660D832D0E94F35D0134110539F245E0A4
:106C40006FE1660D832D0E94F35DC0CF4AE3440ED1
:106C500045E061E2660D842D0E94F35D0E3311055F
:106C600009F262E2660D45E0842D0E94F35DBACF21
:106C700044E66CE9F40180810E949B13F401808357
:106C8000BBCFFBE34F0E0134110534F443E06FE159
:106C9000660D842D0E94F35D2FE3251528F043E057
:106CA000652D842D0E94F35D0F3311050CF0A4CFE8
:106CB00061E2660D43E0842D0E94F35D9DCF6091FB
:106CC000F607CE010E9404340CE3010F25E09695EF
:106CD00087952A95E1F76F2D681B802F0E94A65D8E
:106CE000812F837021F460E2802F0E94A65D1F5FD8
:106CF000A096103421F740E460E08CE5DF91CF915D
:106D00001F910F91FF90EF90DF90CF90BF90AF90C9
:106D10009F908F907F906F905F904F903F900C94DA
:106D2000F65D2F923F924F925F926F927F928F9279
:106D30009F92AF92BF92CF92DF92EF92FF920F930A
:106D40001F93CF93DF93CDB7DEB76E970FB6F8944E
:106D5000DEBF0FBECDBF8D8F9E8F69878091590199
:106D6000882309F44EC080917E07882319F0815052
:106D700080937E070E94DC1420916706309168069C
:106D80008217930761F090936806809367061092CC
:106D90006A061092690681E08093560132C06091C4
:106DA0001705665F71F180910201823350F1809185
:106DB0006B068F5F80936B06803118F180916906B6
:106DC00090916A06019690936A06809369061092E4
:106DD0006B0647E751E0649F9001659F300D1124D9
:106DE0002817390770F48F719927019751F486EFAE
:106DF0009FEF0E94CB136DE280E10E94386C0E94ED
:106E0000E9130E94531B80934D0580911605282F8E
:106E10002170822E839481FF02C0612C02C033E076
:106E2000632E4091FD014423F1F1E82DF0E0EE0FD7
:106E3000FF1FEE55F84FA081B181E62DF0E0EE0F77
:106E4000FF1FEE55F84F0190F081E02D9D010E944B
:106E500097726B017C019F01DF010E949772C60E41
:106E6000D71EE81EF91E642F70E080E090E02AE053
:106E7000660F771F881F991F2A95D1F724E630E007
:106E800040E050E00E942273CA01B9010E94C8721A
:106E90006C157D058E059F0530F4C701B6010E9473
:106EA000DB337C0102C0E12CF12C9701A4E6B0E0B9
:106EB0000E949F726D8B7E8B8F8B988FB3ED4B2EC4
:106EC000B4E05B2E4EE056E05C874B87BE016F5FFF
:106ED0007F4F7E876D8782EA97E09A8B898BC12CE2
:106EE000D12C712C99859170998FA985AE70AA8F3C
:106EF000B985BA70BB8FE985E670EC8F9C2C8C2D20
:106F00000E94CC1492012E5F3F4F388B2F87D20105
:106F10002D913C91821B930B9C01BC01882777FD2E
:106F20008095982FAAE0660F771F881F991FAA9552
:106F3000D1F7EF85F889121613061CF4228D338DD4
:106F400002C0248535852436310514F424E630E06A
:106F5000442737FD4095542F0E9422738901213028
:106F6000FCEF3F073CF0011524E012072CF000E095
:106F700014E002C000E01CEF8091180580FF11C0F2
:106F80008091160581708B8B1C8A82E090E04B8982
:106F90005C89841B950BC816D90619F411950195C7
:106FA0001109A989BA890D931D93BA8BA98B580130
:106FB00017FF03C0BFE0AB0EB11CF4E0B594A7947B
:106FC000FA95E1F73A2CE4E0CE16D1045CF481E0C6
:106FD000890D0E945C62815091E001C0990F8A95F1
:106FE000EAF706C091E00C2C01C0990F0A94EAF769
:106FF00037FE02C03A2C3194F1E0F31544F0311021
:1070000002C0892F03C0809166068923782A23E075
:10701000291508F422C1398D31114DC08091F1013B
:1070200081FF49C0520149E3A40EB11CF5018181E1
:10703000807C09F440C0F20181AD40E061E08595BB
:10704000859585950E9495168823A9F1D501EC9127
:10705000E770F0E0DF01AA0FBB1FAA5BBE4FEE0F87
:10706000FF1FEC5FFA4F8D919C9120813181821B33
:10707000930B97FD0196AC0155954795F50121813C
:10708000322F330F330F359535953403C001359FBB
:10709000900D11246FE170E00E94EC72660F771F73
:1070A000660F771F2295269526952370213009F0CB
:1070B0008FC6060F171FE114F104C1F0981411F0E8
:1070C000961014C02091FD0130E0D8010E94AE72EC
:1070D000EAE0660F771F881F991FEA95D1F72D897F
:1070E0003E894F89588D0E9422738901892D0E9403
:1070F000021FA82E892D0E947216EA2DF0E0882327
:1071000011F1EE0FFF1FEE0FFF1F2EE02C9DC001AF
:107110002D9D900D1124E80FF91FE157FC4F808140
:107120000E946416682F772767FD7095C8019C5FE1
:1071300097FD0196959587950E94D9298C01000F9E
:10714000111FB12C24C081E0101611060CF480E050
:10715000B82E3EE03C9DC0013D9D900D1124EE0FE8
:10716000FF1FEE0FFF1F8E0F9F1F8B519E4F8B0D2A
:10717000911DFC01E655FE4F80810E946416682F28
:10718000772767FD7095C8010E94D9298C014EE0D0
:107190004C9DC0014D9D900D112454E0A59E800D85
:1071A000911D11248B519E4F8B0D911DFC01E455B7
:1071B000FE4F808144E660E08C590E944B16980196
:1071C000A82FBB27A7FDB0950E94977224E630E058
:1071D00040E050E00E9422738901892D0E947216BE
:1071E00081111450892D0E946816811106C0692DE5
:1071F00080914D050E9496122AC08091F60180FF71
:10720000F6CF692D80914D050E949612282F80910E
:10721000180580FD2195332727FD3095432F532FE7
:1072200023583F4F4F4F5F4FA0E0B4E0A01BB10B7E
:107230000E94C07220E038E040E050E00E942273DB
:10724000211568E036074105510589F2C901880F0B
:10725000991FAD85BE858D939C93EB85FC8511832D
:107260000083FA8DFF23F9F023E02915E0F0892D42
:107270000E946816811113C03B8D332349F0065FCD
:107280001F4F0531110520F0AB85BC851D921C9266
:10729000BC8DBB2321F0ED85FE8511821082EB852C
:1072A000FC85118E108EFFEFCF1ADF0A2B853C85EF
:1072B0002E5F3F4F3C872B874D855E854E5F5F4F2E
:1072C0005E874D8757E0C516D10419F04F84588862
:1072D00015CE1091FA0117218091660680958123C1
:1072E00019F088E10E94326C1093660680E094E009
:1072F00090931D0680931C0690931F0680931E0694
:1073000082E10E94F460811108C083E10E94F46070
:10731000882331F080E090E005C080E09CEF02C05F
:1073200080E094E0909357068093560626E431E07F
:1073300006E216E0E4E0F5E060E0D9018D919D9170
:107340009D01643020F440815181841B950B880F8E
:10735000991FD8018D939D938D016F5F3296683090
:1073600061F726E336E0ECE6F6E041915191619158
:107370007191D9014D935D939D01B6E0EC3AFB0705
:10738000A1F7ECE9F4E0A8E5B6E0808128E082020C
:10739000C00111248D939D93329634E0EA3AF307AD
:1073A000A1F7A090FD01AA2009F46EC0E82CF12CF1
:1073B000EE0CFF1CA701425F594F7A01DA01CD9014
:1073C000DC90062D10E0000F111F025F194FF8012D
:1073D000408151819601D6010E9497721B012C01B8
:1073E0009A01DA010E949772260E371E481E591E16
:1073F0006A2D70E080E090E0EAE0660F771F881F5A
:10740000991FEA95D1F724E630E040E050E00E9471
:107410002273CA01B9010E94C872621573058405FE
:10742000950590F5C201B1010E94DB339C01A4E6F1
:10743000B0E00E949F721B012C01B12C9501D60176
:107440000E94AE722AE0660F771F881F991F2A9547
:10745000D1F7A20191010E942273D7012D933C9391
:10746000F801A081B18195010E94AE723AE0660FE9
:10747000771F881F991F3A95D1F7A20191010E94A9
:107480002273D8012D933C936091FB01862F807E5F
:1074900009F4F8C089858A7089F4E82DF0E0EE0FD0
:1074A000FF1FE25FF94F20813181E62DF0E0EE0F02
:1074B000FF1FE25FF94F8081918104C080E090E07E
:1074C00020E030E049854670A1F4FE013196E80DD8
:1074D000F11DE80DF11D40815181240F351FFE0182
:1074E0003196E60DF11DE60DF11D40815181840FAD
:1074F000951FE091FC01EE2341F0F0E0EE0FFF1F3D
:10750000E45FF94F4081518102C040E050E062FFEA
:1075100003C031952195310963FF03C09195819591
:10752000910964FF03C05195419551096295669593
:107530006770623009F451C018F46130E1F0A2C004
:10754000633009F489C0643009F09CC0FA01E21B81
:10755000F30BF0932106E09320069A01280F391FC0
:107560003093230620932206481B590B509325067F
:107570004093240687C0BC0197FF02C0695F7F4F1C
:10758000B3E075956795BA95E1F7FC01E61BF70B3B
:10759000BC0197FF02C061587F4F660F672F661FBF
:1075A000770BE61BF70B97FF02C081509E4FBC0183
:1075B000672F770F770B6595CF01861B970BBA0165
:1075C000621B730B709321066093200637FF02C085
:1075D0002F5F3F4F3595279546C0B90137FF02C051
:1075E000695F7F4F13E0759567951A95E1F7F9018B
:1075F000E61BF70BB90137FF02C061587F4F660FDA
:10760000672F661F770BE61BF70B37FF02C0215071
:107610003E4FB901672F770F770B65959F01261BAA
:10762000370BBA01681B790B709321066093200613
:1076300097FD019695958795840F951FAC01420F94
:10764000531F5093230640932206821B930B909363
:1076500025068093240616C0BA01621B730B709333
:10766000210660932006240F351FA901480F591FDA
:107670005093230640932206281B390B309325068E
:10768000209324068091590181110E94193380E4CE
:10769000ECE6F6E0DF011D928A95E9F787EC93E0CE
:1076A000909304018093030188EC93E0909306018A
:1076B0008093050189EC93E0909308018093070182
:1076C0008AEC93E090930A0180930901EEEEF5E0D5
:1076D000FA87E9872EE835E0388B2F874EE455E0AE
:1076E0005E874D87312C212C832D0E9430107C0128
:1076F000FC0182810E9464168B87D7018C91815096
:10770000803108F06AC240E061E0F70183810E94A5
:107710009516811116C0A985BA85DC901C92F701D7
:10772000918188EF890F823008F041C2878186708D
:10773000843009F43CC2993009F047C000E01CEFE6
:1077400046C0DD24D394A985BA858C918111D12CB2
:1077500081E0E985FA858083F70121818FEF820F2F
:10776000A82FB0E0FD01EE0FFF1FE25FF94F00818F
:107770001181843150F0831540F4AA0FBB1FAA0F6A
:10778000BB1FA459B94F0D911C91F7013781832F6D
:10779000807361F0832F82958370815041E050E0C7
:1077A00002C0440F551F8A95E2F7242A36FF0FC006
:1077B000253068F4E22FF0E0EE0FFF1FEF5FFE4F81
:1077C000C70108969183808302C000E010E0F701B2
:1077D0008781887459F48085882341F04DE763E8F8
:1077E0000E944B160E948016080F191FF701F681A0
:1077F000FB8B2B85332727FD30953A8B298BF11195
:1078000005C0F7018581882309F4F0C0AD85BE85E8
:10781000AD90BC90EF85F88980819181A2819C0117
:107820004A2F552747FD509529013A01D1100AC02A
:10783000BB2757FDBA95A52F942F832F6801C81A2F
:10784000D90A3EC0F701878186708430D9F4E0817F
:10785000F0E0EE0FFF1FEC5CF94FA081B18120E05A
:1078600034E60E94AE722B013C01FB85FF2351F0F0
:107870002F2F332727FD3095432F532F0E9422733C
:1078800029013A01C301B20120E031E040E050E0BB
:107890000E94227350954095309521953F4F4F4F50
:1078A0005F4F6801C20ED31EC114D10449F0F70125
:1078B0008581D7FE82958F70F4E68F9F5001112449
:1078C000A114B10491F080915901882331F021E095
:1078D000A21AB108A114B10441F0332777FC3A95FC
:1078E000272D162D052DC12CD12CAD85BE85AD9231
:1078F000BC92C114D10409F474C04801AA2497FCB5
:10790000A094BA2CBB89BB2309F467C080915901AC
:10791000882309F443C0EB85EE23A1F029893A8935
:1079200037FF03C0319521953109442737FD409534
:10793000542F60E070E080E293E00E942273CA015D
:10794000B90104C060E070E080E293E0F7012681B5
:107950001C141D0444F090958095709561957F4F9F
:107960008F4F9F4F22952F7030E02115310591F0F8
:10797000E4E6E29FA001E39F500D11249A01442701
:1079800037FD4095542F0E942273420E531E641EF1
:10799000751E04C04424582C692C7A2CBB2777FC14
:1079A000BA95A72D962D852D1C141D0434F4881628
:1079B0009906AA06BB0634F009C088159905AA05E0
:1079C000BB0524F44424582C692C7A2C332777FCEB
:1079D0003A95272D162D052D04C04424582C692CCA
:1079E0007A2CAF85B8894D925D926C92F7018781B0
:1079F00087FF28C044E66CE984810E944B16A82FBB
:107A0000BB27A7FDB0951A161B0644F417FF6AC0E2
:107A100024E630E02A1B3B0BD90109C0109709F47A
:107A200061C0101611060CF05DC0AC59BF4F980133
:107A30000E94977224E630E040E050E00E942273FA
:107A4000890150C0F7016481862F992787FD9095A1
:107A5000A92FB92F8730910590F5FC01EC5AFF4F03
:107A60000C944173F7018181893021F417FD35C0F1
:107A700012500BC017FF36C01BC0F701818189303F
:107A800039F41016110664F11E5F000F111F2AC091
:107A9000101611066CF026C017FF24C01195019531
:107AA000110920C010161106DCF002C017FD15C028
:107AB00000E010E017C01016110694F00EC067FF2A
:107AC00006C0119501951109F6E0F61B6F2F67505E
:107AD000C8010E9404348C0105C000E01CEF02C004
:107AE00000E014E0F701478140FD10C081819FEF65
:107AF000980F943058F4FE013196E80FF11DE80F0D
:107B0000F11D329780819181080F191F9801A98971
:107B1000BA890E9497724B015C014874483051F455
:107B2000F7018085882331F04DE763E80E944B160A
:107B30000E948016D7010C9110E001501109F70145
:107B4000878186958370000F111F000F111F8130F0
:107B500071F0823029F1F801E459F94F8081918167
:107B6000A281B381880E991EAA1EBB1E19C0C50131
:107B7000B40124E630E040E050E00E942273F801B6
:107B8000E459F94F60817181828193810E94C872AA
:107B900020E034E040E050E00E94227349015A01A5
:107BA000F801E459F94F80829182A282B382339422
:107BB00029853A852F5F3F4F3A8729874F85588916
:107BC0004D5F5F4F588B4F876D857E856E5F7F4F12
:107BD0007E876D8770E2371287CD1091590C20FE99
:107BE00005C0111103C08EE10E94326C21FE07C056
:107BF000812F877F803419F48FE10E94326C22FE3E
:107C000009C0812F877F803811F0103919F480E284
:107C10000E94326C82E897E09E878D879D8D9987C0
:107C2000AE8DAA8733E6232E34E0332EECE6F6E061
:107C3000FC87EB87E12CF12CEF86AB85BC854D9062
:107C40005D906D907C90C301B20124E630E040E08D
:107C500050E00E942273EB85FC8521933193419380
:107C60005193FC87EB87AD85BE852D933D93BE87F1
:107C7000AD878E2D0E9437104C01FC0183819481C9
:107C80002181FAE02F026001112428E1C21A2CEFB1
:107C9000D20AD4012C91BAE02B0250011124E8EE53
:107CA000AE1AE3E0BE0A3C2D2D2D8C159D0514F473
:107CB000382F292F032F122F0A151B050CF48501CD
:107CC0004114510461047104A9F077FE04C0D80185
:107CD000AA19BB0903C0D601A01BB10BA3019201D5
:107CE0000E94C07220EA36E841E050E00E94227310
:107CF00029013A01C8010E9435168C01040D151D99
:107D0000C6010E9435166C01C5010E943516C016C9
:107D1000D1060CF48601081719070CF48C01F40144
:107D20008281882319F011950195110980916104D0
:107D3000F0E1F81B2F852F17F8F4F701EE0FFF1F66
:107D4000EE59FB4F9081892F880F880F8595859577
:107D500099F092959695969593709D5F9370923059
:107D600058F040E060E00E949516882329F0D10188
:107D70008C910E9480168C01F894E985FA85019314
:107D80001193FA87E9877894FFEFEF1AFF0A22E050
:107D9000220E311C30E1E316F10409F04DCF6E964E
:107DA0000FB6F894DEBF0FBECDBFDF91CF911F910C
:107DB0000F91FF90EF90DF90CF90BF90AF909F908A
:107DC0008F907F906F905F904F903F902F9008958D
:107DD000223009F070C98B016EC9FF920F931F9377
:107DE000CF93DF93CDB7DEB7C054D1090FB6F89467
:107DF000DEBF0FBECDBF63E0CE0181960E949136FB
:107E000061E0CE0101960E949136E1E4F3E09E012B
:107E10002F5D3F4F8E010F5F1F4F41815281808147
:107E2000882329F0D9018D919C91D80104C0D801F3
:107E30008D919C91D9016D917C91861B970B840F3C
:107E4000951F883EB3E09B073CF489314CEF9407C3
:107E50003CF0482F892F02C048EE83E0942F02C0E7
:107E600098E18CEF9183828335962E5F3F4F0E5FB2
:107E70001F4F83E0E139F80781F607EC13E0F12C9E
:107E80008F2D0E946816811102C0D8011C92F394B4
:107E90000F5F1F4FB4E0FB12F3CF86E00E949857AC
:107EA00081E00E94326CC05CDF4F0FB6F894DEBFF9
:107EB0000FBECDBFDF91CF911F910F91FF9008951D
:107EC0009F92AF92BF92CF92DF92EF92FF920F9369
:107ED0001F93CF93DF93C82F80911405282F2F7005
:107EE000F22E807310927101C038E9F198F4C33218
:107EF00009F462C030F4C03261F1C23209F46BC0DF
:107F0000ACC0C53209F44DC008F441C0C13609F413
:107F100084C0A3C0C43881F158F4C23809F469C0E0
:107F200008F487C08AEC9FE10E94B51383E868C01B
:107F3000CE38C9F0CF3B09F482C0C53809F08DC0F6
:107F400081E080937C078FEE96E40E94311B85E8E8
:107F50001BC043E0241381C08091C80791E08927AA
:107F60008093C8076AC081E080937C070E94AB13AE
:107F70000E94311B8C2F08C081E080937C0781E632
:107F800090E30E94311B84E80E94456166C052E084
:107F9000251363C08091F0078F5F833054F080E039
:107FA00008C082E0281359C08091F007815087FDF6
:107FB00082E08093F00751C0F39493E09F1508F49A
:107FC000F12C8F298093140581E00E94985783E15A
:107FD0000E94326C42C0222311F0FA9402C003E0E6
:107FE000F02E8F298093140581E00E94985784E138
:107FF000EFCF0E94256E8EEC9EE60E94B51382E8BC
:10800000DF91CF911F910F91FF90EF90DF90CF9074
:10801000BF90AF909F900C9445618091BB078230D8
:1080200021F483E08093BB0708C0E3E02E1315C062
:1080300002C00E94C9330E94C41387E1C9CF81E006
:108040000E94456183E00E94456182E00E94456193
:1080500081E08093CC071092F00740E060E08091CF
:10806000F9010E949516C82F882331F08091CC0722
:10807000811102C00E94ED3EC093CC079091020195
:1080800080910105981710F4C6E001C0C4E080E0BB
:108090000E9413124C2F406860E185E20E94AE10EE
:1080A00046E568E186E20E94025D8091BB07882375
:1080B000A1F0823011F426E001C024E04091C40711
:1080C0005091C507022F60E18DE50E943E1020E02F
:1080D00040E068E183E30E943A1100E02091F7015B
:1080E00045E058E060E186E20E94275D8091F6015C
:1080F00080FF06C041E058E060E188E30E94615DD6
:10810000C0E0D0E01FE1D12EEC2EFE01E350F84F8D
:1081100014916C2F80914D050E94961297FD039645
:108120009C013595279535952795243E0CF424EE32
:10813000022F2D310CF00CE18FEF8E0D46E38230D3
:10814000E0F464E0812F0E94F65D809116058E2593
:1081500080FD04C08091F60180FD0CC043E06EE11B
:108160008FEF810F0E94F65D43E06EE181E0810FA9
:108170000E94F65D6D2D601B14C06BE385EE810FD0
:108180000E94F35DEE24EA94E10E43E06AE38E2D53
:108190000E94F35D43E06CE38E2D0E94F35D100FAF
:1081A0006BE347E0812F0E94251F2196C430D10543
:1081B00009F0AACFF1E0FF1508F47FC00BE517E046
:1081C000E12CF9E1DF2EABE1CA2EF801C191D1918A
:1081D0008F018E2D8370F1E0FF1641F19E01D7FFD4
:1081E00002C0215E3F4FE5E035952795EA95E1F71E
:1081F000AE01421B530B9A01D7FF02C0C158DF4F9B
:10820000AE01440F452F441F550B420F531F6E2DD7
:1082100066956695660F660F660F685D8C9D802D6E
:10822000112420E28F5D0E94525F42C053E05E1530
:1082300018F062E2962E02C05EE5952EB82EBB0CB9
:10824000BB0CB80E9E01D7FF04C0222733272C1B7E
:108250003D0BD29EA001D39E500D11249A013E5F8A
:10826000A32EA594A59489E18A1514F449E1A42EBE
:1082700025E543E366E26B0D87EE890D0E94C35D41
:1082800045E064E26B0D892D0E94F65D1C161D060B
:1082900014F4939401C09A1867E26B0D4A2D892D4E
:1082A0000E94F35D6B2D6B5D4A2D892D0E94F35D5D
:1082B000E39498E0E91289CF7CC0E2E0FE126FC03F
:1082C0000E9418268091F007882329F0982F990F93
:1082D000890F880F8D5F182FC82FDD27C7FDD09518
:1082E0006E01F2E0CF0ED11CE12EFF24E7FCF094EA
:1082F000CE14DF04FCF0BB24B394B10E40E060E088
:108300008B2D0E949516082F0E943711AC0123E097
:108310001202400D511D1124B7016C1B7D0B6C5FC7
:108320007F4F660F660F660F23E08AE00E94055DAF
:108330001B2DDACF8091F0078F5F182F110F180FC8
:10834000110FC12FDD27C7FDD0956E0142E0C40E8D
:10835000D11CE12EFF24E7FCF094CE14DF044CF195
:10836000BB24B394B10E40E060E08B2D0E949516C3
:10837000082F0E943711AC01E3E01E02400D511D91
:108380001124B7016C1B7D0B6C5F7F4F660F660F6E
:10839000660F23E084E60E94055D1B2DDACF409135
:1083A000C6075091C70704E024E068E28CE30E940E
:1083B0003E10DF91CF911F910F91FF90EF90DF90D2
:1083C000CF90BF90AF909F900895982F8091810794
:1083D0001916BCF4292F332727FD3095281B3109A6
:1083E000462F50E0421753071CF4892F861B0AC002
:1083F00046505109241735072CF4892F861B8A5FB4
:1084000001C080E0809381070895BF92CF92DF92F0
:10841000EF92FF920F931F93CF93DF93C82E4EE0FE
:10842000682F87EE97E00E94D8228091F207882378
:1084300019F080E29FE002C086E19FE00E944F1F9A
:10844000182F8091F5070E943010EC0120E0488140
:1084500060E086E0810F0E94E310D090E70766E0BD
:108460008D2D0E94E54118E0F12CBB24B39440917E
:1084700081074F0DEE24E394D412E12C50E04F30ED
:10848000510508F045C1FA01E55AFF4F0C944173BC
:108490006EE07FE0812F0E945B5D2E2D206149817F
:1084A000612F84E50E94B310EE2009F431C14CE243
:1084B00061E089810E949B1389832AC166E07FE085
:1084C000812F0E945B5D0DE723E84A81612F80E6E2
:1084D0000E949F1E8A831CC18F8186FF03C04CEFC0
:1084E0005EE002C045EF5EE0612F8CE00E94615DBE
:1084F0000DE723E84885612F80E60E949F1E88874C
:1085000007C18F812E2D49EE5EE0612F83FB882706
:1085100080F90E9465279F8180FB93F90DC08F81B0
:108520002E2D4DED5EE0612F86FB882780F90E949D
:1085300065279F8180FB96F99F83EAC08F818170B8
:108540002E2D47ED5EE0612F9B2D981B892F0E94F9
:1085500065279B2D981B8F8190FB80F98F83D8C056
:108560000F8107FB002700F9002319F041ED5EE0C1
:1085700002C04BEC5EE02E2D612F8CE00E943B5D33
:10858000EE2059F08F8187FB882780F961E00E94F7
:108590009E139F8180FB97F99F838F8187FB88279C
:1085A00080F9081709F4B4C01C82B2C08F8187FF1C
:1085B00009C004E62CE94C81612F80E60E949F1ED1
:1085C0008C83A6C02E2D4C81612F82E10E94CD2785
:1085D000EE2009F49DC046E160EF8C810E949B1360
:1085E0008C8387300CF494C090E6C91291C08750F8
:1085F0008093F60782E694E30E94311B89C063EC06
:108600007EE0812F0E945B5D0E2D2E2D4B81612F10
:108610008EE40E94BB278B837BC06AEB7EE0812FB8
:108620000E945B5D0F810295037049F0402F50E07E
:108630002E2D2064612F84E50E94525F07C02E2DED
:1086400045E853E0612F8EE40E943B5DEE2009F483
:108650005FC063E0802F0E949E1383708295807FAD
:108660009F819F7C1CC062EB7EE0812F0E945B5D3E
:108670002F81269523700E2D48E95EE0612F8EE450
:108680000E94275DEE2009F443C08F81869562E049
:1086900083700E949E138370880F9F81997F982B0F
:1086A0004BCF4D8142954F702CE83EE06E2D812FCF
:1086B0000E942F1D8295807F9D819F700BC04D81F0
:1086C0004F7022E83EE06E2D812F0E942F1D8F708B
:1086D0009D81907F982B9D831BC04E8142954F704A
:1086E00026E73EE06E2D812F0E942F1D8295807F10
:1086F0009E819F700BC04E814F702CE63EE06E2D28
:10870000812F0E942F1D8F709E81907F982B9E83BA
:10871000F394185F87E0F812AACEDF91CF911F91F2
:108720000F91FF90EF90DF90CF90BF9008956F92E0
:108730007F928F929F92AF92BF92CF92DF92EF92F1
:10874000FF920F931F93CF93DF93C82F89E191E19D
:108750000E944F1F40E1E42E0CE02EE531E147E09E
:108760006C2F8DEE97E00E94C722E090ED07EA940F
:1087700066E08E2D0E94E541C03611F0C43641F40A
:10878000E7FC06C0E092F60782E694E30E94311B04
:10879000A12CB12CCC24C39498E0D92EFF24E7FC63
:1087A000F09425E0922E39E0832EC0918107CA0D06
:1087B0000C2F10E0D1E0E016F10609F0D0E07724AC
:1087C0007394C83028F4712C87E08C1528F45FC0AE
:1087D000E6E0EC1508F45BC0B11002C0BD2E02C08B
:1087E000BB24B3942D2F46E151E16D2D80E00E9412
:1087F0003B5DA8014F5F5F4FC93010F482E101C0BB
:1088000087E12D2F6D2D0E94525F772051F0085087
:108810001109809EE001819ED00D1124CD50DC4FC6
:1088200007C0909EE001919ED00D1124C553DC4FEE
:108830008E018AE2682EF80141918F01552747FD8C
:1088400050956D2D862D0E94615FF5E16F0E83E9D5
:108850006812F1CF08E00D0D711002C0C39411C071
:1088600025961AE24991552747FD5095602F812F93
:108870000E94615F1B5E1E37A9F700E10D0DC394D6
:10888000C394A394E7E0AE1611F0D02E8ECFB110B2
:1088900005C0809181078F5F80938107DF91CF9121
:1088A0001F910F91FF90EF90DF90CF90BF90AF900E
:1088B0009F908F907F906F900895BF92CF92DF929C
:1088C000EF92FF920F931F93CF93DF93C82F88E807
:1088D00090E10E944F1FFAE0EF2E0CE02EE531E10F
:1088E0004AE06C2F8AEE97E00E94C7221091EA07B7
:1088F000115066E0812F0E94E541B82EC03899F4EE
:1089000080E80E94456189E180937E07193019F45F
:108910000E94FC6105C0183018F4812F0E94696222
:1089200081E00E94326CE8E0FE2EC12EDD24C7FCFF
:10893000D09488E0B81205C080917E07882389F121
:1089400034C0CB2DD0E0CC16DD0611F401E101C01E
:1089500000E19E012F5F3F4F442737FD4095542F84
:1089600072E0E72E6F2D82E10E94425E80917E07C9
:10897000811104C021E0CC16DD0609F020E0FE01E3
:10898000EE0FFF1FEB52F34E459154916F2D88E18E
:108990000E943B5D88E0F80EB39480E4F812C9CFE2
:1089A0004EC0DD24D394183009F0D12C69E770E172
:1089B0008F2D0E945B5D5AE5C52EC6E0D0E0E091A8
:1089C0001B05F0E0E757FC4F449150E00C2E02C02D
:1089D000559547950A94E2F7437055274C585F4EDA
:1089E0000D2D21E06F2D8C2D0E94055D229786E0D4
:1089F000C80E82E7C812E3CFDD2039F067E180912D
:108A00001B050E94A61380931B0568E06F0D693358
:108A1000B0F480917E07811103C021E0193009F084
:108A200020E040E650E186E0DF91CF911F910F9169
:108A3000FF90EF90DF90CF90BF900C943B5DDF9163
:108A4000CF911F910F91FF90EF90DF90CF90BF904B
:108A500008952F923F924F925F926F927F928F92E2
:108A60009F92AF92BF92CF92DF92EF92FF920F93BD
:108A70001F93CF93DF9300D000D0CDB7DEB7282E61
:108A800086EE9DE00E944F1F80912A07882321F0E7
:108A90000E94EB28182F01C010E080915907811126
:108AA0000BC0E09058070CE02EE531E145E0622D67
:108AB00086EE97E00E94C7226090E6078091C7018A
:108AC000803621F08F3B31F08E32A1F490912A074D
:108AD000992319F010922A070DC09091590791110E
:108AE00009C00E9445611092C701611007C0109231
:108AF0002A0702C06620D9F3198202C081E0898367
:108B000067E0862D0E94E541382E8091590781113A
:108B10001092C70180912A07882369F011160CF47E
:108B200056C1111156C18091C701823609F44FC157
:108B3000833609F44EC14424439411E0512CA32CF4
:108B4000B12C852D0E9430107C01311678F4612FF4
:108B500070E06A197B096830710544F4660F660F8E
:108B6000660F20E0442D81E00E94E3109FE19515FF
:108B700008F4C8C0F701F081FA83F411C3C0C7013B
:108B80000A969C838B83F52CCB80DC809AE0C91AF3
:108B9000D108311608F0A3C0812F90E08A199B09F3
:108BA000883091050CF08CC0782E770C770C770C00
:108BB00080912A07811113C0611211C0F092F5074C
:108BC000EA81E093F307F981FF2359F010922B0714
:108BD00081E080935907EE24E394212C04C0E12C1A
:108BE00002C0EE24E3945F1459F0F6012781269524
:108BF000237000E041EE5DE0672D83E10E94275D78
:108C000020E1EB81FC8139974081672D80E30E9450
:108C1000B3100DE723E88B809C80F8E08F1A910851
:108C2000F4014081672D8DE20E949F1EF401808334
:108C3000EB81FC8137974081442329F020E0672DA8
:108C400088E40E940511EB81FC8136974081442322
:108C500079F0F601878120E087FF06C044E6672DA2
:108C600080E60E94505C04C0672D80E60E94CD27FC
:108C7000F6018681811102C040E201C043E5F601A0
:108C80008581882329F0433511F44AE201C044E488
:108C9000672D89E70E94025D80912A078823F9F0F9
:108CA0008091F4078F111BC020E046E6672D88E114
:108CB0000E94895DF092F5071093E607612E0FC0C0
:108CC000089769F480912A07882349F08091F40776
:108CD0008F1105C08091E6078F5F8093E6071F5FC5
:108CE000F394F0E2FF1609F448C08B819C810A9648
:108CF0009C838B83FC013A9780819A81891709F4C0
:108D000043CF3BC0611237C04092F3075092F50742
:108D1000662D6A19660F660F660F615029E049E1FA
:108D200080E00E94645FE981EE2329F10E942F28F0
:108D3000811121C060E08091F5070E94601D1092B2
:108D40002A0785E092E40F900F900F900F90DF912B
:108D5000CF911F910F91FF90EF90DF90CF90BF9038
:108D6000AF909F908F907F906F905F904F903F90CB
:108D70002F900C94311B1F5FF52C4394F1E14F169B
:108D800011F05F2CDECE80915907882331F02092BC
:108D9000C7010E943D291092800711501093580777
:108DA0000F900F900F900F90DF91CF911F910F9127
:108DB000FF90EF90DF90CF90BF90AF909F908F90FB
:108DC0007F906F905F904F903F902F90089561E05B
:108DD00001C060E08091F5070E94EB27ACCE6F9256
:108DE0007F929F92BF92CF92DF92EF92FF920F936A
:108DF0001F93CF93DF93D82E8DE49AE00E944F1FEC
:108E00001EE1E12E06E022E531E140E06D2D83ED2B
:108E100097E00E94C7221091D307E0905A0767E0BD
:108E2000812F0E94E541F82E87E1F81208C01A311F
:108E300010F48FEF01C081E0D7E1FD2EF80E91E62E
:108E4000D916B1F09D1558F084E4D81661F18D154E
:108E500020F092E4D916E0F541C085E406C094E61E
:108E6000D91609F1D916A0F185E6D81659F036C001
:108E700080918007882391F11092800781E60E94FB
:108E800045612CC0113039F4EE2041F1809180070A
:108E9000882321F104C0163109F5EE20F9F0809104
:108EA0005A0781500CC0113069F498E09E15B0F05B
:108EB00080918007882391F080915A078F5F80937B
:108EC0005A070CC0163151F486E08E1538F0F4CFF5
:108ED00080918007811102C010925A07F1107EC064
:108EE00062E47AE088E00E945B5D113031F48091A9
:108EF0008007811102C001E101C000E12AE043E2E4
:108F000055E068E082E40E94055D80918007811150
:108F10000BC080917D0787FF07C081E080938007A9
:108F200010927D0710925A0780918007882381F064
:108F300020917D07332727FD30958E2D90E08217F5
:108F4000930734F41092800710927D0710925A070D
:108F5000113009F071C480918007882309F46CC432
:108F600080915A0790917D07891B87FD03C08093EC
:108F70005A0702C010925A0780915A078A301CF093
:108F800089E080935A0710927D07CE2DD0E0CE5213
:108F9000DB4FFE01EF5AFF4F80810E94C72E2091C8
:108FA0005C0130915D01232B29F49D2D9F7D92540E
:108FB000923018F461E40E94A6130E94D92ECF5A71
:108FC000DF4F88839E2D990F9E0D990F21E0482F2A
:108FD00068E082E4890F0E94505C2EC491E09F15E6
:108FE00048F1D8E0C0911505C695C695C695C770DD
:108FF0006BE37AE08D2F0E945B5D123089F466E0AE
:109000008C2F0E94A613C82F8770880F880F880F97
:1090100090911505977C982B9093150501E001C060
:1090200000E02C2F4FE05AE06D2F8CE50E94275D69
:10903000D85F04C082E0F8121DC0D8E0C0912105BD
:1090400064E07AE08D2F0E945B5D133049F463E0A9
:109050008C2F0E94A613C82F8093210501E001C028
:1090600000E02C2F4AED59E06D2F82E40E94275D2D
:10907000D85F04C093E0F91231C0D8E0C0912E054A
:10908000C95F63ED79E08D2F0E945B5D143039F488
:1090900067E08C2F0E94A613C82F21E401C020E4B2
:1090A0004C2F50E06D2F86E60E94525F40912E05B6
:1090B000552747FD50952C2F332727FD30952750F6
:1090C00031094217530729F0C750C0932E050E945B
:1090D000E913C8E0CD0FC93328F0B0C384E0F8121B
:1090E0001EC0C8E064EC79E08C2F0E945B5D1530F7
:1090F00051F444E661E080911F050E94A313809320
:109100001F0521E401C020E440911F0550E06C2FB1
:1091100086E60E94525FC85FC93328F08FC395E08E
:10912000F9121DC0C8E063EB79E08C2F0E945B5DF3
:10913000163049F465E0809120050E94A6138093C3
:10914000200521E401C020E44091200550E06C2F6F
:1091500086E60E94525FC85FC93328F06FC386E07D
:10916000F81220C0C8E06AEA79E08C2F0E945B5DAB
:10917000173061F44DE26AE0809100050E94A3136C
:10918000809300050E94126021E401C020E4409118
:10919000000550E06C2F86E60E94525FC85FC9331D
:1091A00028F04CC397E0F9121DC0C8E06AE979E0E5
:1091B0008C2F0E945B5D183051F448E768E2809183
:1091C00001050E94A3138093010521E401C020E45E
:1091D000409101056C2F86E60E949810C85FC93344
:1091E00028F02CC388E0F81222C0C8E067E879E0D4
:1091F0008C2F0E945B5D193051F44EE666EF809132
:1092000017050E94A3138093170521E001C020E0F9
:1092100040911705552747FD5095465F5F4F6C2FCE
:1092200080E70E94525FC85FC93328F007C399E006
:10923000F91217C0C8E021E01A3009F020E080914F
:10924000180546E759E06C2F81700E9445279091E0
:10925000180580FB90F990931805C85FC93328F072
:10926000EDC28AE0F81218C0C8E021E01B3009F016
:1092700020E0809118054AE659E06C2F86958170B0
:109280000E9445279091180580FB91F9909318054D
:10929000C85FC93328F0D2C29BE0F91219C0C8E0F8
:1092A00021E01C3009F020E0809118054BE559E0E1
:1092B0006C2F82FB882780F90E9445279091180522
:1092C00080FB92F990931805C85FC93328F0B6C2A5
:1092D0008CE0F81219C0C8E021E01D3009F020E050
:1092E000809118054DE459E06C2F83FB882780F9A5
:1092F0000E9445279091180580FB93F990931805DB
:10930000C85FC93328F09AC29DE0F9121DC0C8E0B9
:1093100060E479E08C2F0E945B5D1E3051F446E1E1
:109320006AEE809103050E94A3138093030521E058
:1093300001C020E0409103056C2F80E60E940511DA
:10934000C85FC93350F07AC28EE0F81629F0D8E031
:1093500000E0C0E1BC2E4CC0C8E021E01F3009F0A5
:1093600020E080911E054FE259E06C2F86FB882794
:1093700080F90E94452790911E0580FB96F99093F5
:109380001E05D8E0DC0FD93318F358C2011133C0E1
:109390006FE179E08D2F0E945B5D01112FC0C091BC
:1093A0001A051B112EC068E78C2F0E94A613C82F28
:1093B00021E0CC2341F1206495E0C99FA001112454
:1093C0006D2F86E60E94525F43E76D2F8091580C07
:1093D0000E94025D01111EC0C0931A05D85FD933E7
:1093E00008F02CC281E08B0D0F5F8231B1F0B82EF6
:1093F000FB14C0F7CBCF6FE079E0CCCFC091220552
:10940000D0CF20E0D6CF45E853E06D2F86E60E940E
:109410003B5DE0CFC0932205E1CF81E18F15E0F005
:1094200021E0123109F020E08091180582958170C9
:10943000C1E041E059E06D2F9C2F981B892F0E94BD
:109440004527C81B80911805C0FB84F98093180537
:10945000D85FD93308F0F2C182E08B0DF816D8F44A
:1094600021E0181320E080911E0582958170C1E0F3
:1094700045EF58E06D2F9C2F981B892F0E944527A0
:10948000C81B80911E05C0FB84F980931E05D85F20
:10949000D93308F0D3C183E08B0DF816D0F421E066
:1094A000181320E0809115058170C1E044EE58E06A
:1094B0006D2F9C2F981B892F0E944527C81B8091D8
:1094C0001505C0FB80F980931505D85FD93308F0E6
:1094D000B5C184E08B0DF816D8F421E0181320E014
:1094E0008091150586958170C1E04DEA52E16D2F9E
:1094F0009C2F981B892F0E944527C81B809115051A
:10950000C0FB81F980931505D85FD93308F096C167
:10951000B5E0CB2ECB0CFC1408F079C069ED78E0F7
:109520008D2F0E945B5DA9E26A2EA2E17A2EC2E431
:109530009924939480912D05892101E009F400E09C
:1095400021E0A3016D2F8C2F0E94055D990CCA5F4D
:109550008FEF681A780AC23769F71C1154C08091DE
:109560005A0790917D07891B87FD03C080935A0796
:1095700002C010925A0780915A078A301CF089E085
:1095800080935A0710927D074E2D50E0475D5D4E47
:109590008E2D880F8E0D880F02E021E06D2F8E5BDF
:1095A0000E94055D90E6D91649F08EE6D81631F096
:1095B00080915C0190915D01892B29F18D2D0E9494
:1095C00045611092800721E030E002C0220F331F76
:1095D000EA94E2F740912D054227C9018873992743
:1095E000892B19F440932D0509C0842F822319F08B
:1095F000276C242301C0242B20932D0581E00E9499
:1096000098570E943758D85FD93308F017C186E0C1
:109610008B0DF816E0F421E0181320E08091150579
:1096200082FB882780F9C1E04AEC58E06D2F9C2F1F
:10963000981B892F0E944527C81B80911505C0FBE8
:1096400082F980931505D85FD93308F0F7C087E019
:109650008B0DF816E0F421E0181320E08091150539
:1096600087FB882780F9C1E04CEB58E06D2F9C2FD9
:10967000981B892F0E944527C81B80911505C0FBA8
:1096800087F980931505D85FD93308F0D7C088E0F3
:109690008B0DF816E0F421E0181320E080911805F6
:1096A00085FB882780F9C1E042EB58E06D2F9C2FA5
:1096B000981B892F0E944527C81B80911805C0FB65
:1096C00085F980931805D85FD93308F0B7C089E0D1
:1096D0008B0DF816B8F421E0181320E080911E05D8
:1096E00087FB882780F946EA58E06D2F0E944527BE
:1096F00090911E0580FB97F990931E05D85FD93392
:1097000008F09CC08AE08B0DF816E0F421E01813F5
:1097100020E08091180586FB882780F9C1E04EE99A
:1097200058E06D2F9C2F981B892F0E944527C81B3E
:1097300080911805C0FB86F980931805D85FD9334E
:1097400008F07CC08BE08B0DF816B8F421E01813FC
:1097500020E080911E0540E958E06D2F85FB8827A9
:1097600080F90E94452790911E0580FB95F9909302
:109770001E05D85FD93308F061C08CE08B0DF81658
:10978000A8F421E0181320E08091320546E858E063
:109790006D2F81700E9445279091320580FB90F9D2
:1097A00090933205D85FD93308F048C08DE0B80EE9
:1097B000FB1408F043C041E858E06D2F86E00E949A
:1097C000615DD83328F008E00D0F093378F036C01A
:1097D00004E2C0E02C2F46E751E16D2F802F0E945C
:1097E0000B5CCF5F085EC430A9F7EDCF1B110DC035
:1097F00080918007882359F063E0809116050E94CC
:10980000A6138093160522E003C020E001C021E0EA
:10981000409116054F5C602F82E10E94505CD4E2BB
:10982000C0E0CF5F20E04C2F602F8D2F0E94B3103F
:10983000D85EC430B1F702C0D0E1D4CBDF91CF9174
:109840001F910F91FF90EF90DF90CF90BF909F906E
:109850007F906F9008958F929F92AF92BF92CF9218
:10986000DF92EF92FF920F931F93CF93DF93C82F56
:1098700087EE9FE00E944F1F6CE0A62ECC24C3947D
:1098800075EEE72E7FE0F72E0CE02EE531E148E0A3
:109890006C2F88EE97E00E946E20C090E807CA9473
:1098A000F0905A0766E08C2D0E94E541A82E18E042
:1098B000DD24C7FCD0942A2D30E0C216D30639F43B
:1098C00080918007882329F052E0B52E04C0B12C86
:1098D00002C0BB24B394E901CC0FDD1FC20FD31F1C
:1098E000C55CDB4F62EE7FE0812F0E945B5D88E00C
:1098F0008A1510F448E301C041E34A0D612F8CE062
:109900000E94025DFF2011F000E001C00B2D2A81B2
:109910002F7047E75FE0612F83E10E94275D8A8116
:109920008F700E942210982E81E091102EC0F816A0
:1099300011F020E001C02B2D4881612F8DE30E94A2
:10994000B31088818532B4F09BED892E880E698131
:10995000882D0E94BD1D9C0182E0F81611F000E0E8
:1099600001C00B2D82E0E82E482D612F8AE60E946F
:10997000341E62C082E0F81611F020E001C02B2DE9
:109980004981552747FD509553C0981216C0F816C7
:1099900011F020E001C02B2D4881612F8DE30E9442
:1099A000051182E0F81611F020E001C02B2D49814D
:1099B000612F84E50E9405113FC082E0981217C014
:1099C00081E0F81611F020E001C02B2D4881612FB5
:1099D0008DE30E94B31082E0F81611F020E001C080
:1099E0002B2D4981612F87E50E94B31025C063E7C5
:1099F0007FE0812F0E945B5D81E0F81611F020E08E
:109A000001C02B2D4881552747FD50954F5F5F4F73
:109A1000612F8FE40E94525F82E0F81611F020E07F
:109A200001C02B2D4981552747FD50954F5F5F4F52
:109A3000612F8CE60E94525F4A8142954F704930F7
:109A40000CF04F5F83E0F81203C02B2D286001C09B
:109A500028E0612F89E60E9405118091800781111D
:109A600007C080915C0190915D01892B09F465C06C
:109A7000BB2009F462C081E0F81639F1F816A0F0B5
:109A800082E0F81609F43EC083E0F81256C08A81DD
:109A90006FE082958F700E949E138295807F9A81DD
:109AA0009F70982B9A8349C08A816EE08F700E94C4
:109AB0009E138F709A81907F982B9A830E94221018
:109AC0009816D9F11882198238C081E0981661F091
:109AD000981640F082E0981651F083E098122DC05D
:109AE00063E60BC06EE209C046E16AEE02C04EE2D8
:109AF00060E088810E949B1303C088810E949E13AE
:109B000088831BC081E0981669F0981640F082E0C7
:109B1000981671F083E0981210C063E60AC04DE712
:109B200063E802C046E16AEE89810E949B1304C08B
:109B30006EE289810E949E138983A394185F10347A
:109B400009F0B9CEDF91CF911F910F91FF90EF9067
:109B5000DF90CF90BF90AF909F908F900895AF927D
:109B6000BF92CF92DF92EF92FF920F931F93CF930A
:109B7000DF93B82E8BE59DE00E944F1FB3E1AB2E23
:109B8000CDE0CC2EDDE4ED2EDDE0FD2E0CE02EE56B
:109B900031E141E06B2D8EED97E00E946E20109137
:109BA000DE07D0905A0767E0812F0E94E541C82F59
:109BB0002091FF0430E02F5F3F4F442737FD409551
:109BC000542F02E0E02E01E160E08AE20E94425E52
:109BD000C1113BC068E47DE088E00E945B5D00E16C
:109BE0002AE045EE51E068E082E40E94055D113014
:109BF00009F0AEC329E040E467E08AE30E94645FB5
:109C00008D2D880F8D0D880F2091800746E068E02C
:109C1000845C0E94895D80918007882309F498C341
:109C2000CD2DD0E0CB51DE4F88810E94C72E61E45C
:109C30000E949E130E94D92E9881981709F488C318
:109C4000888382E00E94985783C3C23020F5C8E021
:109C500067E37DE08C2F0E945B5D123081F420E68B
:109C6000B21204C08091EF010E94E11361E3809180
:109C7000EF010E949E138093EF0121E001C020E0DC
:109C80004091EF0150E04C5F5E4F6C2F88E50E94E1
:109C9000525FC85F03C0C23091F4C8E063E272E172
:109CA0008C2F0E945B5D133009F0B1C381E0D812A4
:109CB00051C3809180078111ACC301E0ABC3C330B5
:109CC000D1F4C8E06FE27DE08C2F0E945B5D143020
:109CD00051F449E367EC8091F0010E949B1380935B
:109CE000F00141E001C040E021E06C2F8CE30E94D4
:109CF0003A11C85F03C0C430E1F4C8E066E27DE019
:109D00008C2F0E945B5D153051F445E16BEE809124
:109D100060040E949B138093600441E001C040E016
:109D200022E06C2F8CE30E943A11C85FC93320F007
:109D300073C3C53021F5C8E063E272E18C2F0E9445
:109D40005B5D163071F48091F10161E081700E94D9
:109D50009E139091F10180FB90F99093F10101E045
:109D600001C000E02091F101217040E15DE06C2F25
:109D70008CE30E94275DC85FC93320F04DC3C63015
:109D8000B9F4C8E021E0173009F020E08091F60135
:109D900049E05DE06C2F81700E9465279091F6018B
:109DA00080FB90F99093F601C85FC93320F034C36B
:109DB000C730C1F4C8E021E0183009F020E08091FC
:109DC000F60142E05DE06C2F829581700E9465276C
:109DD0009091F60180FB94F99093F601C85FC93326
:109DE00018F01AC3C830E9F469EF7CE08C2F0E94A8
:109DF0005B5D193049F464E08091F7010E949E1385
:109E00008093F70101E001C000E02091F70149EDE6
:109E10005CE06C2F8CE30E94275DC85FC93320F0A3
:109E2000FBC2C930D1F4C8E061ED7CE08C2F0E9408
:109E30005B5D21E01A3009F020E0022F4091F9012A
:109E40006C2F86E30E94BB278093F901A8E0EA2EDD
:109E5000EC0E88E38E1530F4DFC2CA3009F050C032
:109E6000F8E0EF2E68EC7CE08E2D0E945B5DECE369
:109E7000CE2EC0E0D0E0DC1202C01B3061F0209199
:109E8000FA0130E00C2E02C0359527950A94E2F7CE
:109E9000022F017001C002E0AE014054534F21E097
:109EA0006E2D8C2D0E94055D219626E0C20E86E661
:109EB000C812E1CF1B30F9F420E6B21631F0209140
:109EC0005C0130915D01232BB1F08B2D0E94456127
:109ED0001092800721E030E00D2C01C0220F0A947F
:109EE000EAF78091FA0182278093FA0182E00E94CA
:109EF00098570E943758C8E0CE0DC93328F08CC25D
:109F0000CB3009F0DAC0C8E06AEB7CE08C2F0E940D
:109F10005B5D1C3041F4D11006C08091800788231E
:109F200021F002E003C000E001C001E04091F40133
:109F300086E0489FA00111244556534F26E06C2F20
:109F400084E20E94055D8091F401882359F09DEF21
:109F5000980F9230F0F561E97CE08C2F0E945B5DF8
:109F6000D8E406C065E97CE08C2F0E945B5DDCE3F1
:109F70001C3049F421E0D21206C08091800788236A
:109F800021F002E003C000E001C001E02091F501F2
:109F90002E5F43E75CE06C2F8D2F0E94275D1C3005
:109FA00049F482E0D81206C080918007882321F00E
:109FB00022E003C020E001C021E04091F80182E3EB
:109FC0004802A0011124445D5E4F6C2F88E28D0F82
:109FD0001EC08130F1F46CE67CE08C2F0E945B5D4A
:109FE0001C3049F421E0D21206C0809180078823FA
:109FF00021F022E003C020E001C021E04091F50102
:10A00000552747FD50954F5F5F4F6C2F8EE70E949D
:10A01000525F1C3009F04DC080918007811107C04C
:10A0200020915C0130915D01232B09F442C0D09155
:10A03000F40180911E0585FF02C064E001C063E069
:10A0400081E0D81661F0D81620F022E0D216F1F0A7
:10A050002BC08D2F0E949E138093F40125C0DD2319
:10A0600021F08DEF8D0F823038F444E06EEF809157
:10A07000F5010E949B1307C0D130B1F46CE78091C9
:10A08000F5010E949E138093F5010EC0DD2321F09F
:10A090008DEF8D0F823040F44AE06CEF8091F80133
:10A0A0000E949B138093F8018091F4018D1310920C
:10A0B000F501C85FC93328F0AFC1CC3009F077C0D3
:10A0C000C8E08091F401882321F09DEF980F923031
:10A0D00010F56DE57CE08C2F0E945B5D1D3011F466
:10A0E00021E201C020E24091FE0185E04802A0018A
:10A0F00011244F515F4F6C2F8CE40E94525F1D3032
:10A1000009F051C044E16CEE8091FE010E949B1366
:10A110008093FE0148C08130B9F4D1E01D3009F0D0
:10A12000D0E02D2F47E45CE06C2F80E00E943B5D87
:10A13000DD23C9F120E8B21236C081E08093930C90
:10A1400080E00E94326C2FC06EE37CE08C2F0E9476
:10A150005B5D4091F50147FD04C043301CF042E0D7
:10A1600001C040E04093F5011D3031F4809180073B
:10A17000882321F002E003C000E001C001E089E093
:10A180004802A00111244E5D534F29E06C2F8CE34F
:10A190000E94055D1D3039F462E08091F5010E9456
:10A1A0009E138093F501C85FC93320F035C1CD30CF
:10A1B00051F5C8E065E17CE08C2F0E945B5D1E30AC
:10A1C00099F48091F60167E08295869587700E94E8
:10A1D0009E138295880F807E9091F6019F71982B37
:10A1E0009093F60121E001C020E04091F6014295F4
:10A1F000469547704F5C6C2F82E70E94505CC85FA9
:10A20000C93320F009C1CE3021F5C8E06BE07CE015
:10A210008C2F0E945B5D1F3071F48091FB0161E027
:10A2200081700E949E139091FB0180FB90F99093A6
:10A23000FB0101E001C000E02091FB01217043E03F
:10A240005CE06C2F8CE30E94275DC85FC93320F06F
:10A25000E3C0CF30C1F4C8E021E0103109F020E0C4
:10A260008091FB0149EF5BE06C2F869581700E9425
:10A2700065279091FB0180FB91F99093FB01C85FEA
:10A28000C93320F0C9C0C031C1F4C8E021E01131A8
:10A2900009F020E08091F10141EF5BE06C2F8695A1
:10A2A00081700E9465279091F10180FB91F9909354
:10A2B000F101C85FC93320F0AFC0C131D1F4C8E0AB
:10A2C00021E0123109F020E08091F10148EE5BE0DD
:10A2D0006C2F82FB882780F90E9465279091F101FD
:10A2E00080FB92F99093F10168E06C0F693328F0DC
:10A2F00093C0C23109F090C068E080917E0781115F
:10A3000003C021E0133109F020E044ED5BE080E080
:10A310000E943B5D133109F07FC020E8B2127CC07F
:10A320001092800789E180937E0780E80E94456152
:10A330001092290786E698E2DF91CF911F910F9145
:10A34000FF90EF90DF90CF90BF90AF900C94311BB7
:10A35000C0E17ECCD1105BC08091800700E08823F3
:10A3600011F022E001C021E04091F2015091F3018F
:10A370006C2F87E40E943E10133009F046C0809194
:10A380008007811106C020915C0130915D01232B73
:10A39000E1F16CE370E08091F2019091F3010E9491
:10A3A000EC72962FD82FDD2021F021E0D21691F00B
:10A3B0002CC06BE3892F0E949E132CE38202C00104
:10A3C00011248D0F911DD7FD9A959093F3018093E1
:10A3D000F2011BC04EE361E082E08D0F0E949B13EF
:10A3E000D81BDE5F2091F2013091F3012D1B310962
:10A3F000D7FD339537FD05C03093F3012093F2016B
:10A4000004C01092F3011092F201C85F5BCC00E02F
:10A4100001C002E020E0A8CFDF91CF911F910F9102
:10A42000FF90EF90DF90CF90BF90AF900895AF92E4
:10A43000CF92EF92FF920F93CF93DF93C82F8AE9C9
:10A440009BE00E944F1F86E0A82EC12C99E9E92EBF
:10A450009BE0F92E0CE02EE531E142E06C2F8BED14
:10A4600097E00E946E20C091DB0767E08C2F0E946E
:10A47000E541D091FB01D295D695D7706EE87BE08F
:10A4800088E00E945B5DC13089F464E08D2F0E94FA
:10A490009E13D82F982F9295990F907E8091FB0153
:10A4A0008F71892B8093FB0101E001C000E02D2F0B
:10A4B0004EE65BE068E084E50E94275D63E67BE0B2
:10A4C00080E10E945B5DC23049F464E28091FC014E
:10A4D0000E949E138093FC0121E001C020E0409186
:10A4E000FC0160E184E50E94B31068E57BE088E14F
:10A4F0000E945B5DC33049F464E68091FD010E94D7
:10A500009E138093FD0121E401C020E44091FD01F0
:10A5100050E068E184E50E94525F21E0C43009F018
:10A5200020E08091FB014AE45BE060E282FB882747
:10A5300080F90E9485279091FB0180FB92F990930E
:10A54000FB0121E0C53009F020E08091FB014CE3E4
:10A550005BE068E283FB882780F90E948527909161
:10A56000FB0180FB93F99093FB0121E0C63009F0D9
:10A5700020E08091FB014EE25BE060E38295817018
:10A580000E9485279091FB0180FB94F99093FB0139
:10A59000DF91CF910F91FF90EF90CF90AF90089502
:10A5A0005F926F927F928F929F92AF92BF92CF9263
:10A5B000DF92EF92FF920F931F93CF93DF93D82EEA
:10A5C0008FE091E10E944F1FB1E1AB2ECC24C394E8
:10A5D000CDE0EC2EC1E1FC2E0CE02EE531E146E0B1
:10A5E0006D2D8CEE97E00E946E20C090EC07CA940F
:10A5F000B0905A0766E08C2D0E94E541982E80E8C5
:10A60000D81227C09FE09C1520F14C2D552747FDFF
:10A610005095FA01E919F109EE0FFF1FE55AF84FBD
:10A6200020813181B11015C085E0849FF001859FA4
:10A63000F00D1124E15CFC4F8281882319F03195E3
:10A64000219531093483238382E00E9498570E9428
:10A650003758E8E0AE2EEC2CFF24E7FCF09480E1C4
:10A66000981609F4BEC0892D0E943710EC01092DFF
:10A6700010E0F801EE0FFF1FE55AF84F20813181FD
:10A680008A81EB81FC81882319F0F195E195F1092C
:10A690002E1B3F0B233331051CF081110AC09EC0D5
:10A6A0002E3C3F4F1CF4882321F098C06DE2862E8B
:10A6B00002C05FE7852E939420E0492D6A2D80E04B
:10A6C0000E94E310482D6A2D8BE40E94025D809168
:10A6D000FB0181FF03C04DE7642E02C034E6632E08
:10A6E000812C562C5194E016F10641F4B81006C0A6
:10A6F00080918007811105C021E004C020E0712C09
:10A7000009C022E080917F078823C9F377247394DE
:10A710001092710182E0881691F193E0891609F494
:10A7200043C081E08816B1F020624B815C816A2DC4
:10A7300080E30E94525F772009F446C022E048EE91
:10A7400053E068E17CEF8B819C810E94DC129C834A
:10A750008B833AC048814456552747FD50956A2D52
:10A7600088E40E94525F772079F18881845688833B
:10A7700049E1652D0E949B138C59888325C049812E
:10A780004C59552747FD50956A2D86E60E94525F29
:10A790007720D1F089818C598983462D67EE0E94FC
:10A7A0009B138456898310C04A816A2D8CE60E94CF
:10A7B0006220772049F061E08A810E949E1391E037
:10A7C000811101C090E09A83839494E089128BCF29
:10A7D00088E08A0D803491F1A82E41CF2EE7822E99
:10A7E0006ACFC1E090E1C912C0E080917E0781117B
:10A7F00023C02C2F4CEF50E16A2D82E10E943B5D7B
:10A80000CC23E1F080E8D81219C089E180937E075B
:10A8100080E80E944561DF91CF911F910F91FF90D9
:10A82000EF90DF90CF90BF90AF909F908F907F90F0
:10A830006F905F900C94ED3E20E0DCCFDF91CF91E4
:10A840001F910F91FF90EF90DF90CF90BF90AF904E
:10A850009F908F907F906F905F9008956F927F92FE
:10A860008F929F92AF92BF92CF92DF92EF92FF9220
:10A870000F931F93CF93DF93C82F80E590E10E9441
:10A880004F1F41E1A42E52E0C52E6DE4E62E60E19B
:10A89000F62E0CE02EE531E149E06C2F89EE97E0D1
:10A8A0000E946E20A090E907AA9490905A0766E053
:10A8B0008A2D0E94E541B82E18E0CA2CDD24C7FC81
:10A8C000D094B11020C06DE370E1812F0E945B5DD8
:10A8D000A1100FC080918007882311F0C2E001C051
:10A8E000C1E060E1809161040E949E138093610445
:10A8F00001C0C0E04091610450E02C2F612F8CE634
:10A900000E94525F59C180E18B1508F455C100E1E6
:10A9100080916104081BEB2CF12CE701CC0FDD1FAB
:10A92000C05ADB4F20E04B2D612F80E00E94E310E6
:10A930000B1508F4C3C0812CCE14DF0441F4981029
:10A9400006C080918007811105C001E004C000E0CD
:10A95000712C07C002E080917F078823C9F3772418
:10A9600073948881811021C0807C803421F08038EC
:10A9700021F446E503C041E401C043E5202F612FE7
:10A980008EE10E94505C772009F493C0888162E0D8
:10A9900082958695869583700E949E138295880F76
:10A9A000880F807C98819F7330C091E0891230C0FD
:10A9B000982F907C903819F026E1622E02C099E120
:10A9C000692E482F440F440F4595459547314CF06B
:10A9D00029EE240F46E250E1612F8AE20E94275DB2
:10A9E00005C0202F612F8AE20E940511772009F40B
:10A9F00060C08881880F880F462D6AEE8595859501
:10AA00000E949B138F739881907C982B988351C0E0
:10AA1000982F907C4981903491F447FD03C04F30CA
:10AA200024F401C040E0242F01C02FE0298341EC31
:10AA300051E1612F80E60E94275D4FE017C09038FA
:10AA400041F5880F880F89359CF047FD04C04930D7
:10AA50001CF049E001C040E0498321E0240F4FE7AA
:10AA600052E1612F80E60E94275D49E060E01BC053
:10AA70004F360CF04FE64983552747FD5095405817
:10AA80005F4F202F612F80E60E94525F4FE660E803
:10AA90000AC0552747FD5095202F612F80E60E9460
:10AAA000525F4DE763E8772021F089810E949B1374
:10AAB0008983839483E088123FCF7EC063E270E194
:10AAC000812F0E945B5D812CCE14DF0441F498102D
:10AAD00006C080918007811105C001E004C000E03C
:10AAE000712C07C002E080917F078823C9F3772487
:10AAF00073948881811013C0482F4F71202F612FCC
:10AB00008EE10E940511772009F452C0888165E129
:10AB10008F710E949E138F719881907E1BC091E06F
:10AB200089121BC0282F22952695277047EF5FE0DA
:10AB3000612F8CE30E94275D7720D1F1888166E048
:10AB40008295869587700E949E138295880F807EDD
:10AB500098819F71982B98832BC0829586958770DA
:10AB600090E04981069774F0493008F049E0498344
:10AB700021E0240F4FE752E1612F80E60E94275D1C
:10AB800049E00BC04A3F08F04AEF498350E0202FCC
:10AB9000612F86E60E94525F4AEF772049F050E02D
:10ABA000898122E060E070E090E00E94DC128983FD
:10ABB000839483E0881288CFB394185F103409F02F
:10ABC00080CEDF91CF911F910F91FF90EF90DF909A
:10ABD000CF90BF90AF909F908F907F906F9008958F
:10ABE0001F93CF93DF93EC011AE088810E94C72E58
:10ABF0000E94D92E89931150C1F7DF91CF911F91F7
:10AC00000895E3EDF4E080E090E021913191820F2E
:10AC1000931F24E0EB3EF207C1F7089581E6E2EDD1
:10AC2000F4E0DF011D928A95E9F78AE08093D2046F
:10AC300089E1809300058AE58093010581E0809396
:10AC40001605E3EDF4E020E032E080E891E02193A6
:10AC5000319395878487938F828FB4E0E13EFB0721
:10AC6000B1F74AE050E068EF72E183E295E00E94BC
:10AC700047730E9401569093FE048093FD0408954B
:10AC8000CF93C82F2DEE32E0E5EEF1E0DF01C901F0
:10AC90001D920197E9F74AE050E06DEE72E1CF01B5
:10ACA0000E9447738C2F90E06AE070E001960E944A
:10ACB000EC72605D6093EA01805D8093EB0180E05F
:10ACC000CF910C9469620F931F93CF93DF93EB01A5
:10ACD000042F803138F561E0680F8BE098E00E9426
:10ACE000B15910E0A80160E270E0CE010E946873E3
:10ACF0004AE050E0BE018BE098E00E94355A0A9786
:10AD000089F48BE098E00E94A359C00FD11F0097EF
:10AD100049F06AE070E00E94EC72805D8A93862FB1
:10AD2000972FF5CFDF91CF911F910F9108958F5FEE
:10AD30000C945859CF93C82F803188F561E0680F83
:10AD40008BE098E00E94B1592DEE32E0E5EEF1E0A3
:10AD5000DF01C9011D920197E9F74DEE52E0BF01F5
:10AD60008BE098E00E94355A8F3F910509F018F466
:10AD70008C2F0E94405685EE91E00E94F055809104
:10AD80008D04811107C08091F601869583708E5FD6
:10AD900080938D040E94C933CF910C94C413CF913A
:10ADA0000895FF920F931F93CF93DF93CDB7DEB734
:10ADB0002F970FB6F894DEBF0FBECDBF01E0080F8E
:10ADC000102F1031C8F4FF24F394F10E8F2D0E9440
:10ADD000585981110FC0602F8BE098E00E94B15943
:10ADE00061E0610F28E532E042E082E098E00E94F5
:10ADF0001D5B06C01F2DE5CF103169F780E01AC03A
:10AE00004FE050E0BE016F5F7F4F8BE098E00E9403
:10AE1000CE59882351F0482FBE016F5F7F4F82E0EB
:10AE200098E00E949A5AA895EBCF82E098E00E94A1
:10AE3000485B81E02F960FB6F894DEBF0FBECDBF02
:10AE4000DF91CF911F910F91FF900895EF920F9393
:10AE50001F93CF93DF930E944559882381F10E946D
:10AE6000BB5887FD2CC060E08BE098E00E94B15990
:10AE700081E6E2EDF4E0DF011D928A95E9F741E613
:10AE800050E0BF018BE098E00E94355A83E295E0E4
:10AE90000E94F0558091D2048A3028F480918E016E
:10AEA000816080938E018AE08093D204C091FD047A
:10AEB000D091FE040E940156C817D90781F161E0C4
:10AEC0008DED92E10E94CC1A8BEC92E10E944B1224
:10AED0000E9420590E940E5688ECE82E01E610E0F0
:10AEE00022ED34E041E060E08BE098E00E94795B85
:10AEF0008136910529F060E08CEB92E10E94CC1A3A
:10AF000080E00E94405698ECE92E0DEE12E025EE0E
:10AF100031E042E061E08BE098E00E94795B809153
:10AF2000FF04DF91CF911F910F91EF900C949A56EF
:10AF3000882379F090911608982B90931608F8942E
:10AF400080915A0C90915B0C7894909315088093A3
:10AF500014080895EF920F931F93CF934091160812
:10AF6000442309F47FC0811110C0F89480915A0CD9
:10AF700090915B0C78942091140830911508821BF5
:10AF8000930B8436910508F46DC08091F807811108
:10AF900069C0C42FC47042FD02C081E001C083E0DB
:10AFA0008093F8071092160840FF26C034E1E32E84
:10AFB00001E610E022ED34E041E061E189EF97E045
:10AFC0000E94795B8136910519F461E180E029C026
:10AFD0008091FF07823051F48091160881602BC068
:10AFE0008091FF07823001F1C1113AC060E083E037
:10AFF00093E10E94CC1A34C041FF32C024E1E22E1A
:10B000000DEE12E025EE31E042E061E189EF97E0DC
:10B010000E94795B8D3E924019F78091FF0461E1B7
:10B020008F5F0E9466591CC080911608C11102C032
:10B03000826001C0866080931608F89480915A0C53
:10B0400090915B0C789484569109909315088093A5
:10B0500014088091950C833019F4A8951092950CE2
:10B060001092F807CF911F910F91EF900895809162
:10B070001608882359F081E00E94AA578091950C08
:10B080008330A9F7A8951092950CF1CF089540E46C
:10B0900050E060E070E087E198E00C94506041E09F
:10B0A00050E062E070E089E198E00C945060CF934A
:10B0B000DF931F92CDB7DEB7698390E1899FB0011E
:10B0C000112441E050E0CE0101960E9450600F90A3
:10B0D000DF91CF910895CF93DF931F92CDB7DEB765
:10B0E00090E1899FB001112441E050E0CE0101962A
:10B0F0000E946F7389810F90DF91CF910895CF9354
:10B10000DF93D82FC82F8C2F0E946B58882329F0EB
:10B110008C2F0E946B58C82FF6CF609119088C2F86
:10B120000E945758D0931908DF91CF910C944F5833
:10B13000CF93C0911908CC2359F08C2F0E946B58E3
:10B14000809319080E944F5860E08C2F0E94575836
:10B150008C2FCF910895CF93DF9380911908C0E091
:10B16000D0E0882321F02F960E946B58FACFCE01B1
:10B17000DF91CF910895DF92EF92FF920F931F938B
:10B18000CF93DF9380E8E5EEF1E0DF011D928A9531
:10B19000E9F7CBE1D8E0F12CB4E1FB1205C08091D6
:10B1A000190809E118E002C08E01888190E0E12CC5
:10B1B000DD24D394DF0C009701F19C012450310968
:10B1C0002C37310530F4FC01EB51FE4F2081222356
:10B1D00071F0EE2029F060E08E2D0E94575804C0D7
:10B1E000F80110820E94475880E090E0E4CFD082BE
:10B1F000E82E0E946B5890E0DECFF3942396F5E1A1
:10B20000FF12CACFC4E0D0E0FE01EB51FE4F8081B7
:10B21000811109C0609119088C2F0E945758C09362
:10B2200019080E944F582196C038D10569F780E06F
:10B23000DF91CF911F910F91FF90EF90DF900895D4
:10B24000CF9380E4E7E1F8E0DF01982F1D929A9513
:10B25000E9F794E0909317088093180880E18093B1
:10B260001A0884E0C1E0C80F6C2F0E945758CF37EE
:10B2700011F08C2FF7CF60E08FE70E94575884E0E1
:10B2800080931908CF910C94475840E450E060E057
:10B2900070E087E198E00E946F7380911708843016
:10B2A00029F481E090911808903409F080E0089525
:10B2B00090E0FC01EE0FFF1FE80FF91FE95EF74F6A
:10B2C00081E09481911101C080E00895CF93DF93D4
:10B2D00090E0EC01CC0FDD1FC80FD91FC95ED74F1E
:10B2E0008C819D81AE8170E0FB01EE0FFF1FE60FA8
:10B2F000F71FE95EF74F2481358146812C833D831A
:10B300004E8384839583A683DF91CF910C94475815
:10B31000CF9390E09C01220F331F280F391FF901B2
:10B32000E95EF74FC481F901E55EF74F10821182A3
:10B3300012820E944758CC2321F08C2FCF910C947D
:10B340007F58CF910895FC01808190E0FC01EE0FC1
:10B35000FF1FE80FF91FE45EF74F918180819F7016
:10B360000895CF93DF93FC0160831282118270E015
:10B37000CB01880F991F860F971FEC01C95ED74F2D
:10B380002C812383148215821682FC01E35EF74F21
:10B39000808182958F70DF91CF910895AF92BF9297
:10B3A000CF92DF92EF92FF920F931F93CF93DF9391
:10B3B0001F92CDB7DEB78C01FC01808190E0FC01CB
:10B3C000EE0FFF1FE80FF91FE45EF74F8081218128
:10B3D000922F9F70F80121813281821B930B7A0199
:10B3E0008417950708F47C015B016701C114D1043F
:10B3F00029F1F8018381882309F164816F5F6483F7
:10B4000070E0F0E18F9F600D711D112441E050E06C
:10B41000CE0101960E946F738981F50181935F01CE
:10B42000F80184818F3030F0148283810E946B5840
:10B43000F8018383F1E0CF1AD108D8CFF8018181D8
:10B4400092818E0D9F1D8C199D09928381838E2D73
:10B450008C190F90DF91CF911F910F91FF90EF907A
:10B46000DF90CF90BF90AF9008957F928F929F9280
:10B47000AF92BF92CF92DF92EF92FF920F931F9302
:10B48000CF93DF934C016B018A01C0E0D0E05C01F7
:10B4900025E0A20EB11CC017D107E8F5F4018581A3
:10B4A0008F7781F0F4014581F42FFF777F2E2F2FC6
:10B4B00030E0C8018C1B9D0B8217930760F4702E3F
:10B4C0007C1A09C041E050E0B501C4010E94CE5988
:10B4D000813041F320C0E72CF12CC6018C0F9D1F59
:10B4E00047FF06C0A70160E070E00E9468730CC0CF
:10B4F000A701BC01C4010E94CE59871529F0FE01A5
:10B50000E80FF11DCF0108C0CE0DDF1DF4018581CC
:10B5100087198583C0CFCE01DF91CF911F910F9105
:10B52000FF90EF90DF90CF90BF90AF909F908F9063
:10B530007F900895AF92BF92CF92DF92EF92FF92E9
:10B540000F931F93CF93DF93EC018B01D42E8B814C
:10B55000811111C089819A81892B69F4E880F12CCD
:10B560000E9498588B83F701EE0FFF1FEE0DFF1D11
:10B57000E95EF74F8483CD2C8FE0A82ECC2009F410
:10B5800045C02F813885F89480915A0C90915B0CBE
:10B590007894281B390B37FF02C082E004C08B81EE
:10B5A000811103C081E08E8331C09C819F3078F08F
:10B5B0001C820E946B58811106C00E949858682F07
:10B5C0008B810E9457588B810E946B588B838B8193
:10B5D000882341F36C819A2D961BBC2C9C1508F492
:10B5E000B92EEB2CF12C70E090E1899F600D711D5C
:10B5F00011246F5F7F4FA701C8010E9450600E0D9C
:10B600001F1D8C818B0D8C83CB18B8CF6D2D70E0F6
:10B610006C19710929813A81260F371F3A832983D2
:10B620008D2D8C19DF91CF911F910F91FF90EF908D
:10B63000DF90CF90BF90AF900895EF92FF920F935D
:10B640001F93CF93DF93EC01F62EE42E89010E9425
:10B65000B1596F2D70E0FB01EE0FFF1FE60FF71FD2
:10B66000E45EF74F1082E29430EFE322E182F89437
:10B6700040915A0C50915B0C7894400F511F5887A1
:10B680004F83DF91CF911F910F91FF90EF9008951D
:10B690001F93CF93DF93EC01888190E0FC01EE0FC4
:10B6A000FF1FE80FF91FE45EF74F898180839A81BD
:10B6B0009F708181807F892B81838B81882329F0F2
:10B6C0000E946B58182F81110BC010E00E94475840
:10B6D000112359F0812FDF91CF911F910C947F5846
:10B6E00060E08B810E945758F1CFDF91CF911F917D
:10B6F00008957F928F929F92AF92BF92CF92DF92E6
:10B70000EF92FF920F931F93CF93DF931F92CDB7CA
:10B71000DEB76C0159012E2D30E00E941D5B1982AD
:10B720004501E12CF12C77247394F40181914F01B0
:10B730009981811108C071104EC08081811105C0AE
:10B74000772473941CC071100AC080E09F3718F4EE
:10B75000E016F10679F5772089F0782E01C0712C7A
:10B76000992341F19068998341E0BE016F5F7F4F5B
:10B77000C6010E949A5A8130E1F027C0782E9923A1
:10B78000C9F041E0BE016F5F7F4FC6010E949A5A27
:10B790008130D9F44981B701641B71096A0D7B1DA1
:10B7A000C6010E949A5A9981891719F0981B9983AA
:10B7B0000CC0198289818F5F8983FFEFEF1AFF0A1E
:10B7C0000E151F0508F0B1CF08C089818F7787015A
:10B7D000081B110902C0872DB9CFC6010E94485B22
:10B7E000C8010F90DF91CF911F910F91FF90EF90C3
:10B7F000DF90CF90BF90AF909F908F907F900895F3
:10B8000080E094E0E8E5F8E0DF019C011D92215022
:10B810003040E1F70895FF920F931F93CF93DF938A
:10B82000FA0174913196A491B0E0179693E0B59522
:10B83000A7959A95E1F71A2FDA011396FA01329635
:10B840004491249FA00DB11D1124669566956695BF
:10B8500090E0F0E86F9F800D911D112420E030E012
:10B8600060E0885A974F472F50E0611798F40A2FED
:10B87000EC01C20FD31FFD01FE2EF01AF71620F4C3
:10B88000F490F9923196F8CFA40FB51F6F5F20584E
:10B890003F4FEBCFDF91CF911F910F91FF90089514
:10B8A000FF920F931F93CF93DF9346312CF4842F95
:10B8B000880F840F880FA0C076E0780FA42FBB27D5
:10B8C000A7FDB09520FD08C021FD02C090E005C095
:10B8D0009091590C96FFFACF91E066956695669522
:10B8E000C82FD0E030E8639FC00DD11D1124C85A85
:10B8F000D74FFE0122FF53C04E3211F07CE0780F8B
:10B900008AE04802F0011124E054F1409D012052E8
:10B91000310937FF03C09D0121513109A90124E0FC
:10B92000559547952A95E1F780EA849F9001859F78
:10B93000300D11242E0F3F1F2A5E3C4E85E08823D8
:10B9400081F0F9010491E056FF4F6491A9014F5F26
:10B950005F4FFA011491F901EF55FF4FF4909A01EE
:10B9600004C010E060E000E0F12C2F5F3F4F99230E
:10B9700021F0009510956095F094DE01AF57BF4F10
:10B98000FCE0A835BF0740F408831983FE01E058A6
:10B99000FF4F6083FC922296815088F62CC023FFD3
:10B9A00008C02196292F2195208375E0780F51E05A
:10B9B00001C050E025E04202F0011124E750F64EAC
:10B9C00085E04491552311F0843059F03CE0C835AE
:10B9D000D30738F49E012F5F3F4F91114095488364
:10B9E000E901815031968111ECCF4CE0C835D40784
:10B9F00010F491959883872FDF91CF911F910F912C
:10BA0000FF90089520E00C94505CEF92FF920F930A
:10BA10001F93CF93DF93F62E122F902F9071E92E64
:10BA2000EA01112369F0EE2011F0488102C0FE0105
:10BA30004491202F6F2D0E94505C11502196F1CF20
:10BA4000DF91CF911F910F91FF90EF9008950F9389
:10BA5000FA0194914F5F5F4F929F400D511D112449
:10BA6000292F0E94055D0F9108950F9300E00E9419
:10BA7000055D0F910895FF920F931F93CF93DF936E
:10BA8000062F122F922F9071F92EFA01FF2011F03C
:10BA9000408101C04491EF012196442331F0212FD0
:10BAA000602F0E94505CFE01F1CFDF91CF911F917A
:10BAB0000F91FF900895AB0120E0682F80E00C9477
:10BAC0003B5D20E00C943B5DFF920F931F93CF935F
:10BAD000DF93082FF62EEA0114E1180F15504C2FB2
:10BAE0004F704A301CF0495C28E002C0405D20E005
:10BAF0006F2D812F0E94505C34E0D695C7953A9502
:10BB0000E1F71013EBCFDF91CF911F910F91FF90D1
:10BB10000895222321F09091590C96FD0895480F25
:10BB2000669566956695E82FF0E090E8699FE00DD0
:10BB3000F11D1124E85AF74F8E1B982F9E0F941772
:10BB400020F4908190959193F8CF0895962F969533
:10BB500096959695E82FF0E080E8989FE00DF11D0E
:10BB60001124E85AF74F8CE0E835F80758F467706D
:10BB700081E090E0062E01C0880F0A94EAF79081D8
:10BB800098279083089547FF02C0840F4195962F10
:10BB9000969596959695E82FF0E080E8989FE00DB1
:10BBA000F11D1124E85AF74F677031E001C0330FDF
:10BBB0006A95EAF74423B1F08CE0E835F80790F491
:10BBC000822F90E020FF08C02081232720839595B5
:10BBD0008795282F206803C095958795282F415079
:10BBE0003196E8CF08952FEF0C94C35D962F96956C
:10BBF00096959695282F30E0F90180E8989FE00D02
:10BC0000F11D1124E85AF74F962F940F96959695AB
:10BC1000969580E8989F200D311D1124285A374FA2
:10BC2000862F8770A1E0B0E001C0AA0F8A95EAF7DD
:10BC3000A1958081A827A083E217F30750F4E0586C
:10BC4000FF4F8CE0E835F807E0F490819095908301
:10BC5000F3CF8CE0E835F807A0F4842F992787FD0F
:10BC60009095860F911D68E070E00E94EC7221E0D3
:10BC700030E001C0220F8A95EAF721958081822762
:10BC8000808308953F924F925F926F927F928F923E
:10BC90009F92AF92BF92CF92DF92EF92FF920F935B
:10BCA0001F93CF93DF93182FB62E802F05FF04C06C
:10BCB00004FF04C002E003C000E001C001E0982FCF
:10BCC0009F77C92EE7FE04C0E1946624639401C007
:10BCD000612C57FF0AC050954095309521953F4FF4
:10BCE0004F4F5F4F7724739401C0712C82FF06C0C1
:10BCF0009CE09093580CCAE0DC2E05C096E090932F
:10BD0000580CB5E0DB2E86FF28C071101D0D283EB3
:10BD100083E038074105510514F01D0D05C0243698
:10BD200031054105510514F01D0D05C02A303105BE
:10BD3000410551050CF01D0D002381F0023031F456
:10BD400024363105410551054CF41D0D2A303105CD
:10BD5000410551051CF41D0D01C01D198091580CA1
:10BD6000810F8093580C023011F490EFC90E882493
:10BD70008394F2E09F2EA12CFF24E7FCF094A6E030
:10BD80005A2E5B0CE82DF0E0EE16FF060CF460C0B6
:10BD90006AE070E0C9010E94EC72382EEB01E0E32A
:10BDA0004E2E480E2C2D442D6B2D812F0E94505C61
:10BDB000081131C0C2FE1AC08FEF830D833008F422
:10BDC0009394CE016AE070E00E94EC72823011F030
:10BDD0008430E9F484E3481204C0AA24A394A10E99
:10BDE00017C0AA24AA94A10E939412C07EEF472EE6
:10BDF000410E8FEF810FC0FE05C047E06B2D0E9402
:10BE0000F65D03C0652D0E94A65D142D01C0A12E14
:10BE1000209709F000E09E01442737FD4095542FFC
:10BE2000211531054105510581F4002331F002301F
:10BE300059F491E0981540F008C0C4FE09C06110A3
:10BE400004C080EFC80E01C000E01D1983949ACF92
:10BE5000AA2061F0492D6CE06B0D8A2D0E94F35DE4
:10BE6000492D6DE06B0D8A2D0E94F35D772039F02E
:10BE70002C2D4DE26B2D812F8D190E94505C80E09E
:10BE8000DF91CF911F910F91FF90EF90DF90CF90B6
:10BE9000BF90AF909F908F907F906F905F904F90EA
:10BEA0003F900895EF920F93022F9A01442737FD98
:10BEB0004095542F95E0E92E0E94425E0F91EF903D
:10BEC000089520E00C94525F0F931F93CF93DF935C
:10BED000182FC62F042FD22F422F0E94F65D02305A
:10BEE00038F04D2F6C2F8FEF800F810F0E94F65D81
:10BEF00002501F5F6FEF6C0F6D0F402F812F0E945C
:10BF0000F35D402F6C2F812FDF91CF911F910F9107
:10BF10000C94F35D0F931F93CF93DF93182FC62FCD
:10BF2000D22FE42FF0E03297053608F004E60E9F9A
:10BF3000C0010F9F900D112464E670E00E94EC7226
:10BF4000062F2D2F6C2F812F0E94645F002369F034
:10BF5000D150DC0FCF5F1F5FCD1738F4402F6C2F0F
:10BF6000812F0E94F35DCF5FF7CFDF91CF911F91BB
:10BF70000F910895A998AB98AC988BBBAD9AAD98EA
:10BF8000AB9AA99A089581E080935708AA9825E072
:10BF90002A95F1F7000085E08A95F1F70000AA9A4A
:10BFA0008CED95E025E02A95F1F7000001970097C8
:10BFB000C9F782EE0E94BA5F8EEA0E94BA5F81EAF8
:10BFC0000E94BA5F86EA0E94BA5F84EA0E94BA5F62
:10BFD00082EA0E94BA5F80EC0E94BA5F8FE20E9400
:10BFE000BA5F85E20E94BA5F81E80E94BA5F82E28E
:10BFF0000E94BA5F8FEA0E94BA5F82E280930005D6
:10C00000109257080895CF93C82F81E08093570866
:10C0100081E80E94BA5F8C2F0E94BA5F1092570885
:10C02000CF910895809100050C9403601F93CF93E6
:10C03000DF9381E08093570810E0C8E5D8E084E002
:10C040000E94BA5F80E10E94BA5F812F806B0E94DC
:10C05000BA5FA998AB9AAC98FE01CE0180589F4F69
:10C0600020812BBBAD9AAD9821812BBBAD9AAD98A9
:10C0700022812BBBAD9AAD9823812BBBAD9AAD9895
:10C080003496E817F90761F7EF01AB9AA99A1F5F99
:10C090001830A9F610925708DF91CF911F9108959B
:10C0A000BF92CF92DF92EF92FF920F931F93CF93A5
:10C0B000DF937B018A01080F191FEC01E81AF90AC6
:10C0C0006701CC0EDD1EC017D107C1F0B990809179
:10C0D000F8078270E19B05C08823E1F30E946F1B83
:10C0E000F6CFDFBACEBAE09A8DB3B81649F3BDBA2F
:10C0F0008FB7F894E29AE19A8FBFE2CFDF91CF91A8
:10C100001F910F91FF90EF90DF90CF90BF90089517
:10C110008091890C1092890C0895FC0180818F70A8
:10C12000880F611181608F709081907F982B908330
:10C1300081818F5F81838281882351F09F7041F4D8
:10C14000833621F0842F80628093890C11821282C1
:10C150008281883069F148F4813091F188F0823031
:10C1600039F1843009F03FC023C08F35C1F018F495
:10C170008031F1F00895813649F0823671F10895E9
:10C1800080818F708F3079F581E62BC040664093B7
:10C19000890C10926A06109269068FE522C081818F
:10C1A000803211F4406816C08832E9F480E119C089
:10C1B0009181903328F090E0959587958283118244
:10C1C000828190E00197218130E082239323892BA3
:10C1D00051F440644093890C08958181803418F0B3
:10C1E00088E0828311820895282F30E02F303105B6
:10C1F0006CF4F901EE0FFF1FE20FF31FE45AF34F47
:10C2000090819F7081E09F3071F52EC090E0FC011D
:10C210003F97E930F10538F5E659FF4F0C9441732B
:10C2200091B194701DC093B390781AC0909163003F
:10C23000917016C0909163009095987011C0809194
:10C24000630083FF10C091B102C091B190959074CA
:10C2500007C091B1907104C093B3F9CF91B19072BE
:10C2600081E0911101C080E008958F7090E08F30DF
:10C27000910551F0FC01EE0FFF1FE80FF91FE45A82
:10C28000F34F82E68283118208958F7090E08F30A1
:10C29000910549F0FC01EE0FFF1FE80FF91FE45A6A
:10C2A000F34F83E682830895EF92FF920F931F93DB
:10C2B000CF93DF9380915A0C90915B0C01969093F1
:10C2C0005B0C80935A0C8093590C16B31095CCE5F7
:10C2D000DCE0F12C11FB662760F94F2DCE010E94A6
:10C2E0008D60F3941695239686E0F812F3CFE0B2B2
:10C2F000E094C9E7DCE100E010E0FC1AFE01849163
:10C300004C2F4F0D8E2161E009F460E0C801825985
:10C31000934F0E948D6021960D5F1F4F08311105CC
:10C3200069F79091CC0161E0C92FC07295FF60E080
:10C330004EE086E89CE00E948D6086B390E0809598
:10C3400090958E7799278C2B19F089E08093700156
:10C35000DF91CF911F910F91FF90EF900895EF9291
:10C36000FF920F931F93CF93DF93F82E80E04AE064
:10C37000282F30E0429FF001439FF00D1124EB5134
:10C38000FE4F928DF91650F5803261F18AE0E82E69
:10C39000E29E8001E39E100D1124E801C150DE4FA2
:10C3A0006FE170E0621B730BE69EA001E79E500DEB
:10C3B00011242F5F3F4FE29EC001E39E900D112498
:10C3C000BE0181509E4F0E945673FE011192EA9465
:10C3D000E9F7F801EB51FE4FF28E06C09923A1F266
:10C3E0008F5FC6CFCFEFD1E0CE01DF91CF911F910C
:10C3F0000F91FF90EF90089580E491E0EFEFF1E06E
:10C40000DF019C011D9221503040E1F7089588E240
:10C41000EBECF3E0DF011D928A95E9F788E4E3EFA6
:10C42000F3E0DF011D928A95E9F70895FB0188305A
:10C43000A8F029E0829FC00111248B519E4F20E07B
:10C4400030E04191DC01A20FB31FAA53BE4F4C93C1
:10C450002F5F3F4F29303105A1F7089525E0829FD6
:10C46000C00111248B519E4F20E030E04191DC014E
:10C47000A20FB31FAA51BE4F4C932F5F3F4F2530E1
:10C480003105A1F7089590E00197FC01EE0FFF1F21
:10C49000E80FF91FDF01A35CBB4F6F708C91807FA9
:10C4A000862B8C93EB51FE4FDF01AA5ABD4F4C9364
:10C4B000E95AFD4F2083089590911605E82FF0E08A
:10C4C00084E0989FE00DF11D1124E059FC4F849108
:10C4D00008958F929F92AF92BF92CF92DF92EF9288
:10C4E000FF920F931F93CF93DF93CDB7DEB76D9776
:10C4F0000FB6F894DEBF0FBECDBFF82E85E0E8E2A0
:10C50000F1E0DE01559601900D928A95E1F785E004
:10C51000EDE2F1E0DE01509601900D928A95E1F78F
:10C5200085E0E2E3F1E0DE011B9601900D928A9531
:10C53000E1F785E0E7E3F1E0DE01169601900D9268
:10C540008A95E1F785E0ECE3F1E0DE0111960190D8
:10C550000D928A95E1F71A8E1B8E1C8E1D8EE0912E
:10C560001B05F0E0E757FC4F46E050E0A1E0E49106
:10C570000E2F10E021E030E0C801042E02C0959596
:10C5800087950A94E2F783709927BC016F5F7F4F0C
:10C59000EAE1F0E0EC0FFD1F8E0F9F1F621773079B
:10C5A00011F4FC01A0832F5F3F4F25303105B1F717
:10C5B000AF5F42505109A530E9F6F11028C00E9442
:10C5C000FC618A8D0E94AF618C0181E00E945C62F7
:10C5D000F801818354E6F52EF2828B8D0E94AF61C3
:10C5E0008C0182E00E945C62F8018183F2828C8D72
:10C5F0000E94AF618C0183E00E945C62F80181833C
:10C60000F2828D8D0E94AF618C0184E08AC0F1E0DE
:10C61000FF120EC08C8D0E94AF61FC0188E0818307
:10C620008CE98283F3828781897F84608783F2C16A
:10C6300082E0F81249C08C8D0E94AF61FC0118E0C5
:10C6400011833CE9E32EE28285E183838781897F40
:10C65000846087838EE00E94AF6102E2FC01018367
:10C6600044E6F42EF2828EE00E94AF61FC01118359
:10C67000E28284E183838781897F846087838EE07F
:10C680000E94AF61FC011183F28281E08383878184
:10C69000897F8460878383E00E945C6290915B0461
:10C6A000907F926090935B04809359048DE980930E
:10C6B0005A0480915E04807F816080935E040093C1
:10C6C0005C0410925D04A6C1F3E0FF1230C00E942A
:10C6D000FC61EA8C8E2D0E94AF618C0181E00E948A
:10C6E0005C62F801818324E6F22EF2828E2D0E9494
:10C6F000AF618C0182E00E945C62F80181838CE969
:10C700008283EB8C8E2D0E94AF618C0181E00E94B0
:10C710005C62F8018183F2828E2D0E94AF618C01F0
:10C7200082E00E945C62F8018183F28273C1F4E0CE
:10C73000FF1230C00E94FC61EB8C8E2D0E94AF6115
:10C740008C0182E00E945C62F801818394E6F92EFC
:10C75000F2828E2D0E94AF618C0184E00E945C62A7
:10C76000F8018183F282ED8C8E2D0E94AF618C01E5
:10C7700082E00E945C62F8018183F2828E2D0E9429
:10C78000AF618C0184E00E945C62F80181838CE9D6
:10C79000828340C1F5E0FF12D1C00E94FC610E947B
:10C7A000076281E00E94AF615AE0B52EFC01B182C0
:10C7B00064E6D62ED28282E00E94AF617BE0C72E73
:10C7C000FC01C182D28283E00E94AF61ECE0EE2ED8
:10C7D000FC01E182D28284E00E94AF618C0181E0A1
:10C7E0000E945C62F8018183D28285E00E94AF6181
:10C7F0008C0183E00E945C62F8018183D282A4E014
:10C80000AA2EA38287E0848387818160878385E065
:10C810000E94AF618C0183E00E945C62F801818319
:10C82000D282F382B8E08B2E8482878181608783F5
:10C8300085E00E94AF618C0183E00E945C62F80198
:10C840008183D28216E0D12ED38209E0902E948289
:10C8500087818160878385E00E94AF61FC018182CE
:10C860008CE9828381E083838781897F84608783E9
:10C8700086E00E94AF61FC0191828EE1828388EFA5
:10C8800083838BE00E94AF618C0183E00E945C6235
:10C89000F801818386E4982E9282A382B4828781F4
:10C8A000816087838BE00E94AF618C0183E00E94EE
:10C8B0005C62F80181839282F382C4828781816005
:10C8C00087838BE00E94AF618C0183E00E945C62F1
:10C8D000F80181839282D382E48287818160878399
:10C8E0008091FB018F7180628093FB018FE18093C7
:10C8F000FC01BE016B5E7F4F80E00E941662BE01AC
:10C90000605F7F4F81E00E941662BE01655F7F4FCE
:10C9100082E00E941662BE016A5F7F4F83E00E9440
:10C920001662BE016F5F7F4F84E00E941662BE01F7
:10C930006F5F7F4F85E00E9416626CC0F6E0FF12C9
:10C9400016C086E00E94AF61FC01F18282E382831F
:10C9500088EF838314E6108786E00E94AF61FC01B4
:10C96000F1828EEC828388E08383108753C087E056
:10C97000F81250C08FE00E94AF61FC0114E21183F5
:10C9800084E6828388E8868380E10E94AF61FC01AF
:10C9900089E081830EE602838AE0838380E10E943E
:10C9A000AF61FC0148E0F42EF18282E982838BE0E2
:10C9B00083838781897F8460878380E10E94AF6160
:10C9C000FC01F18202838CE083838781897F84600C
:10C9D000878380913D04807F8B6080933D0493E248
:10C9E00090933B0410933C0480914004807F8160CD
:10C9F0008093400490933E0489E680933F048091A5
:10CA00004304807F8260809343049093410487E9CC
:10CA10008093420482E00E9498570E9437586D9696
:10CA20000FB6F894DEBF0FBECDBFDF91CF911F913F
:10CA30000F91FF90EF90DF90CF90BF90AF909F90BD
:10CA40008F9008950F931F93CF93DF939091FB01E5
:10CA500091FF03C060E075E002C060E074E01091F7
:10CA6000F601129516951770882331F0AEEDBCE0F3
:10CA7000833021F420E103C0A6E9BCE028E09091D6
:10CA8000F501990F910F920F4091F80124E64202AF
:10CA9000A0011124485A5D4F0091FE01E8EEF3E039
:10CAA0009F010203E001039FD00D11249E01285332
:10CAB0003045241B350BFD01882339F032964D9308
:10CAC0005C93833011F418EF190FCC27DD27C61BB8
:10CAD000D70B1917F0F4A12FB0E0AA0FBB1FA55A6E
:10CAE000B84F0D90BC91A02D6A177B070CF4DB01A9
:10CAF000AC17BD070CF4DE01A854B44F2A1B3B0B46
:10CB0000A41BB50BB183A083538342831F5F34966C
:10CB1000E0CF31832083DF01882371F01296285EF5
:10CB200033403093920C2093910C1D921C92DF9114
:10CB3000CF911F910F910895149653834283F5CF9F
:10CB4000E0912601F091270129E090E130E0482FA3
:10CB50004170341302C0905F04C0915090833196AD
:10CB600090E186958068215011F0342FF0CF915FCD
:10CB70009193F0932701E093260108951F93CF939B
:10CB8000DF93182F26E93CE03093270120932601FC
:10CB9000C09114018C2F877461F08091F501882376
:10CBA00021F0813021F4C0E906C0C0E804C0C8E922
:10CBB00002C0C7FF06C087E10E94F460882309F421
:10CBC0005AC0C7FD5AC040E060E085E10E9495165A
:10CBD000882309F452C0C062C09314018091FF04FD
:10CBE0008F5F80931501E7E1F1E0ABE5B7E090E0FE
:10CBF0006DE0911729F14D915D91649F9001659FC2
:10CC0000300D112485E0359527958A95E1F73E5F33
:10CC100037FD06C02F3F83E038072CF4822F05C074
:10CC200080E030E002C08FEF33E0EF012197292F41
:10CC3000220F220F232B288380839F5F3296D9CF28
:10CC4000C4E1D1E089910E94A06581E0C232D80799
:10CC5000C9F7E0912601F0912701108231978FEFFB
:10CC6000808386E99CE09093250180932401DF91E5
:10CC7000CF911F910895CF77A4CFCF7DADCF1F92D5
:10CC80000F920FB60F9211242F938F939F93EF93D0
:10CC9000FF9388B391E0892788BBE0912401F0914C
:10CCA0002501CF01019690932501809324012081D5
:10CCB000822F90E097BD86BD293C08F0C09A8091F4
:10CCC000950C81608093950CFF91EF919F918F91CE
:10CCD0002F910F900FBE0F901F9018951F920F92DB
:10CCE0000FB60F9211242F933F938F939F93EF933F
:10CCF000FF9388B391E0892788BBE0912601F091EA
:10CD00002701808128B539B580FD03C0205E3F4FE3
:10CD100002C0205F3F4F39BD28BD90E095958795B3
:10CD2000009791F4CF0101969093270180932601FB
:10CD3000818181110AC0809178009091790080539F
:10CD4000984F99BD88BD01C080838091950C81600A
:10CD50008093950CFF91EF919F918F913F912F912F
:10CD60000F900FBE0F901F901895EDE7F0E08081B7
:10CD7000857E808317981F9AAAE8B0E01C921092D3
:10CD80008B0082E88C938081806280830895EDE738
:10CD9000F0E080818F7D8083179AAAE8B0E01C9232
:10CDA00010928B008AE08C93808188618083089543
:10CDB0001F920F920FB60F9211248F939F93EF93B0
:10CDC000FF938091260D882321F01F9A1092260D43
:10CDD00004C01F9881E08093260DE0911201F0912C
:10CDE00013018081918190938700809386008091C8
:10CDF000910C9091920C9093850080938400828195
:10CE00009381892B11F0329607C08091FB018170CC
:10CE10008093260DEEEDFCE0F0931301E0931201F8
:10CE20008091950C81608093950CFF91EF919F917B
:10CE30008F910F900FBE0F901F901895EAE8FCE0BD
:10CE4000208126952695282B208381818F5F8183E1
:10CE5000843048F0A281B381CD010196938382830F
:10CE60002C93108211820895882339F08091900CC0
:10CE70008F5F8093900C80E803C01092900C80EC40
:10CE80000E941E678091900C8530B8F70895CF936B
:10CE9000DF93C82FE0918E0CE827F0E0EE0FFF1F24
:10CEA000EB51F34E2591349140918F0C50E02427A3
:10CEB000352730938F0C20938E0CD8E08C2F807800
:10CEC0000E943467CC0FD150C9F7DF91CF910895FC
:10CED000CF9380EC0E941E67C6E080E80E941E6728
:10CEE000C150D9F780ECCF910C941E67EF92FF925E
:10CEF0000F931F93CF93DF93C091F40180911E0590
:10CF000085FF04C08091E1018111C4E08091940CFF
:10CF10008C1709F48EC0C093940C1EBC1DBC1CBCA5
:10CF200087B7837C87BF80917D008E7F80937D0053
:10CF30008CE386BF8FE380937C00C23079F118F4D4
:10CF4000C130A1F006C0C33009F444C0C43009F4B4
:10CF50005DC00E94B56680E49CE99BBD8ABD87B731
:10CF6000806187BF1FBC8AE08EBD63C00E94B5662A
:10CF700080E797E199BD88BD80EA9FE090937900B2
:10CF80008093780087B7886087BF80917D0081603B
:10CF900080937D001FBC82E08EBD56C00E94B566A6
:10CFA00088EC90E090937900809378008CE291E097
:10CFB0009DBD8CBD80EE9BEA97BD86BD87B7806224
:10CFC00087BF80917D00816080937D001FBC8AE1D6
:10CFD0008EBDB9C080E49CE99BBD8ABD87B78061E6
:10CFE00087BF1FBC8AE08EBD83E00E94226580E57A
:10CFF00093EC909387008093860088E893E1909368
:10D000008500809384000E94C766A7C084E00E94C8
:10D01000226580E593EC909387008093860088E8F2
:10D0200093E190938500809384000E94C766C09826
:10D030009DC0C13049F008F490C0C23009F483C0EB
:10D04000C33009F48AC092C07894EAE8FCE086E92B
:10D050009CE090932701809326019383828315821D
:10D0600014821082118216820E9468678091F501F5
:10D070000E9447678091930C0E94476780E00E945E
:10D0800047671092930CCBE5D7E028813981C9011D
:10D09000880F991F820F931F97FD03967C01F594CB
:10D0A000E794F594E79486E3E81A87EFF80A2A8173
:10D0B0003B81C901880F991F820F931F97FD03962B
:10D0C0008C0115950795159507950653174F8E2DCD
:10D0D0000E9447679F2D9F70802F8295807F892BAC
:10D0E0000E944767C80154E0969587955A95E1F7E5
:10D0F0000E944767249687E0CB36D80731F6C09167
:10D100008E0C80918F0C0E9447678C2F0E9447677E
:10D110000E94686780918B0C882321F080E00E9438
:10D120001E67F8CFE0918C0CF0918D0C10828091ED
:10D13000780090917900805C934690937900809379
:10D140007800C09A13C0789486E0DF91CF911F9148
:10D150000F91FF90EF900C94BE6580E0DF91CF912E
:10D160001F910F91FF90EF900C942265DF91CF916A
:10D170001F910F91FF90EF9008951F920F920FB69D
:10D180000F9211242F933F934F935F936F937F934D
:10D190008F939F93AF93BF93CF93DF93EF93FF93BF
:10D1A0008CB59DB52091270D222321F0C09A1092B5
:10D1B000270D04C0C09821E02093270DC0912201C3
:10D1C000D09123019E012E5F3F4F30932301209386
:10D1D0002201288139813BBD2ABDE0E1F1E0282F01
:10D1E0003181381708F481833081231708F4808354
:10D1F0008A819B81892BD9F486E99CE09093230155
:10D20000809322018091FB01809581708093270D8E
:10D2100087B78F7E87BF0E9476678091F40188234D
:10D2200011F0833021F487B7806187BF78948091B3
:10D23000950C81608093950CFF91EF91DF91CF91D8
:10D24000BF91AF919F918F917F916F915F914F911E
:10D250003F912F910F900FBE0F901F9018951F9226
:10D260000F920FB60F9211242F933F934F935F931A
:10D270006F937F938F939F93AF93BF93EF93FF939E
:10D280008091F4018230C1F480E492EA97BD86BDBA
:10D2900080917800909179008F3F910538F488E56E
:10D2A00098E9909379008093780008C088EC90E02A
:10D2B00090937900809378000E947667FF91EF91B8
:10D2C000BF91AF919F918F917F916F915F914F919E
:10D2D0003F912F910F900FBE0F901F9018951F92A6
:10D2E0000F920FB60F9211242F933F934F935F939A
:10D2F0006F937F938F939F93AF93BF93EF93FF931E
:10D300008091F40178949091940C981771F0943076
:10D3100061F48091E101882321F080911E0585FD53
:10D3200003C00E94766703C084E00E942265FF91DB
:10D33000EF91BF91AF919F918F917F916F915F918D
:10D340004F913F912F910F900FBE0F901F90189506
:10D35000909115059873903129F49BEA899F812D4E
:10D36000112402C0983111F486950895983211F471
:10D37000880F0895903319F4982F990F890F089505
:10D38000FC01A5E6B0E08C918B7F8C931482158212
:10D390001082118216A617A608950C94C06921E088
:10D3A000FC018481811101C020E0822F0895FC01DD
:10D3B00021818081281B277098E0921B81E09330A7
:10D3C00008F480E00895CF93DF93FC0184818823E3
:10D3D000F1F08150848382819381890F828386A5B5
:10D3E0008823F1F187A59FEF980F97A7882331F045
:10D3F0008091650084608093650032C080916500F3
:10D400008B7F809365008091200587A729C01B989A
:10D41000809165008B7F809365008581882319F05A
:10D42000815085831DC0808191818917C9F090E06A
:10D43000EF01C80FD91F2E8122832E8924832E85C8
:10D4400023832E8D258328A926A717A62EA13FEF7B
:10D45000320F3EA3211104C0019687709927808363
:10D46000DF91CF9108958F929F92AF92BF92CF920A
:10D47000DF92EF92FF920F931F93CF93DF935C01A4
:10D48000162FD42EF22E0E94D769882339F190915D
:10D490001505987319F1F501C181D0E04E01FFEF38
:10D4A0008F1A9F0A87E088229924F50180818815C8
:10D4B000A9F0112329F090911F05965F910F01C0EB
:10D4C00090E0CA0DDB1D9E838D2D0E94A8698E8B76
:10D4D000FE8EE8AA0EA3CE86F5018182DF91CF9160
:10D4E0001F910F91FF90EF90DF90CF90BF90AF9082
:10D4F0009F908F900895CF92DF92EF92FF920F93BB
:10D500001F93CF93DF93EC01162FF42ED22E0E949F
:10D51000D769882301F1909115059873E1F01123E3
:10D5200029F090911F05965F910F01C090E09A83BA
:10D530008F2D0E94A8698C83DD82EEA61FA6CB8268
:10D5400088818983002339F001502D2D4F2D612FC3
:10D55000CE010E94336ADF91CF911F910F91FF900E
:10D56000EF90DF90CF900895CF92EF920F931F939B
:10D57000CF93DF93EC01062F642F809115058695DC
:10D5800086958695877038812981321364C110E0B1
:10D590000132110508F05FC1F801ED58FF4F0C94FE
:10D5A0004173C12CEE24E39400E021E03AC1C12C88
:10D5B000EE24E39400E021E02EC1C12CEE24E3949C
:10D5C00000E021E04EE12EC192E0C92EEE24E3946A
:10D5D00002E022E04AE064E63BC1C12CEE24E39481
:10D5E0000AE022E045E06FE5CE010E94336A01E0E7
:10D5F0002AE045E06FE5CE010E94336A0AE022E0AE
:10D6000045E06FE525C1CC24CA94E12C02E023E07B
:10D610004AE060E5CE010E94336ACC24C39423E043
:10D620004AE06CE3CE010E94336AC12C82E0E82E0E
:10D6300000E021E04AE06FC0C12CEE24E39401E059
:10D6400021E045E066E4CE010E94336A22E04FE02B
:10D6500062E3CE010E94336A22E04FE0F8C0C12CA1
:10D66000EE24E39402E021E045E06EE6CE010E9464
:10D67000336A03E021E045E06CE7EAC0C12CE12C0D
:10D6800000E025E045E062E3CE010E94336A25E038
:10D6900045E06AE5CE010E94336A02E024E043E0FF
:10D6A0006EE6D6C0C12CEE24E39403E02AE045E008
:10D6B00060E5CE010E94336A01E024E145E060E5C7
:10D6C000CE010E94336A03E02AE045E0C0C0CC24CA
:10D6D000C394EE24E39402E025E044E16AE0B8C09C
:10D6E000C12CEE24E39402E02AE044E062E3CE01A0
:10D6F0000E94336A01E024E148E066E4CE010E9422
:10D70000336A02E02AE048E062E3CE010E94336A15
:10D7100001E024E144E066E49BC0C12CEE24E394E4
:10D720000AE02AE005C0C12CEE24E39402E022E3E3
:10D7300045E068E78DC0C12CEE24E39401E009C008
:10D74000C12CEE24E39402E004C0C12CEE24E39447
:10D7500003E02AE044E160E07BC0C12CEE24E394C6
:10D7600000E021E048E25EC0813009F474C0C12CC1
:10D77000E12C00E021E04AE06BE455C0813009F47F
:10D780006AC0C12CE12C00E021E04AE061E44BC01A
:10D79000C12CE12C00E021E046E045C0C12CEE2484
:10D7A000E39405C0813009F456C0C12CE12C00E09F
:10D7B00037C0C12CE12C00E004C0C12CEE24E3945E
:10D7C00001E021E04AE020C0C12CEE24E39402E015
:10D7D00021E04AE06AE727C0C12CEE24E39403E08D
:10D7E00021E04AE06CE71FC0C12CEE24E39403E083
:10D7F00009C0C12CEE24E39402E004C0C12CEE2445
:10D80000E39401E023E04FE068E70DC0C12CEE2473
:10D81000E39401E029E144E105C0C12CE12C02E0E0
:10D8200022E04AE066E4CE010E947B6A14C0CC2468
:10D83000C394E12C02E023E044E16CE3CE010E94BA
:10D84000336ACC24CA94EE24E39423E044E160E5F7
:10D85000CE010E94336ADF91CF911F910F91EF901B
:10D86000CF90089546E4682F8FE891E00C94B46A55
:10D870009091210591FF03C0862F0C94E6130C9420
:10D88000326CFF920F931F93CF93DF93EC01162F0F
:10D89000F42E47FF03C0842F0E94E613D7FF06C073
:10D8A000D195C195D1098AE10E94E613112371F047
:10D8B000123019F464E670E002C06AE070E0CE0154
:10D8C0000E94EC72262FC22FD72F082F64E670E03B
:10D8D000CE010E94EC729B01562F482FC82FD92FE2
:10D8E0002115310551F12A303105DCF06AE070E094
:10D8F000C9010E94EC729B018C01EC01653171053C
:10D900001CF48EE6820F05C08CE8820F0E94E113A2
:10D910008EE60E94E6130115110559F1502F11E012
:10D9200001C010E084E6850F0E94E613111121C0AA
:10D930002097F9F08C2F845715C08CE8840F0E9433
:10D94000E1131123B1F0123081F46AE070E0802F0E
:10D9500090E00E94EC72C82F86E0860F0E94E613CA
:10D960008CE88C0F0E94E11304C086E0800F0E94B7
:10D97000E6131F1444F48F2DDF91CF911F910F9167
:10D98000FF900C94E613DF91CF911F910F91FF90C0
:10D9900008951F920F920FB60F9211242F933F9369
:10D9A0004F935F936F937F938F939F93AF93BF93A7
:10D9B000CF93DF93EF93FF932CB18BB18C7161F018
:10D9C00010926D0D10926C0D10926B0D10926A0DED
:10D9D00081E08093700D20E08091700D90E0FC015B
:10D9E0003197E831F10508F006C1EC56FF4F0C9471
:10D9F0004173253299F038F4213271F0233209F065
:10DA0000FAC089E0C5C0203569F0283549F02B32CD
:10DA100009F0F1C086E0BCC083E0BAC08CE0B8C0B9
:10DA20008FE0B6C082E1B4C0213209F0B0C084E01A
:10DA3000AFC0213209F0ABC084E18093700D209318
:10DA40006E0D81E080936F0D80E0E82FF0E0E859E3
:10DA5000F24F10828F5F8230C0F37FC02B3209F00B
:10DA600096C087E095C02B3209F091C084E1809385
:10DA7000700D20936E0D81E080936F0D80E0E82F94
:10DA8000F0E0E859F24F10828F5F8230C0F365C03A
:10DA9000233209F07CC08AE07BC0233209F077C0D2
:10DAA00088E18093700D20936E0D81E080936F0D5F
:10DAB00080E0E82FF0E0E859F24F10828F5F82306B
:10DAC000C0F34BC0253209F062C08DE061C0253241
:10DAD00009F05DC088E18093700D20936E0D81E0A8
:10DAE00080936F0D80E0E82FF0E0E859F24F10824C
:10DAF0008F5F8230C0F331C0283509F048C080E123
:10DB000047C0283509F043C088E18093700D209309
:10DB10006E0D81E080936F0D80E0E82FF0E0E85912
:10DB2000F24F10828F5F8230C0F317C0203579F535
:10DB300083E12EC0203559F588E18093700D209344
:10DB40006E0D81E080936F0D80E0E82FF0E0E859E2
:10DB5000F24F10828F5F8230C0F38093710D4BC003
:10DB600085E116C086E114C087E112C02A3379F43A
:10DB700088E10EC02A3259F050916F0D2C3259F4C1
:10DB800084E18093700D5F5F50936F0D34C081E02E
:10DB90008093700D30C060916E0D30E07BE03230CC
:10DBA00040F5832F90E0FC01E659F24F4081641369
:10DBB0001EC0FC01E459F24F4081541318C0EC011F
:10DBC000C859D24F48814A3090F4789FF001799F2C
:10DBD000F00D1124DF01A40FB11DAE5AB24F2C93EA
:10DBE0004F5F4883E40FF11DEE5AF24F10823F5F02
:10DBF000D6CF3093710DFF91EF91DF91CF91BF910F
:10DC0000AF919F918F917F916F915F914F913F91D4
:10DC10002F910F900FBE0F901F9018951098189885
:10DC20001092900089E189B959981AB886E08093DA
:10DC300095005F9B02C08CB1FCCF08955398089566
:10DC4000539A089554985798089520E03BE0822F06
:10DC500090E0FC01E859F24F1082389FF001399FA3
:10DC6000F00D1124EE5AF24F1082FC01E659F24FEA
:10DC70001082FC01E459F24F108281E0820F823061
:10DC800010F4282FE4CF8093710D81E08093700D04
:10DC9000549A579A0895CF93C82F21E045EE5EE13C
:10DCA00060E080E00E943B5D21E04C2F60E086E672
:10DCB000CF910C94505CCF93DF9390E0EC01C65968
:10DCC000D24F2881DC01A459B24F261303C02C91F6
:10DCD000241791F02BE0289FF001299FF00D1124CB
:10DCE000EE5AF24F1082FC01E859F24F108268831D
:10DCF0004C9381E08093700DDF91CF910895813630
:10DD000091F038F48036A9F40E94226E8AEC9FE1EB
:10DD10000EC0823629F0833661F48AE790E707C0A7
:10DD200080ED9EE604C00E94226E80E69FE30E9482
:10DD3000B51341E061E280E00E945B6E42E061E287
:10DD400081E00E945B6E81E30E944B6E43EB5FE1DA
:10DD500068E08EE10E94615D8091520D882319F088
:10DD600042E55DE002C041E451E024E160E18CE085
:10DD70000E943B5D48EA5FE160E28EE10E94615DE6
:10DD800080915D0D882319F04DE55DE002C041E40E
:10DD900051E024E168E286E00C943B5D0C947F6ED8
:10DDA000823661F0833639F0813661F40E94226E4A
:10DDB00080E69FE305C08FE79EE602C087E19FE60D
:10DDC0000E94B51343E061E280E00E945B6E44E094
:10DDD00061E281E00E945B6E82E30E944B6E4AE941
:10DDE0005FE168E086E00E94615D8091520D8823CA
:10DDF00019F042E55DE002C041E451E024E160E158
:10DE00008CE00E943B5D4EE85FE160E286E00E94AC
:10DE1000615D80915D0D882319F04DE55DE002C0E4
:10DE200041E451E024E168E28CE00C943B5D8236F1
:10DE300061F0833639F0813661F40E94226E80E60B
:10DE40009FE305C080ED9EE602C08EE59FE60E943E
:10DE5000B51345E061E280E00E945B6E46E061E25E
:10DE600081E00E945B6E83E30E944B6E44E85FE1B9
:10DE700068E086E00E94615D8091520D882319F070
:10DE800042E55DE002C041E451E024E160E18CE064
:10DE90000E943B5D45E75FE160E286E00E94615DD4
:10DEA00080915D0D882319F04DE55DE002C041E4ED
:10DEB00051E024E168E28CE00C943B5D823661F035
:10DEC000833639F0813661F40E94226E80E69FE34A
:10DED00005C087E19FE602C085EA9FE60E94B51370
:10DEE00047E061E280E00E945B6E48E061E281E031
:10DEF0000E945B6E84E30E944B6E4DE65FE168E03A
:10DF000086E00E94615D8091520D882319F042E500
:10DF10005DE002C041E451E024E160E18CE00E9458
:10DF20003B5D44E65FE160E286E00E94615D8091D6
:10DF30005D0D882319F04DE55DE002C041E451E03C
:10DF400024E168E28CE00C943B5D823661F083361C
:10DF500039F0813661F40E94226E80E69FE305C0AD
:10DF60008EE59FE602C08CEE9FE60E94B51349E065
:10DF700061E280E00E945B6E4AE061E281E00E9423
:10DF80005B6E85E30E944B6E46E55FE168E086E0EC
:10DF90000E94615D8091520D882319F042E55DE099
:10DFA00002C041E451E024E160E18CE00E943B5D6D
:10DFB0004BE45FE160E286E00E94615D80915D0D6F
:10DFC000882319F04DE55DE002C041E451E024E111
:10DFD00068E28CE00C943B5D823661F0833639F068
:10DFE000813661F40E94226E80E69FE305C085EAD7
:10DFF0009FE602C083E390E70E94B51341E06BE225
:10E0000080E00E945B6E42E06BE281E00E945B6E0A
:10E0100086E30E944B6E4FE35FE168E086E00E947A
:10E02000615D8091520D882319F042E55DE002C0E8
:10E0300041E451E024E160E18CE00E943B5D42E379
:10E040005FE160E286E00E94615D80915D0D882362
:10E0500019F04DE55DE002C041E451E024E168E2E1
:10E060008CE00C943B5D823661F0833639F081366A
:10E0700061F40E94226E80E69FE305C08CEE9FE66D
:10E0800002C08AE790E70E94B51343E06BE280E0AC
:10E090000E945B6E44E06BE281E00E945B6E87E36E
:10E0A0000E944B6E46E25FE168E086E00E94615D9F
:10E0B0008091520D882319F042E55DE002C041E4F1
:10E0C00051E024E160E18CE00E943B5D49E15FE1C9
:10E0D00060E286E00E94615D80915D0D882319F009
:10E0E0004DE55DE002C041E451E024E168E28CE0EE
:10E0F0000C943B5D823661F0833639F0813661F4F1
:10E100000E94226E80E69FE305C083E390E702C091
:10E110008FE79EE60E94B51341E063E280E00E9433
:10E120005B6E41E065E281E00E945B6E88E30E94E5
:10E130004B6E49E05FE168E086E00E94615D80919E
:10E14000520D882319F042E55DE002C041E451E040
:10E1500024E160E18CE00E943B5D4BEF5EE160E218
:10E1600086E00E94615D80915D0D882319F04DE588
:10E170005DE002C041E451E024E168E28CE00C94EF
:10E180003B5D86B380958E7708958FEF8ABB1BBA6F
:10E1900091E897BB9EE798BB9EE394BB91EC95BB3F
:10E1A00011BA82BB88E082B987EF83B9109261000F
:10E1B0001092620084E1809364008BEF809365008D
:10E1C0000E94C35F0E940E6E80E487B985E886B91D
:10E1D00087E083BF8CE981BF82E085BD87B7836418
:10E1E00087BF1FBC8AE08EBD10928B0082E88093AF
:10E1F0008A0080917D00806280937D00789480E623
:10E200009FE3909367018093660189E10E94036018
:10E210000E942657D090FF040E94C170C0E081FD8B
:10E2200005C08695CF5FC730D1F71FC0C630E9F073
:10E230008C2F0E9497568823C1F0C093FF048C2F27
:10E240000E949A5681E00E9498570E94005C24E048
:10E2500049ED51E060E086E10E943B5D88E10E946B
:10E2600013120E9416600E94DA110E94126081E06F
:10E27000809356010E94B517109256010E94E9132F
:10E280008091180584FF05C08091150582FD4FC05F
:10E2900044C080912105882321F06CE187E00E9431
:10E2A000386C0E9494170E94005C20E048EA53E01A
:10E2B00060E080E00E940B5C80911E0584FD08C038
:10E2C00000E12AE043E255E068E380E00E94055D5A
:10E2D0000E9416600E9412600E94DA110E940A10C9
:10E2E0000E94DC148C01F894C0915A0CD0915B0C04
:10E2F0007894C057DE4F0E9416600E9494170E94C7
:10E300000A100E94DC147C010E94C1708111BCCFF4
:10E31000E016F10609F4F9C0B7CF0E94AB58883C6B
:10E32000910528F460E08AEC91E00E94CC1A0E94EA
:10E330000A108091150580FD39C080911605817005
:10E3400012E0181B0E940A10E12FF0E0EE0FFF1FF1
:10E35000EE52FB4F218132818091180580FF06C06B
:10E36000319521953109458D568D02C047855089DB
:10E37000241B350BE9016096812F0E94F614C81703
:10E38000D907A4F46BEB71E089EA91E00E94E111F6
:10E390000E940A100E949417812F0E94F614C81739
:10E3A000D90724F40E94C170882391F3D0912D05E0
:10E3B0008091150581FD56C08D2F8873883041F0FE
:10E3C000803131F0803221F0D77CD860D0932D0598
:10E3D00016E1C0E0812F0E94F460CC0FC82B1150D1
:10E3E0001E30C1F71C2F1D2763E971E08DEA92E111
:10E3F0000E94E11110FF04C060E082E00E94071259
:10E4000011FF04C063E087E10E94071212FF04C0FD
:10E4100066E08CE20E940712812F887371F0C3FFBF
:10E4200002C069E007C0C4FF02C06CE003C0C5FFC2
:10E4300004C06FE081E40E94071216FF04C062E18D
:10E4400086E50E94071217FF04C065E18BE60E9473
:10E4500007120E941660CD1729F00E94C170882310
:10E4600009F45EC080911505887B29F460E083E89B
:10E4700091E00E94CC1A80918E01882351F060E0D7
:10E4800088E591E00E94CC1A80918E018E7F809366
:10E490008E010E94DA1180EF90E090930101809349
:10E4A00000018091EF010E94E1130E9476672DE048
:10E4B00088E190E00FB6F894A89581BD0FBE21BD0C
:10E4C00060E08BE597E00E94913681E690E39093BF
:10E4D0006901809368010E9412608091FF04D81640
:10E4E00029F081E00E9498570E94375880ED97E00C
:10E4F0009BBD8ABD80E186BF81E08093E20187B742
:10E50000806187BF0E946F1BFDCFF89480915A0CE9
:10E5100090915B0C7894C817D90709F0ECCEB4CE73
:10E520000E94941755CF8FE891E00C94CD690E941A
:10E530009F72332312F48A1B9B0B0C94B072A29F20
:10E54000B001B39FC001A39F700D811D1124911DC7
:10E55000B29F700D811D1124911D08950E949F721C
:10E56000B7FF0895821B930B08950E949F72A59F89
:10E57000900DB49F900DA49F800D911D11240895BE
:10E58000B7FF0C94B5720E94B572821B930B08956D
:10E59000DB018F939F930E94B572BF91AF91A29FB1
:10E5A000800D911DA39F900DB29F900D1124089591
:10E5B000AA1BBB1B51E107C0AA1FBB1FA617B707A9
:10E5C00010F0A61BB70B881F991F5A95A9F78095C5
:10E5D0009095BC01CD01089597FB072E16F4009489
:10E5E00007D077FD09D00E94D87207FC05D03EF411
:10E5F000909581959F4F0895709561957F4F0895EF
:10E60000A1E21A2EAA1BBB1BFD010DC0AA1FBB1F36
:10E61000EE1FFF1FA217B307E407F50720F0A21BA8
:10E62000B30BE40BF50B661F771F881F991F1A9415
:10E6300069F760957095809590959B01AC01BD013F
:10E64000CF010895052E97FB1EF400940E943973A4
:10E6500057FD07D00E94007307FC03D04EF40C94C2
:10E66000397350954095309521953F4F4F4F5F4FEF
:10E67000089590958095709561957F4F8F4F9F4F2E
:10E680000895EE0FFF1F0590F491E02D0994FB0112
:10E69000DC014150504048F005900D920020C9F730
:10E6A00001C01D9241505040E0F708956817790766
:10E6B00068F4FB01DC01E40FF51FA40FB51F02C0D5
:10E6C00002900E9241505040D8F708950C947F73F9
:10E6D000DC0101C06D9341505040E0F70895DC012A
:10E6E000CB01FC01E199FECF06C0FFBBEEBBE09A77
:10E6F00031960DB20D9241505040B8F70895FB018C
:10E70000DC0102C001900D9241505040D8F70895AD
:04E71000F894FFCFAB
:10E71400F0004AC703C803C903CA036400000A021D
:10E72400FF00DE0CFF0000AA05FF09FF0DFF1354D4
:10E7340014AA960C960C960C9CEC1E465A50463C19
:10E744004664645A505A64E2F10032649CCE00324A
:04E75400643F00001E
:00000001FF
